:100000000C9421110C9452110C9452110C94521115
:100010000C9452110C9452110C9452110C945211D4
:100020000C9452110C9452110C9452110C945211C4
:100030000C9452110C9452110C9452110C945211B4
:100040000C9452110C94254B0C9452110C94521197
:100050000C9452110C9452110C9474C30C9418DC2F
:100060000C9452110C942CDA0C9452110C945211E1
:100070000C9452110C9452110C9452110C94521174
:100080000C942C530C9452110C9452110C94521148
:100090000C9452110C9452110C9452110C94521154
:1000A0000C9452110C9452110C94FE520C94521157
:1000B0000C9452110C9452110C9452110C94D05275
:1000C0000C9452110C9452110C9452110C9480C245
:1000D0000C9457C20C9452110C9452110C9452115E
:1000E0000C945211BB2CB42EED30942FC449C4494A
:1000F00026348E34DA34C449C4491737BB39893AB7
:10010000C449BA3CC449C4490F3EC449C4494841E2
:10011000C74139440846974695DA98DA87DA8BDA88
:1001200091DACFDA9CDAA0DAA6DAAADAAEDAB4DAB1
:10013000B8DABCDACFDAC2DAC6DACADA34DB39DBEB
:100140003EDB48DB52DBCBDB5CDB64DB6CDB76DB92
:1001500080DB8ADB99DBA3DBCBDBADDBB7DBC1DB91
:10016000084AD73B3BCE016E84BCBFFDC12F3D6C1E
:1001700074319ABD56833DDA3D00C77F11BED9E484
:10018000BB4C3E916BAAAABE000000803F05A84C64
:10019000CDB2D44EB93836A9020C50B99186880830
:1001A0003CA6AAAA2ABE000000803F004E414E494C
:1001B0004E495459494E46CDCCCC3D0AD7233C1725
:1001C000B7D13877CC2B329595E6241FB14F0A0072
:1001D0000020410000C84200401C4620BCBE4CCA62
:1001E0001B0E5AAEC59D7400407A10F35A00A072DF
:1001F0004E18090010A5D4E80000E8764817000062
:10020000E40B54020000CA9A3B000000E1F505002F
:100210000080969800000040420F000000A0860178
:10022000000000102700000000E803000000006448
:1002300000000000000A00000000000100000000B3
:10024000002C76D888DC674F0823DFC1DFAE59E188
:10025000B1B796E5E3E453C63AE651997696E8E6F7
:10026000C28426EB898C9B62ED407C6FFCEFBC9CCA
:100270009F40F2BAA56FA5F490055A2AF75C936BDC
:100280006CF9676DC11BFCE0E40D47FEF520E6B597
:1002900000D0ED902E0300943577050080841E0871
:1002A0000000204E0A000000C80C333333330F988F
:1002B0006E12831141EF8D2114893BE65516CFFE56
:1002C000E6DB18D1844B381BF77C1D901DA4BBE4E2
:1002D00024203284725E228100C9F124ECA1E53D24
:1002E00027434F4D4D554E49434154494F4E0044CD
:1002F000525952554E004552524F525300494E46A4
:100300004F004543484F0047322F47332062616416
:1003100020706172616D65746572730A005A207095
:10032000726F6265206F75742E206265640A0047E3
:100330003238205A20466F7262696464656E0A0022
:1003400047323900205A3A200020593A20004265AD
:100350006420583A20004D65736820706F696E7490
:100360002063616E6E6F74206265207265736F6CBE
:100370007665640A00456E642066696C65206C6968
:1003800073740A00426567696E2066696C65206C4B
:100390006973740A002E0A0046696C652862696EEA
:1003A000292064656C657465640044656C657469D6
:1003B0006F6E2862696E29206661696C65640053FE
:1003C00044207072696E74696E672062797465206A
:1003D000004E6F74205344207072696E74696E67AA
:1003E0000A002569730025696D2025697300256958
:1003F000682025696D2025697300256964202569B9
:10040000682025696D202569730025697920256993
:1004100064202569682025696D2025697300507264
:10042000696E742074696D653A200050726F74654E
:10043000637465642050696E0A000203FD02F602CF
:10044000EF02E1026F66660044454255473A004BB1
:10045000494C4C45442E20004D3131332053006F20
:100460006B002F2F200053657474696E67205472DF
:100470006176656C20416363656C65726174696F58
:100480006E3A200053657474696E67205265747209
:1004900061637420416363656C65726174696F6E3A
:1004A0003A200053657474696E67205072696E74E7
:1004B00020416363656C65726174696F6E3A2000F8
:1004C00053657474696E67205072696E7420616E32
:1004D000642054726176656C20416363656C65725B
:1004E0006174696F6E3A20000001363726FF033CC5
:1004F0003D38FF0E2E303E12FFFF0C0809FFFFFFB4
:100500001A1C18FFFF08440AFF43FFFFFFFFFFFF0D
:10051000206F7574206F662072616E67650A0053E4
:100520006572766F20003A200020536572766F2046
:100530000043290A0061626C656420286D696E20A1
:1005400074656D702000436F6C64206578747275FB
:10055000646573206172652000546F6F206661725C
:100560002066726F6D207265666572656E636520C8
:10057000706F696E740A00207A70726F62655F7ABC
:100580006F66667365743D20007A5F6D696E3A2010
:10059000202D3230207A5F6D61783A202032300091
:1005A0005A204F666673657420004E6F2063617336
:1005B00065206C696768740A004163746976652018
:1005C00045787472756465723A2000556E6B6E6F73
:1005D000776E20636F6D6D616E643A2022004D323C
:1005E00034004D3233202573004D313036205332E4
:1005F0003535004D31303920532569004D313930C2
:1006000020532569004739322045257300473020A3
:100610005A2573004D31303920532569004D313949
:100620003020532569004D323400473238004D34B4
:100630003230205330004D343230205331004731B6
:100640002046313030205A30004731205835302094
:100650005933303020463336303000473120463170
:100660003030205A330047312046313030205A3064
:100670000047312058333030205933303020463352
:100680003630300047312046313030205A33004771
:10069000312046313030205A300047312058333035
:1006A000302059353020463336303000473120462F
:1006B000313030205A330047312046313030205A13
:1006C00030004731205835302059353020463336F8
:1006D00030300047312046313030205A3300473126
:1006E0002046313030205A300047312058313830E0
:1006F00020593138302046333630300047312046DB
:10070000313030205A330047323900473930004702
:10071000323800473238205A3000473238004D38DE
:10072000340047312046323030205A302E300047D6
:1007300032380047393220452573004730205A258A
:1007400073004D31303920532569004D3139302047
:10075000532569004732382058302059300047323D
:1007600038205830205930004D3432302053310079
:100770004D343230205330002020506C616E6E6555
:100780007242756666657242797465733A2000201C
:1007900046726565204D656D6F72793A2000436F32
:1007A0006D70696C65643A204A616E203137203281
:1007B0003032300A00207C20417574686F723A2014
:1007C000456E6465722D3520506C75730A003230A9
:1007D00031392D30392D303400204C61737420555F
:1007E0007064617465643A200056657220312E375A
:1007F000302E3220424C0A004D61726C696E00202E
:10080000536F6674776172652052657365740A0070
:10081000205761746368646F672052657365740A5A
:10082000002042726F776E206F7574205265736579
:10083000740A002045787465726E616C205265738D
:1008400065740A00506F77657255700A00737461A1
:1008500072740A006572726F722077726974696EC1
:100860006720746F2066696C650A00205A3A002080
:10087000593A0020583A00656E6473746F707320A3
:100880006869743A2000446F6E6520736176696E02
:10089000672066696C652E0A004D32390024F4D455
:1008A0003050C38E20C2A24017828B7011127A91F1
:1008B0000D816CD90AA861E108C7586607615143E8
:1008C000061E4B5D05C145A7041A411104093D9858
:1008D00003713931034036DB0265339102D4305461
:1008E00002802E1D02632CEE01752AC501B028A0DE
:1008F00001102781018F2564012B244B01E0223454
:1009000001AC211F018D200D01801FFC00841EED14
:1009100000971DDF00B81CD200E61BC600201BBCE0
:1009200000641AB200B219A8000A19A0006A189946
:1009300000D117910040178B00B516840031167E48
:1009400000B31579003A157300C7146F0058146A84
:1009500000EE1366008813630025135E00C7125B68
:10096000006C12570015125400C111510070114F44
:100970000021114B00D61049008D1047004610444D
:100980000002104200C00F4000800F3E00420F3CAA
:1009900000060F3B00CB0E3800930E37005C0E357F
:1009A00000270E3400F30D3200C10D3100900D30E0
:1009B00000600D2E00320D2D00050D2C00D90C2BE2
:1009C00000AE0C2900850C29005C0C2700350C2793
:1009D000000E0C2600E80B2400C40B2400A00B23FF
:1009E000007D0B23005A0B2100390B2100180B202E
:1009F00000F80A1F00D90A1E00BB0A1E009D0A1D2E
:100A000000800A1D00630A1C00470A1B002C0A1BF9
:100A100000110A1A00F7091A00DD091900C40919A2
:100A200000AB091900920917007B09180063091728
:100A3000004C09160036091600200916000A09158F
:100A400000F5081500E0081400CC081400B80814DC
:100A500000A4081400900813007D0812006B08130E
:100A6000005808120046081200340811002308112B
:100A7000001208110001081100F0071000E0071033
:100A800000D0071000C0071000B0070F00A107102A
:100A90000091070E0083070F0074070F0065070E13
:100AA0000057070E0049070E003B070D002E070EEA
:100AB0000020070D0013070D0006070D00F9060CB6
:100AC00000ED060D00E0060C00D4060C00C8060C74
:100AD00000BC060C00B0060C00A4060B0099060C26
:100AE000008D060B0082060B0077060B006C060BD0
:100AF0000061060A0057060B004C060A0042060A6F
:100B00000038060A002E060A0024060A001A060A01
:100B1000001006090007060A00FD050900F4050992
:100B200000EB050900E2050900D9050900D0050917
:100B300000C7050900BE050900B5050800AD050898
:100B400000A50509009C050800940508008C05080F
:100B500000840508007C050800740508006C050782
:100B600000650508005D050700560508004E0507ED
:100B70000047050700400508003805070031050754
:100B8000002A050700230507001C050600160507B7
:100B9000000F0507000805060002050700FB040614
:100BA00000F5040700EE040600E8040600E204076E
:100BB00000DB040600D5040600CF040600C90406C5
:100BC00000C3040600BD040600B7040600B1040516
:100BD00000AC040600A6040600A00405009B040661
:100BE0000095040500900406008A040500850405AC
:100BF00000800406007A04050075040500700405F1
:100C0000006B04050066040500610405005C040532
:100C10000057040500520405004D04050048040572
:100C200000430405003E0404003A040500350405B1
:100C300000300404002C04050027040400230405EC
:100C4000001E0404001A0404001604050011040424
:100C5000000D040400090405000404040000040459
:100C600000FC030400F8030400F4030400F0030490
:100C700000EC030400E8030400E4030400E00304C0
:100C800000DC030400D8030400D4030400D00304F0
:100C900000CC030400C8030300C503030024F404CC
:100CA000D9201BC40C5C0E9804C4095F026507714F
:100CB00001F405F900FB04B30048048700C103698F
:100CC000005803550003034500BE023A0084023178
:100CD0000053022A002902250004022000E4011C1E
:100CE00000C8011900AF0117009801140084011316
:100CF00000710110006101100051010E0043010D4F
:100D00000036010B002B010B0020010B001501091F
:100D1000000C01090003010800FB000800F30008B3
:100D200000EB000700E4000600DE000600D8000625
:100D300000D2000600CC000500C7000500C2000577
:100D400000BD000400B9000400B5000400B10004B7
:100D500000AD000400A9000400A5000300A20003E8
:100D6000009F0004009B0003009800030095000210
:100D70000093000300900003008D0002008B00032D
:100D80000088000200860002008400030081000247
:100D9000007F0002007D0002007B0002007900025B
:100DA000007700010076000200740002007200016A
:100DB00000710002006F0002006D0001006C000273
:100DC000006A00010069000200670001006600017E
:100DD0000065000100640002006200010061000182
:100DE00000600001005F0002005D0001005C000186
:100DF000005B0001005A0001005900010058000189
:100E00000057000100560001005500010054000188
:100E10000053000000530001005200010051000186
:100E200000500001004F0001004E0000004E000184
:100E3000004D0001004C0001004B0000004B000180
:100E4000004A00010049000100480000004800017C
:100E50000047000100460000004600010045000078
:100E60000045000100440001004300000043000170
:100E7000004200000042000100410000004100016A
:100E800000400001003F0000003F0001003E000064
:100E9000003E0001003D0000003D0001003C00005C
:100EA000003C0000003C0001003B0000003B000152
:100EB000003A0000003A000100390000003900014A
:100EC0000038000000380000003800010037000042
:100ED0000037000100360000003600000036000137
:100EE000003500000035000000350001003400002E
:100EF0000034000000340001003300000033000023
:100F00000033000100320000003200000032000116
:100F1000003100000031000000310001003000000D
:100F20000030000000300001002F0000002F000002
:100F3000002F0000002F0001002E0000002E0000F6
:100F4000002E0001002D0000002D0000002D0000EB
:100F5000002D0001002C0000002C0000002C0000DF
:100F6000002C0001002B0000002B0000002B0000D3
:100F7000002B0001002A0000002A0000002A0000C7
:100F8000002A0001002900000029000000290000BB
:100F900000290000002900010028000000280000AE
:100FA00000280000002800000028000100270000A1
:100FB0000027000000270000002700000027000194
:100FC0000026000000260000002600000026000089
:100FD000002600010025000000250000002500007B
:100FE000002500000025000000250001002400006D
:100FF0000024000000240000002400000024000160
:101000000023000000230000002300000023000054
:101010000023000000230000002300010022000044
:101020000022000000220000002200000022000038
:10103000002200010021000000210000002100002A
:10104000002100000021000000210000002100011B
:101050000020000000200000002000000020000010
:1010600000200000002000000020000000200001FF
:10107000001F0000001F0000001F0000001F0000F4
:10108000001F0000001F0000001F0001001E0000E4
:10109000001E0000001E0000001E0000004D38343D
:1010A00020582059205A20450047302046333630FA
:1010B00030205831383020593138300042696C695D
:1010C0006E656172204C6576656C696E672047724B
:1010D00069643A0A0020706F736974696F6E206FDB
:1010E0007574206F662072616E67652E0A003F502E
:1010F000726F626520002066697273740A005A007C
:1011000059005800486F6D65200052756E6E696E0B
:101110006720696E204452592D52554E206D6F64E0
:10112000650A00473239204175746F20426564209A
:101130004C6576656C696E670A0028422961636BAD
:1011400000284629726F6E740028522969676874F6
:1011500000284C29656674003F2856296572626F25
:101160007365206C6576656C20697320696D706CA1
:1011700061757369626C652028302D34292E0A0050
:10118000426164205A2076616C75650A004E6F20BA
:1011900062696C696E65617220677269640A0046F3
:1011A000696C652064656C657465643A0044656CBF
:1011B0006574696F6E206661696C65642C20466990
:1011C0006C653A20006F70656E206661696C6564BD
:1011D0002C2046696C653A2000202F002042403ABE
:1011E0000020403A00473238205830205930002043
:1011F000573A004732382058302059300020573AAB
:1012000000205A3A0020593A0020436F756E74202E
:10121000583A0020453A00205A3A0020593A0058DE
:101220003A002E0A006F70656E206661696C656415
:101230002C2046696C653A200057726974696E67A4
:1012400020746F2066696C653A2000534420636106
:101250007264206F6B0A006F70656E526F6F74203E
:101260006661696C65640A00766F6C756D652E69E0
:101270006E6974206661696C65640A004572726FFC
:10128000723A00534420696E6974206661696C0A81
:10129000004D3234004D3233202573006175746F78
:1012A00025692E6700656E7175657565696E6720C5
:1012B00022006563686F3A004B494C4C45442E2030
:1012C000005072696E7465722073746F707065641B
:1012D0002064756520746F206572726F72732E20A2
:1012E00046697820746865206572726F7220616E3D
:1012F0006420757365204D39393920746F2072650B
:1013000073746172742E202854656D7065726174F7
:101310007572652069732072657365742E2053653C
:1013200074206974206166746572207265737461DB
:101330007274696E67290A004E6F204C696E6520D1
:101340004E756D62657220776974682063686563A5
:101350006B73756D2C204C617374204C696E653A0B
:1013600020004E6F20436865636B73756D2077694D
:101370007468206C696E65206E756D6265722C20D4
:101380004C617374204C696E653A20006368656334
:101390006B73756D206D69736D617463682C204C7F
:1013A000617374204C696E653A20004C696E65204B
:1013B0004E756D626572206973206E6F74204C618A
:1013C0007374204C696E65204E756D6265722B31A9
:1013D0002C204C617374204C696E653A20004D31AD
:1013E0003130004D3331004D383420582059205AC7
:1013F00020450053442072656164206572726F72EB
:101400000A00446F6E65207072696E74696E6720A1
:1014100066696C650A0020496E76616C69642065B6
:10142000787472756465722000000000000000008E
:1014300000000000000000B4430000B4430000CDF1
:10144000435072696E7465722073746F7070656456
:101450002064756520746F206572726F72732E2020
:1014600046697820746865206572726F7220616EBB
:101470006420757365204D39393920746F20726589
:1014800073746172742E202854656D706572617476
:101490007572652069732072657365742E205365BB
:1014A000742069742061667465722072657374615A
:1014B0007274696E67290A0053544F502063616C3F
:1014C0006C65642062656361757365206F66204298
:1014D0004C546F756368206572726F72202D207294
:1014E0006573746172742077697468204D39393975
:1014F0000A0020746F6F206C6F6E672065787472BD
:101500007573696F6E2070726576656E7465640AB6
:101510000020636F6C6420657874727573696F6EF8
:101520002070726576656E7465640A0020204D38FF
:101530003531205A005A2D50726F6265204F666611
:1015400073657420286D6D293A0A002044002049F3
:101550000020204D33303120500050494420736525
:101560007474696E67733A0A00205A0020204D3463
:1015700032302053004175746F20426564204C6501
:1015800076656C696E673A0A00205A00205900207F
:10159000204D323036205800486F6D65206F6666EA
:1015A0007365743A0A00204500205A002059002033
:1015B000580020420020540020204D323035205366
:1015C00000416476616E6365643A20533C6D696ED8
:1015D0005F66656564726174653E20543C6D696E3A
:1015E0005F74726176656C5F66656564726174656F
:1015F0003E20423C6D696E5F7365676D656E745F1A
:1016000074696D655F6D733E20583C6D61785F78DD
:10161000795F6A65726B3E205A3C6D61785F7A5FD4
:101620006A65726B3E20453C6D61785F655F6A65F7
:10163000726B3E0A0020540020520020204D3230B0
:1016400034205000416363656C65726174696F6E2C
:101650002028756E6974732F7332293A20503C70BC
:1016600072696E745F616363656C3E20523C7265A3
:1016700074726163745F616363656C3E20543C7493
:10168000726176656C5F616363656C3E0A0020453C
:1016900000205A0020590020204D323031205800BF
:1016A0004D6178696D756D20416363656C6572612C
:1016B00074696F6E2028756E6974732F7332293ABE
:1016C0000A00204500205A0020590020204D3230C9
:1016D000332058004D6178696D756D2066656564CD
:1016E00072617465732028756E6974732F73293A5B
:1016F0000A00204500205A0020590020204D393290
:1017000020580053746570732070657220756E697F
:10171000743A0A0020204D3230302044300A002034
:10172000204D3230302044002044697361626C6582
:10173000640A0046696C616D656E7420736574742B
:10174000696E67733A0020204D3134392043203BC5
:1017500020556E69747320696E2043656C736975DA
:10176000730A002020473231202020203B20556E74
:1017700069747320696E206D6D0A007A5F6D696E01
:101780003A2000795F6D61783A2000785F6D61786A
:101790003A20005265706F7274696E6720656E64DE
:1017A00073746F70207374617475730A0043617091
:1017B0003A454D455247454E43595F504152534576
:1017C000523A300A004361703A434153455F4C49F5
:1017D0004748545F4252494748544E4553533A3064
:1017E0000A004361703A544F47474C455F4C4947A4
:1017F0004854533A300A004361703A534F465457A5
:101800004152455F504F5745523A300A004361708C
:101810003A4C4556454C494E475F444154413A3154
:101820000A004361703A5A5F50524F42453A310ABA
:10183000004361703A4155544F4C4556454C3A313E
:101840000A004361703A5052494E545F4A4F423A3F
:10185000310A004361703A50524F47524553533A50
:10186000300A004361703A4155544F5245504F522F
:10187000545F54454D503A310A004361703A454532
:1018800050524F4D3A310A004649524D5741524548
:101890005F4E414D453A4D61726C696E20566572DE
:1018A00020312E37302E3220424C20284372656181
:1018B0006C69747933442920534F555243455F4333
:1018C0004F44455F55524C3A68747470733A2F2FE9
:1018D0006769746875622E636F6D2F4D61726C69F4
:1018E0006E4669726D776172652F4D61726C696EBB
:1018F0002050524F544F434F4C5F56455253494F1F
:101900004E3A312E30204D414348494E455F54599F
:1019100050453A456E6465722D3520506C757320C4
:1019200045585452554445525F434F554E543A31F1
:1019300020555549443A63656465326132662D34F9
:101940003161322D343734382D396231322D6335DF
:10195000356336326633363766660A00205A002011
:101960005900580020204D61783A2000205A00206C
:101970005900580020204D696E3A20004F6E20001B
:101980004F666600536F667420656E6473746F7083
:10199000733A200020643A0020693A0020703A002F
:1019A00023646566696E65202044454641554C5464
:1019B0005F4B64200023646566696E6520204445A2
:1019C0004641554C545F4B69200023646566696E3F
:1019D00065202044454641554C545F4B70200050D3
:1019E0004944204175746F74756E652066696E692F
:1019F00073686564212050757420746865206C617B
:101A00007374204B702C204B6920616E64204B64F2
:101A100020636F6E7374616E74732066726F6D20D5
:101A200062656C6F7720696E746F20436F6E6669B4
:101A30006775726174696F6E2E680A0050494420A0
:101A40004175746F74756E65206661696C6564219B
:101A50002074696D656F75740A00504944204175A2
:101A6000746F74756E65206661696C6564212054BD
:101A7000656D706572617475726520746F6F206832
:101A80006967680A00204B643A2000204B693A20BD
:101A900000204B703A20000A20436C617373696325
:101AA00020504944200A002054753A2000204B75EC
:101AB0003A2000206D61783A2000206D696E3A204E
:101AC0000020643A200020626961733A20004F666A
:101AD000660A00466164652048656967687420008D
:101AE000426564204C6576656C696E6720004661CE
:101AF000696C656420746F20656E61626C6520425C
:101B00006564204C6576656C696E670A004D657387
:101B10006820706F696E742063616E6E6F742062EE
:101B200065207265736F6C7665640A004D343231DE
:101B300020696E636F727265637420706172616D8B
:101B4000657465722075736167650A000000220084
:101B5000250028002B002E00310034000201000077
:101B6000050108010B0100002000230026002900C8
:101B70002C002F00320000010000030106010901C2
:101B800005050505070508080808020202020A0AF9
:101B90000808040404040101010101010101030317
:101BA000030303030303040707070C0C0C0C0C0CC2
:101BB0000C0C0202020206060606060606060B0BBF
:101BC0000B0B0B0B0B0B0102102020080810204000
:101BD00010204080020102010804020101020408F1
:101BE000102040808040201008040201800402017F
:101BF00080402010080402010804020101020408C8
:101C000010204080010204081020408000000A0BD0
:101C100002090C0D0E08070304010000000000007B
:101C200000000000000000000000000000000000B4
:101C30000000000000000000121110000000000071
:101C40000000000000000000000000000000000094
:101C5000000050726F62696E67206661696C65642E
:101C60000A00205A3A200020593A20004265642098
:101C7000583A2000290A002062797465733B20637A
:101C80007263200053657474696E67732053746FB8
:101C9000726564202800202863616C63756C617430
:101CA000656429210A0020213D2000454550524FFE
:101CB0004D20435243206D69736D61746368202D1C
:101CC000202873746F726564292000290A0020623D
:101CD000797465733B2063726320002073746F72A4
:101CE00065642073657474696E67732072657472BD
:101CF0006965766564202800204D61726C696E3DCF
:101D0000563431290A0028454550524F4D3D004573
:101D10004550524F4D2076657273696F6E206D6924
:101D2000736D61746368200048617264636F6465F9
:101D3000642044656661756C742053657474696EC3
:101D40006773204C6F616465640A00F4010000F45D
:101D500001000064000000E803000000009643005A
:101D60000096430000A0400000C8410000A04200CF
:101D700000A042000048440000BA425072696E74EC
:101D800065722068616C7465642E206B696C6C28C8
:101D9000292063616C6C6564210A000000B4430073
:101DA00000B4430000000000004842000048420028
:101DB000008040000000005761726E696E673A2033
:101DC000486F6D696E672042756D70204469766951
:101DD000736F72203C20310A000202040000A04010
:101DE0000000A040000000400000B4430000B443E5
:101DF0000000CD430101FF62696E004D3131372093
:101E0000494E56414C494420444154412E004739E3
:101E100032205A2573204525730062696E00526591
:101E200073656E643A20006F6B0020746F6F206CD6
:101E30006F6E6720657874727573696F6E2070724B
:101E40006576656E7465640A0020636F6C64206556
:101E50007874727573696F6E2070726576656E74D2
:101E600065640A00627573793A2070617573656400
:101E700020666F7220696E7075740A0062757379DE
:101E80003A2070617573656420666F7220757365A2
:101E9000720A00627573793A2070726F63657373AA
:101EA000696E670A004B494C4C45442E20004B4953
:101EB0004C4C20636175736564206279204B494CFA
:101EC0004C20627574746F6E2F70696E0A004B49F6
:101ED0004C4C45442E20004B494C4C20636175739B
:101EE000656420627920746F6F206D756368206966
:101EF0006E6163746976652074696D65202D206359
:101F0000757272656E7420636F6D6D616E643A20D8
:101F1000007C3C3E5E2B3D3F2F5B5D3B2C2A225CD0
:101F20000070012C0190012701B0012201C0011DA8
:101F300001F00118011002130130020E01600209C4
:101F40000190020401C002FF000003FA004003F503
:101F5000008003F000D003EB002004E6007004E1F1
:101F600000E004DC004005D700C005D2004006CDEB
:101F700000D006C8008007C3003008BE00F008B9D2
:101F800000C009B400B00AAF00B00BAA00D00CA585
:101F900000000EA000500F9B00C010960050129140
:101FA0000000148C00C0158700B0178200B0197DA6
:101FB00000D01B7800001E730040206E0090226944
:101FC00000F024640040275F0090295A00E02B5560
:101FD00000102E500020304B0010324600E03341FC
:101FE0000090353C001037370070383200A0392D92
:101FF00000B03A2800A03B2300603C1E00103D19B1
:1020000000903D1400103E0F00703E0A00C03E05D7
:1020100000003F0000403FFBFF803FF6FFC03FF164
:10202000FF544845524D414C2052554E415741595D
:1020300000546865726D616C2052756E61776179CC
:102040000057726974696E6720746F2066696C65E9
:102050003A20006F70656E206661696C65642C20A3
:1020600046696C653A20006F70656E206661696C28
:1020700065642C2046696C653A200046696C6520D1
:1020800073656C65637465640A002053697A653A08
:10209000200046696C65206F70656E65643A2000AB
:1020A0006F70656E206661696C65642C2046696C92
:1020B000653A20002066696C653A20004E6F7720F3
:1020C000002220706F73002220706172656E743A76
:1020D0002200535542524F5554494E452043414CDE
:1020E0004C207461726765743A22004B494C4C4530
:1020F000442E2000747279696E6720746F206361CA
:102100006C6C207375622D67636F64652066696C03
:102110006573207769746820746F6F206D616E79C4
:10212000206C6576656C732E204D4158206C657669
:10213000656C2069733A0043616E6E6F74206F7036
:10214000656E2073756264697220004572726F72E9
:102150002077726974696E6720746F20454550520C
:102160004F4D210A006265640A002C207379737454
:10217000656D2073746F70706564212048656174AB
:1021800065725F49443A20004572723A204D4158C9
:1021900054454D5020424544004572723A204D410D
:1021A0005854454D50004D415854454D502074727F
:1021B00069676765726564004572723A204D494EE1
:1021C00054454D5020424544004572723A204D49D5
:1021D0004E54454D50004D494E54454D502074725B
:1021E000696767657265640048656174696E672038
:1021F0006661696C65640048656174696E67206634
:1022000061696C65640048656174696E6720666128
:10221000696C65640048656174696E672066616910
:102220006C65640000002100240027002A002D00B6
:102230003000330001010000040107010A0184E6B7
:10224000C9E711241FBECFEFD1E2DEBFCDBF00E052
:102250000CBF15E0A0E0B2E0E2E2FEEE01E00BBF51
:1022600002C007900D92AE36B107D9F72CE1AEE669
:10227000B5E001C01D92A133B207E1F711E1C0E260
:10228000D1E100E006C021970109802FFE010E94E4
:102290004BF6CF31D10780E00807A9F70E9462DC36
:1022A0000C9400F70C9400002F923F924F925F9293
:1022B0006F927F928F929F92AF92BF92CF92DF9256
:1022C000EF92FF920F931F93CF93DF93CDB7DEB7BB
:1022D000CF55D1090FB6F894DEBF0FBECDBF009128
:1022E000331720E6029F800111240F5B194F809164
:1022F000911680FF1AC0E2EBF2E184917F013FEF7B
:10230000E31AF30A811102C0780104C00E9417D9B0
:10231000F701F3CFD7018D917D01882319F00E9439
:1023200017D9F8CF8AE00E9417D981E090E0909306
:10233000581B8093571B10929105109290058FE3C4
:1023400080939B0510929A051092990584E0E8E825
:10235000F5E0DF011D928A95E9F7F80180810F5FB2
:102360001F4F8032D1F38E34C9F4818190ED980FE4
:102370009A3020F08D3211F08B3281F4DF01129609
:102380009D012F5F3F4F8C9180538A3010F4D9010B
:10239000F7CFFD01119680818032D9F3F0935F1B56
:1023A000E0935E1B7F01BFEFEB1AFB0A10816AE22C
:1023B00070E0C7010E9499F6009731F0FC01319757
:1023C00080818032E1F311821D3431F1143521F125
:1023D000173411F1E2EBF2E184918F010F5F1F4F8F
:1023E000882321F00E9417D9F801F6CF60915E1B77
:1023F00070915F1B8BEC95E00E94AD5382E20E94CE
:1024000017D98AE00E9417D91092581B1092571BB7
:102410000E94D8B10C94852AC701FC012081019645
:102420002032D9F320532A30A8F610939B0580E080
:1024300090E06AE03196DF0111972C91022E000C9A
:10244000330B20533109689FA001699F500D11245F
:10245000C901840F951F208120532A3058F390938F
:102460009A0580939905DF0131962C912032D9F39A
:102470001D34D1F48E31910591F03CF487319105F2
:1024800071F08C31910581F40AC08537910564F0B3
:102490008737910524F0803AE3E09E0729F4B09352
:1024A0009105A09390057DC0109291051092900522
:1024B00000915E1BEE24E394F12CFD0131962C91EA
:1024C000222309F46EC02132A9F41D3499F480321C
:1024D000910581F4F0939105E093900563E270E03B
:1024E000CF010E9499F6009711F40C94951EDC011F
:1024F0001C9257C021542A31A0F5AF01FA01308156
:102500004F5F5F4F3032D1F340ED430F4A3040F020
:1025100043ED430F423020F03B3211F00C94AB29D5
:10252000AF01622F70E0DB0133E0B595A7953A95D6
:10253000E1F7A857BA4F2770670102C0CC0CDD1C29
:102540002A95E2F796013C91232B2C9341155105D6
:1025500011F0401B01C040E0DB01A259BA4F4C937F
:102560000AC02091900530919105232B21F4B0935E
:102570009105A0939005208121542A3110F4DF01A8
:102580009CCFDF01AD014F5F5F4F2C9120532A306C
:1025900010F4DA01F7CFFD01119620812032D9F332
:1025A000EECF80919B058D3411F40C94951E8435EB
:1025B00011F40C946A29873409F00CCF2090990506
:1025C00030909A052CE12216310409F485C694F462
:1025D00044E02416310444F452E0251631040CF092
:1025E000FEC037FE2FC010CF84E02816310409F456
:1025F0002EC60ACF9AE22916310411F40C94E31D79
:102600006CF4BDE12B16310411F40C94C01CEEE106
:102610002E16310411F40C94C41CF6CEFBE52F16D3
:10262000310411F40C94481D2CE52216310411F4E8
:102630000C944D1D3AE52316310409F0E5CE1092B5
:102640009805E2CE80916002882309F4DDCE0E94D5
:1026500082540E949AAE8091D71B813021F482E08F
:102660008093D71BD1CE90917712992309F4CCCEC9
:10267000823009F4C9CE8091220690912306893BCD
:102680009105DCF06091220670912306072E000C64
:10269000880B990B0E94B7EC9B01AC016091FC0583
:1026A0007091FD058091FE059091FF050E94B1ECAF
:1026B00087FF03C00E94A8ABE5CF1092391781E0D5
:1026C00080933C0280EA9FE09093F91B8093F81B73
:1026D0008091D51B882349F182E090E090937E158C
:1026E00080937D1585E08093711512E81093741521
:1026F00084E190E1A0E0B0E08093751590937615A9
:10270000A0937715B09378150E94566661E070E04B
:1027100080E090E00E94D4DB81E09AE590937E1502
:1027200080937D158BE090E028C08EE090E0909340
:102730007E1580937D1585E08093711512E81093C6
:10274000741584E190E1A0E0B0E08093751590935A
:102750007615A0937715B09378150E94566661E0C0
:1027600070E080E090E00E94D4DB81E09AE59093F5
:102770007E1580937D1585E390E09093801580937E
:102780007F1587E0809371151093741584E890E0AD
:10279000A0E0B0E08093751590937615A09377151F
:1027A000B09378150E94566681E080933F1780931E
:1027B000D71B8091C71A9091C81A019739F40E94CB
:1027C0009E6A7093C81A6093C71A04C01092C81A00
:1027D0001092C71A1092C51A1092C61A15CE80917F
:1027E0006002882309F410CE0E94825482E50E9480
:1027F000FBD8882309F43CC10E9495D84B015C01A9
:102800008091D2169091D316A091D416B091D5167E
:102810008CA79DA7AEA7BFA72091D6163091D7163B
:102820004091D8165091D91628AB39AB4AAB5BAB67
:102830008091931A9091941AA091951AB091961A3A
:1028400088AF99AFAAAFBBAF2091971A3091981A71
:102850004091991A50919A1A2CAB3DAB4EAB5FAB9D
:1028600020E030E0A901C501B4010E94B1EC882349
:1028700009F42AC128AD39AD4AAD5BAD6CA57DA583
:102880008EA59FA50E94B1EC81110DC02CA93DA978
:102890004EA95FA968A979A98AA99BA90E94B1EC50
:1028A000882309F411C111E032E02316310409F044
:1028B00010E020E030E0A901C501B4010E94B1ECB4
:1028C000881F8827881F181759F080E090E0A0E83B
:1028D000BFEB28968CAF9DAFAEAFBFAF28970AC0B5
:1028E00020E030E040E85FE328962CAF3DAF4EAFEC
:1028F0005FAF28972CA53DA54EA55FA568AD79AD26
:102900008AAD9BAD0E944AF324966CAF7DAF8EAF2B
:102910009FAF249728A939A94AA95BA96CA97DA9C9
:102920008EA99FA90E944AF36B017C0124962CADCD
:102930003DAD4EAD5FAD2497CA01B9010E9416EDC1
:102940002B013C01A7019601C701B6010E9416EDBB
:102950009B01AC01C301B2010E944BF30E94B7F589
:102960006CAF7DAF8EAF9FAF20E030E040E05FE323
:102970000E9416ED2B013C01A5019401C501B40193
:102980000E9416ED4B015C01A3019201C301B2014B
:102990000E9416ED9B01AC01C501B4010E944AF3EF
:1029A0000E94B7F528962CAD3DAD4EAD5FAD289792
:1029B0000E9416ED4B015C01C701B60190582CAD89
:1029C0003DAD4EAD5FAD0E9427F4A50194010E947C
:1029D00016ED6B017C0128AD39AD4AAD5BAD6CA540
:1029E0007DA58EA59FA50E944BF320E030E040E03E
:1029F0005FE30E9416ED9B01AC01C701B6010E9486
:102A00004BF32CA53DA54EA55FA50E944AF36B0193
:102A10007C012CA93DA94EA95FA968A979A98AA919
:102A20009BA90E944BF320E030E040E05FE30E946E
:102A300016ED2B013C012CAD3DAD4EAD5FAD2496A6
:102A40006CAD7DAD8EAD9FAD24970E9427F4A5019E
:102A500094010E9416ED9B01AC01C301B2010E94DA
:102A60004BF328A939A94AA95BA90E944AF314C0CB
:102A700089E40E94FBD8882329F00E9495D86B0135
:102A80007C0103C0C12CD12C76018AE40E94FBD8C2
:102A90008823E9F00E9495D868AF79AF8AAF9BAFE1
:102AA00020E030E0A901C701B6010E94B1EC81111C
:102AB0001BC020E030E0A90168AD79AD8AAD9BADC7
:102AC0000E94B1EC811110C0ECE7F2E1ADC320E04F
:102AD00030E0A901C701B6010E94B1EC8823A1F33F
:102AE00018AE19AE1AAE1BAED701C601B0588CA7EE
:102AF0009DA7AEA7BFA728AD39AD4AAD5BAD505875
:102B000028AB39AB4AAB5BAB9C01AD01BC01CD013D
:102B10000E9416ED4B015C0128A939A94AA95BA9BD
:102B2000CA01B9010E9416ED9B01AC01C501B401B7
:102B30000E944BF30E94B7F564966CAF7DAF8EAFE9
:102B40009FAF64978091D2169091D316A091D4161E
:102B5000B091D5168CAB9DABAEABBFAB9C01AD01BC
:102B6000C701B6010E944BF328966CAF7DAF8EAFC4
:102B70009FAF28972091D6163091D7164091D8163E
:102B80005091D9162CAF3DAF4EAF5FAF28AD39ADE8
:102B90004AAD5BAD6CAD7DAD8EAD9FAD0E944BF38C
:102BA00068966CAF7DAF8EAF9FAF68978091931A98
:102BB0009091941AA091951AB091961A2C968CAF78
:102BC0009DAFAEAFBFAF2C9728962CAD3DAD4EADAF
:102BD0005FAD2897BC01CD010E944AF36B017C01D7
:102BE0002091971A3091981A4091991A50919A1AF7
:102BF00060962CAF3DAF4EAF5FAF609768962CAD3F
:102C00003DAD4EAD5FAD689760966CAD7DAD8EAD60
:102C10009FAD60970E944AF34B015C018091DA16E8
:102C20009091DB16A091DC16B091DD166C968CAFFE
:102C30009DAFAEAFBFAF6C979C01AD0160919B1A89
:102C400070919C1A80919D1A90919E1A0E944AF34D
:102C500024966CAF7DAF8EAF9FAF2497A7019601EE
:102C60006CA57DA58EA59FA50E9416ED2B013C01AC
:102C7000A501940168A979A98AA99BA90E9416EDCA
:102C80009B01AC01C301B2010E944BF32B013C013B
:102C9000A50194016CA57DA58EA59FA50E9416EDAA
:102CA0004B015C01A701960168A979A98AA99BA992
:102CB0000E9416ED9B01AC01C501B4010E944AF3CC
:102CC000A30192010E94BEF36B017C0120E030E081
:102CD000A9010E94B1EC87FF0AC02BED3FE049EC4F
:102CE00050E4C701B6010E944BF36B017C0192E0F6
:102CF0002916310451F42BED3FE049EC50E4C701B3
:102D0000B6010E944AF36B017C0120E030E0A9018A
:102D1000C701B6010E94B1EC811124C02C962CADE4
:102D20003DAD4EAD5FAD2C976CA97DA98EA99FA935
:102D30000E94B1EC811116C060962CAD3DAD4EAD38
:102D40005FAD60976CAD7DAD8EAD9FAD0E94B1EC77
:102D5000811108C00BEDC02E0FE0D02E09ECE02E43
:102D600000E4F02EA701960164966CAD7DAD8EADAA
:102D70009FAD64970E9416ED9B01AC010E9416ED79
:102D80004B015C0124962CAD3DAD4EAD5FAD24975B
:102D9000CA01B9010E9416ED9B01AC01C501B40145
:102DA0000E944BF30E94B7F54B015C012FE632E124
:102DB00043E85AE30E94B1EC87FD30C2C501B4017B
:102DC0000E94C0F40E9494F47DAF6CAFDB01AB2B8A
:102DD00021F4E1E0F0E0FDAFECAF4090DE16509062
:102DE000DF166090E0167090E1162CAD3DADB90194
:102DF00080E090E00E94B5EC4B015C019B01AC01CE
:102E0000C701B6010E9427F46CAB7DAB8EAB9FABC4
:102E1000A501940124966CAD7DAD8EAD9FAD249738
:102E20000E9427F464966CAF7DAF8EAF9FAF64971E
:102E3000A301920160919F1A7091A01A8091A11A2A
:102E40009091A21A0E944AF3A50194010E9427F4CE
:102E5000A0966CAF7DAF8EAF9FAFA0972CA93DA978
:102E60004EA95FA9CA01B9010E9416ED20E030E029
:102E700040E05FE30E9416ED9B01AC0160E070E072
:102E800080E89FE30E944AF324966CAF7DAF8EAF3B
:102E90009FAF24976C968CAD9DADAEADBFAD6C97DA
:102EA00089879A87AB87BC874D865E866F86788ACE
:102EB00060910B0270910C02072E000C880B990B8D
:102EC0000E94B7EC209134023091350240913602D5
:102ED000509137020E9416ED2AE037ED43E25CE3A1
:102EE0000E9416ED2C966CAF7DAF8EAF9FAF2C97E6
:102EF0000E940CDC9B01AC0128533F4F4F4F5F4FAA
:102F000060962CAF3DAF4EAF5FAF60974CA45DA411
:102F10006EA47FA422242394312C19E1D12E4CAD30
:102F20005DAD4215530509F435C10E9435D30E94A9
:102F30000CDCDC01CB0160962CAD3DAD4EAD5FAD40
:102F40006097821B930BA40BB50BB7FD10C00E94BA
:102F50000CDC9B01AC0128533F4F4F4F5F4F6096F5
:102F60002CAF3DAF4EAF5FAF60970E94A8ABDA9435
:102F7000DD2009F441C028A939A94AA95BA92496F2
:102F80006CAD7DAD8EAD9FAD24970E9416ED4B01CB
:102F90005C019201A3016CA97DA98EA99FA90E9441
:102FA00016EDA50194010E944BF37B018C01920167
:102FB000A30124966CAD7DAD8EAD9FAD24970E948C
:102FC00016ED4B015C0128A939A94AA95BA96CA996
:102FD0007DA98EA99FA90E9416ED9B01AC01C50198
:102FE000B4010E944AF32B013C01C701D80188AB10
:102FF00099ABAAABBBAB4DC0B10180E090E00E94A1
:10300000B5EC2CA93DA94EA95FA90E9416ED4B0174
:103010005C010E9424F46B017C01C501B4010E9493
:10302000ADF54B015C01A70196016CA57DA58EA5B0
:103030009FA50E9416ED2B013C0128AD39AD4AAD8C
:103040005BADC501B4010E9416EDA30192010E947F
:103050004BF32B013C01A50194016CA57DA58EA528
:103060009FA50E9416ED4B015C0128AD39AD4AAD1C
:103070005BADC701B6010E9416ED9B01AC01C50115
:10308000B4010E944AF368AB79AB8AAB9BABA9E170
:10309000DA2E9201A30128966CAD7DAD8EAD9FAD69
:1030A00028970E944BF369837A838B839C8328A99A
:1030B00039A94AA95BA968966CAD7DAD8EAD9FAD6F
:1030C00068970E944BF36D837E838F839887649605
:1030D0002CAD3DAD4EAD5FAD649769857A858B852E
:1030E0009C850E944BF369877A878B879C87A09683
:1030F0002CAD3DAD4EAD5FADA0976D857E858F85C6
:1031000098890E944BF36D877E878F87988B80917B
:103110003302882321F0CE0101960E9408A8C090B6
:10312000930589819A81AB81BC8188A399A3AAA3C5
:10313000BBA38D819E81AF81B8858CA39DA3AEA3D7
:10314000BFA389859A85AB85BC8588A799A7AAA7BF
:10315000BBA7AE01485D5F4FBE016C5D7F4FCE01E6
:1031600080960E9436812C96ECACFDAC0EAD1FAD66
:103170002C979E01235F3F4FAE01485D5F4FBE011C
:103180006C5D7F4FCE0180960E941D743FEF231A25
:10319000330AC5CEC09093058091931A9091941AEA
:1031A000A091951AB091961A88A399A3AAA3BBA33C
:1031B0008091971A9091981AA091991AB0919A1AA1
:1031C0008CA39DA3AEA3BFA380919B1A90919C1A40
:1031D000A0919D1AB0919E1A88A799A7AAA7BBA7EC
:1031E000AE01485D5F4FBE016C5D7F4FCE018096A2
:1031F0000E9436812C96ECACFDAC0EAD1FAD2C9729
:103200002FE93AE1AE01485D5F4FBE016C5D7F4F33
:10321000CE0180960E941D740E94316E0E940DD9CD
:10322000F3C80E9417D9F80184918F010F5F1F4FD7
:103230008111F7CFE7E0F3E084918F010F5F1F4F1B
:10324000882309F4E1C80E9417D9F801F5CF80E579
:103250000E94FBD8882379F080918C0590918D0590
:10326000009749F04AE050E060E070E00E9430EBE7
:103270006B017C0103C0C12CD12C760183E50E9437
:10328000FBD8882361F00E9495D820E030E04AE71F
:1032900054E40E9416ED0E9494F46B017C010E949C
:1032A0003AD70E940DD98091A31A9091A41AA091A7
:1032B000A51AB091A61AC80ED91EEA1EFB1E0E94BE
:1032C0000CDCDC01CB018C199D09AE09BF09B7FFED
:1032D0009BC80E94A8ABF3CF0E943AD780E00E941F
:1032E000716B0E94336C11E01093F40588E50E9425
:1032F000CCD8E82E89E50E94CCD8082F8AE50E9418
:10330000CCD8F82EE11004C0011104C0182705C064
:10331000011102C010E001C0182F0E94276E111188
:1033200005C0E11003C0002309F440C020E030E0F4
:1033300040EA50E46091EA167091EB168091EC1629
:103340009091ED160E944BF360939B1A70939C1A18
:1033500080939D1A90939E1A2091DA163091DB1675
:103360004091DC165091DD160E9471F518165CF440
:1033700019821A821B821C82BE016F5F7F4F8BE90C
:103380009AE10E94446D111105C0E11003C00111C2
:1033900007C00CC080E090E00E94CBA61123B9F3D7
:1033A00081E090E00E94CBA6111103C0FF2009F438
:1033B000CEC08091F505882321F08091F60581111A
:1033C0001AC0E2EBF2E184918F010F5F1F4F811170
:1033D00003C0EFE2F3E004C00E9417D9F801F3CF75
:1033E00084918F010F5F1F4F882309F4B0C00E94A2
:1033F00017D9F801F5CF0E941ED84090E2165090E0
:10340000E3166090E4167090E51620E030E044E3A7
:1034100053E4C301B2010E944BF34B015C01609382
:10342000931A7093941A8093951A9093961A809198
:10343000E6169091E716A091E816B091E9168CA7D0
:103440009DA7AEA7BFA720E030E044E353E4BC0152
:10345000CD010E944BF36B017C016093971A70932E
:10346000981A8093991A90939A1A8091DA169091EB
:10347000DB16A091DC16B091DD1680939B1A909319
:103480009C1AA0939D1AB0939E1AA3019201C501A4
:10349000B4010E944AF34B015C012FE632E143E89C
:1034A0005AEB0E9471F587FD0AC021E230E044EB3F
:1034B00053E4C501B4010E94B1EC18161CF4E2EB10
:1034C000F2E133C02CA53DA54EA55FA5C701B6010D
:1034D0000E944AF36B017C012FE632E143E85AEB8C
:1034E0000E9471F587FDEBCF21E230E044EB53E41D
:1034F000C701B6010E94B1EC18160CF319821A82AA
:103500001B821C829E012F5F3F4F4AED56E167E907
:103510007AE183E99AE10E94536C82E090E00E9494
:10352000CBA615C00E9417D9F80184918F010F5FB7
:103530001F4F8111F7CFEDE1F3E084918F010F5F11
:103540001F4F882321F00E9417D9F801F6CF0E945F
:103550001ED88091D91B813009F059C080933C025C
:1035600080E090E00E94E7C68091D51B882319F186
:1035700084E090E090937E1580937D1585E08093A4
:10358000711512E81093741584E190E1A0E0B0E0A9
:103590008093751590937615A0937715B093781551
:1035A0000E94566681E09AE590937E1580937D1582
:1035B0008CE090E022C080E190E090937E158093B3
:1035C0007D1585E08093711512E81093741584E1E0
:1035D00090E1A0E0B0E08093751590937615A093EC
:1035E0007715B09378150E94566681E09AE590931E
:1035F0007E1580937D1586E390E0909380158093EF
:103600007F1587E080937115109374152AC085305B
:10361000B1F581E080933C0280E090E00E94E7C633
:103620001092D91B8091D51B882349F081E09AE53F
:1036300090937E1580937D158CE290E008C081E028
:103640009AE590937E1580937D1581E590E09093A7
:10365000801580937F1587E08093711582E88093B1
:10366000741584E890E0A0E0B0E080937515909325
:103670007615A0937715B09378150E9456668091C1
:103680008F05882309F450C018A219A21AA21BA200
:1036900020E030E040EA50E46091DA167091DB16E9
:1036A0008091DC169091DD160E944AF369837A833B
:1036B0008B839C83BE01605E7F4FCE0101960E948A
:1036C000446D87EA9AE10E941D67809178128823F1
:1036D00019F081E08093771281E090E09093681276
:1036E00080936712109271121092721210927312DC
:1036F000109274120E940CDC60936D1270936E1223
:1037000080936F12909370128091670E9091680E63
:10371000A091690EB0916A0E8093691290936A121B
:10372000A0936B12B0936C128091771A8093F4057A
:103730000E94196C0E94C85D8091D91B982F9D7FB3
:10374000943009F07FC090913617992309F478C01E
:103750001092361710923C029091D51B992351F18B
:10376000843069F460918E05862F90E0A0E0B0E08F
:10377000BC01CD01635E7F4F8E4F954A29C08630D4
:1037800009F05EC018A219A21AA21BA219821A82FD
:103790001B821C82BE01605E7F4FCE0101960E949B
:1037A000446D81E09AE590937E1580937D1586E1C6
:1037B00090E02EC0843099F460918E05862F90E0C1
:1037C000A0E0B0E0BC01CD01695B7F4F8E4F954A10
:1037D00024E830E040E050E00E94FA6631C08630D4
:1037E00079F518A219A21AA21BA219821A821B82A9
:1037F0001C82BE01605E7F4FCE0101960E94446D27
:1038000081E09AE590937E1580937D1580E490E0A9
:103810009093801580937F1587E08093711582E8DF
:103820008093741584E890E0A0E0B0E08093751573
:1038300090937615A0937715B09378150E945666ED
:103840001092D91B20E030E040E251E46091D216A2
:103850007091D3168091D4169091D5160E9416EDD2
:103860000E948FF470937E1560937D1505E00093A0
:10387000711512E81093741588E490E1A0E0B0E0AF
:103880008093751590937615A0937715B09378155E
:103890000E94566620E030E040E251E46091D61686
:1038A0007091D7168091D8169091D9160E9416ED76
:1038B0000E948FF470937E1560937D1500937115AF
:1038C000109374158AE490E1A0E0B0E08093751540
:1038D00090937615A0937715B09378150E9456664D
:1038E00020E030E040E251E46091DA167091DB169E
:1038F0008091DC169091DD160E9416ED0E948FF4E7
:1039000070937E1560937D15009371151093741557
:103910008CE490E1A0E0B0E080937515909376156B
:10392000A0937715B09378150E9456669091771200
:1039300080918F05992391F0811110C080913717E4
:1039400081110FC081E08093371780E493E090935A
:103950001511809314110E94C5D703C081111092D4
:103960008F058091D91B813031F40E94716B1092C8
:10397000D91B0C94041280E00E94716B0C94041209
:103980000E94EB560C940412C090D216D090D3161D
:10399000E090D416F090D51688E50E94FBD88111EE
:1039A00008C020E030E0A901C701B6010E944BF336
:1039B00002C00E9495D868A379A38AA39BA3C09054
:1039C000D616D090D716E090D816F090D91689E583
:1039D0000E94FBD8811108C020E030E0A901C70196
:1039E000B6010E944BF302C00E9495D86B017C0186
:1039F00069837A838B839C832091E2163091E3164E
:103A00004091E4165091E51668A179A18AA19BA185
:103A10000E944AF34B015C012FE632E143E85AEB86
:103A20000E9471F587FF02C00C94041221E230E07D
:103A300044EB53E4C501B4010E94B1EC181614F430
:103A40000C9404122091E6163091E7164091E81686
:103A50005091E916C701B6010E944AF36B017C013F
:103A60002FE632E143E85AEB0E9471F587FF02C06E
:103A70000C94041221E230E044EB53E4C701B60198
:103A80000E94B1EC181614F40C9404120C94BC2986
:103A900081E0809398050C94041285E40E94FBD881
:103AA000B82E811102C00E943AD775E6872E72E0C7
:103AB000972EE2EDCE2EE6E1DE2EF4E8EF2EFAE1CF
:103AC000FF2E00E010E0A12C33243394D4018D911B
:103AD0004D010E94FBD8882359F1F60140805180A6
:103AE000628073800E9495D8D6016D937D938D93EB
:103AF0009C9313970330E1F0023011F43092F705F4
:103B0000A30192010E944AF39B01AC01F70160817D
:103B10007181828193810E944BF3D7016D937D93D4
:103B20008D939C931397C8010E94A36EAA24A3941B
:103B30000F5F1F4FB4E0CB0ED11CE4E0EE0EF11C82
:103B40000430110519F6AA2019F00E941ED837C0BA
:103B5000BB20A9F1C090DE16D090DF16E090E016F1
:103B6000F090E1162091BE163091BF164091C0161C
:103B70005091C116C701B6010E9416ED0E947DF555
:103B80006093D3117093D4118093D5119093D61173
:103B9000C701B6010E948FF42FB7F8946093EC1B15
:103BA0007093ED1B8093EE1B9093EF1B2FBF109231
:103BB000C3111092C4111092C5111092C6110E9427
:103BC000C85D0C94041280916002882311F40C9457
:103BD000041289E40E94FBD8082F882321F00E9458
:103BE00065D8162F01C010E08AE40E94FBD8E82EA9
:103BF000882321F00E9465D8F62E01C0F12C002305
:103C000011F0143028F4EE2089F0F3E0FF1570F481
:103C1000E6E5F3E084918F010F5F1F4F882311F4D5
:103C20000C9404120E9417D9F801F4CF0E94276E59
:103C3000002339F12091731A3091741A1203B001E4
:103C4000139F700D112480916F1A9091701A680F54
:103C5000791F072E000C880B990B0E94B7EC20915E
:103C6000E2163091E3164091E4165091E5160E9459
:103C70004BF36093931A7093941A8093951A9093D0
:103C8000961AEE2041F12091751A3091761A4F2D37
:103C90004203B001439F700D11248091711A9091DD
:103CA000721A680F791F072E000C880B990B0E945F
:103CB000B7EC2091E6163091E7164091E816509146
:103CC000E9160E944BF36093971A7093981A8093A9
:103CD000991A90939A1A80E50E94CCD881110E947B
:103CE00086D886E40E94FBD88823D9F00E9495D814
:103CF0006B017C0120E030E0A9010E9471F51816EB
:103D000084F420E030E040E752E4C701B6010E94AD
:103D100027F46093340270933502809336029093B7
:103D200037020E949AAE0C940412809199059091EA
:103D30009A058637910509F48EC60CF0C2C08D3401
:103D4000910509F4F1C30CF058C08A31910509F4CA
:103D500045C24CF58531910509F4E5C184F4823101
:103D6000910509F4A0C58431910509F49AC14197E0
:103D700011F00C9404120E9449AE0C940412873185
:103D8000910509F4DCC10CF4D4C18831910509F422
:103D9000ECC1499711F00C940412109277120E9412
:103DA00010C90C9404128F31910509F4C7C274F440
:103DB0008C31910509F46EC20CF42FC24E9711F0AC
:103DC0000C9404120E94D8630C9404128A32910558
:103DD00009F467C32CF4809709F466C20C940412AA
:103DE0008B34910509F49CC38C34910511F00C942B
:103DF00004120E9410C90C9404128A36910509F429
:103E000018C5BCF58435910509F44DC5ECF482352F
:103E1000910509F43FC50CF041C58135910511F0BC
:103E20000C9404120E94EDC60E943AD70E9438AE4C
:103E300010923B1710923A1768EE73E080E090E022
:103E40000E94B6C20C9404128C35910509F474C515
:103E500034F48535910509F454C50C940412883660
:103E6000910509F465C38936910509F495C40C944C
:103E700004128F36910509F497C384F48C369105AA
:103E800009F437C40CF4F4C48D36910509F4C9C49F
:103E90008E36910509F475C30C940412813791058F
:103EA00009F42FC40CF429C48237910509F4CDC557
:103EB0008337910511F00C9404120E94CF8A0C9460
:103EC00004128C3251E0950711F40C948E270CF0FB
:103ED00066C08B3C910509F46EC6ACF58C38910533
:103EE00009F43CC48CF48837910509F4EFC50CF44F
:103EF000E9C58937910511F00C9404121092F4056C
:103F00001092771A0C9404128E3B910509F48DC41B
:103F100034F48B39910509F45BC40C940412883C89
:103F2000910509F4DAC5893C910511F00C9404124D
:103F300015E6E12E12E0F12E02EA16E182EBC82E20
:103F400086E1D82E1EC6833D910509F4DAC694F4A5
:103F50008D3C910509F4B8C60CF44AC68E3C910517
:103F600011F00C940412A5E6EA2EA2E0FA2E00E06D
:103F700010E0AEC68D3D910509F4D6C634F48C3DF3
:103F8000910509F4C2C60C940412823E910509F40D
:103F9000E7C68831914009F412C70C940412843AA0
:103FA000E1E09E0711F40C941D28ACF5833621E066
:103FB000920709F472C084F48E3241E0940709F448
:103FC000DBC70CF4D5C78F32914011F00C9404126A
:103FD0000E94588B0C9404128139B1E09B0711F4B4
:103FE0000C9413284CF48039914011F00C94041275
:103FF0000E943AD70C940412823921E0920711F4FE
:104000000C9418288A39914011F00C9404120E94E3
:10401000278A0C940412863F41E0940711F40C9413
:10402000FE28FCF48C3AA1E09A0711F40C942128A4
:104030004CF4853A914011F00C9404120E94E788E8
:104040000C940412843FF1E09F0711F40C94FA28B9
:10405000853F914011F00C9404120E94849A0C94B4
:104060000412833533E09307A1F03CF4873F91407D
:1040700011F40C9402290C940412803AA3E09A07DC
:1040800009F44FC1873E934011F40C9458290C94C5
:104090000412E2EBF2E10C941429ECE7F2E10C9447
:1040A0004429E4E8F3E084918F010F5F1F4F8823D8
:1040B00021F00E9417D9F801F6CF10921C1510922A
:1040C0001B1588EA92E10E94ECB38BE1E8EAF2E189
:1040D000DE01159601900D928A95E1F78091A61266
:1040E0009091A7129C838B838DEE92E09A838983B3
:1040F00040E050E0BE016F5F7F4F8BE993E00E948C
:104100002AC9CE0101960E949AA8E5E7F3E08491BE
:104110008F010F5F1F4F882311F40C9404120E942B
:1041200017D9F801F4CF0E9458680E94A2A80C94F5
:10413000041210927712109278120C940412E091EB
:104140009005F09191058081882329F0803209F44F
:1041500010823196F8CF40E061E080919005909117
:1041600091050E9442CB0C94041268EF7EE088EA2D
:1041700092E10E94A4D2811103C0EAEAF3E00FC0E9
:10418000E8E9F3E084918F010F5F1F4F811103C0B5
:10419000E5E9F3E00EC00E9417D9F801F3CF84914E
:1041A0008F010F5F1F4F882399F30E9417D9F801E1
:1041B000F6CF84918F010F5F1F4F882321F00E945B
:1041C00017D9F801F6CF80917812882319F081E091
:1041D000809377120E94B8C80C94041280917812D0
:1041E000882311F40C94041283E50E94FBD88823E1
:1041F00011F40C9404120E9465D8AB01BC014093E9
:10420000121550931315609314157093151582E4CD
:1042100094E10E9480D00C94041280917812811154
:1042200003C0E1EDF3E02AC0EFEBF3E084918F01EE
:104230000F5F1F4F882321F00E9417D9F801F6CF96
:1042400060911215709113158091141590911515A8
:104250004AE00E941ED98FE20E9417D960910E1584
:1042600070910F1580911015909111154AE00E94E0
:104270001ED98AE00E9417D90C94041284918F01F0
:104280000F5F1F4F882311F40C9404120E9417D95A
:10429000F801F4CF40E060E08091900590919105A5
:1042A0000E9442CB0C9404128091771281110E94DB
:1042B0003AD7E0909005F090910580E50E94CCD827
:1042C000182F882319F00E9486D8182F8091781211
:1042D000882311F40C940412412F61E0C7010E945D
:1042E00042CB83E50E94FBD8882381F00E9465D8E9
:1042F000AB01BC0140931215509313156093141534
:104300007093151582E494E10E9480D08091781218
:10431000882319F081E08093771211110C94041214
:1043200059CF809190059091910521E020937612CC
:1043300040E060E00E9442CB0C9404120E949E6A0E
:104340007B018C0120E831E541E050E00E94EDF274
:10435000C9016DE671E00E9424F64B015C01C801C1
:10436000B70120E13EE040E050E00E94EDF2CA01DA
:10437000B90128E130E040E050E00E94EDF2762EF5
:10438000672EC62ED72E6CE3262E312C412C512CB5
:10439000C801B701A20191010E94EDF2F62EE72EAD
:1043A000CA01B901A20191010E94EDF2CB018E0177
:1043B0000F5F1F4F81149104D1F0EF92FF927F9312
:1043C0006F936F927F92BF92AF929F928F928AE08B
:1043D00094E09F938F931F930F930E9483EC0FB6EB
:1043E000F894DEBF0FBECDBFE2EBF2E145C0A114F1
:1043F000B10489F0EF92FF927F936F936F927F9257
:10440000BF92AF928AEF93E09F938F931F930F9386
:104410000E9483ECE4CFCD2879F0EF92FF927F9356
:104420006F936F927F928EEE93E09F938F931F9383
:104430000F930E9483ECD3CF892B69F0EF92FF9208
:104440007F936F9386EE93E09F938F931F930F93C9
:104450000E9483ECC4CFEF92FF9282EE93E09F9391
:104460008F931F930F930E9483EC0F900F900F90E8
:104470000F900F900F90B8CF84917F019FEFE91AB2
:10448000F90A882321F00E9417D9F701F5CFB80166
:104490008EE194E00E94AD538AE00E9417D90C94FB
:1044A000041283E50E94FBD8882311F40C940412B3
:1044B0000E9475D8E82E80E50E94FBD8882311F46D
:1044C0000C9404120E9465D8162FC62ED72ED7FE44
:1044D00002C00C940412E8EEF4E08491181303C0B7
:1044E000ECE7F2E109C03196A5E0E031FA07A9F75F
:1044F0009AC70E9417D9F80184918F010F5F1F4F4F
:104500008111F7CFEBE2F4E084918F010F5F1F4F31
:10451000882311F40C9404120E9417D9F801F4CFE7
:104520000E94B8C80C9404120E943D660C940412B8
:1045300088E690E00E94356F81110C9404128091FE
:10454000911683FF02C00C94041283E50E94FBD8ED
:10455000882399F00E9495D80E948FF4CB010E9485
:10456000E7C60E9495D820E030E04AEA52E40E9473
:10457000B1EC181614F00E943D660E94CF720C94A4
:1045800004128EE40E94FBD8882311F40C940412C8
:104590000E9465D860934B1B70934C1B80934D1BFE
:1045A00090934E1B0C94041283E50E94CCD8882370
:1045B00059F083E50E94FBD8882319F00E9475D832
:1045C00001C080E080939116E2EBF2E184918F01CB
:1045D0000F5F1F4F811103C0E8E4F4E004C00E94A4
:1045E00017D9F801F3CF84918F010F5F1F4F8823F4
:1045F00021F00E9417D9F801F6CF80919116811110
:1046000003C0E4E4F4E034C05AE3C52E54E0D52EF0
:10461000E12CF12C20E08091911690E00E2C02C04C
:10462000959587950A94E2F780FF17C0BB24B39451
:10463000B20E222319F08CE20E9417D9F60185915F
:104640009491FC0184918F010F5F1F4F882321F00B
:104650000E9417D9F801F6CF2B2DBFEFEB1AFB0AFA
:10466000E2E0CE0ED11CF5E0EF16F104A1F63CC05D
:1046700084918F010F5F1F4F8823B1F10E9417D9DA
:10468000F801F6CF8AE50E94CCD8882309F4ECC55E
:104690000E9495D86B017C0120E030E040EA51ECAB
:1046A0000E9471F587FDD3C520E030E040EA51E477
:1046B000C701B6010E94B1EC18160CF4C8C5C0922F
:1046C0002E17D0922F17E0923017F09231170E94D8
:1046D000239260912E1770912F178091301790912F
:1046E000311742E00E94A3D98AE00E9417D90C94A6
:1046F000041210923D020C9404128FE494E00E9484
:10470000BEA883E50E94FBD8811103C0E2EBF2E171
:104710000DC00E9475D8809355028D3310F40C940F
:1047200004128CE3809355020C94041284918F013F
:104730000F5F1F4F882321F00E9417D9F801F6CF91
:104740004091550250E060E070E088E594E00E94FE
:104750005A538AE00E9417D90C9404128091911642
:1047600083FF02C00C94041283E50E94FBD88823C7
:1047700011F40C9404120E9495D80E948FF46E37A5
:10478000710514F06DE770E07093210660932006C8
:104790000E944FC60C94041289E690E00E94356F87
:1047A000811111C0EFE5F4E084918F010F5F1F4F7D
:1047B000882321F00E9417D9F801F6CF0E94875E66
:1047C0008AE00E9417D91092581B1092571B9DC661
:1047D00083E50E94FBD8882311F40C9404120E94F4
:1047E00075D880935D1B8D3318F08CE380935D1B2F
:1047F0000E940CDC6B017C0120915D1B30E0A8EE77
:10480000B3E00E943BF3C60ED71EE81EF91EC0920D
:10481000591BD0925A1BE0925B1BF0925C1B0C94CC
:1048200004120E9443610C9404120E940A5F0C94CB
:10483000041283E50E94FBD8882339F00E9465D8D2
:104840008B016F3F710519F010F00FEF10E080E55C
:104850000E94FBD8811106C010933B1700933A17B2
:104860000C9404120E9475D881110C940412F4CF98
:1048700080E50E94FBD8811106C010923B17109270
:104880003A170C9404120E9465D8672B11F00C940F
:104890000412F3CF109297050C94041281E08093D8
:1048A00097050C94041283E50E94FBD88823A1F09D
:1048B0000E9495D820E030E04AE754E40E9416EDCB
:1048C0000E9494F4609356027093570280935802AA
:1048D000909359020C94041288E50E94CCD881115F
:1048E000BBC589E50E94CCD88111B6C58AE50E9476
:1048F000CCD88111B1C585E40E94CCD88111ACC55A
:10490000D6C583E50E94CCD8882311F40C940412F8
:104910000E9495D820E030E04AE754E40E9416ED6A
:104920000E9494F46093601B7093611B8093621BE0
:104930009093631B0C94041235E6C32E32E0D32E01
:1049400042EBE42E46E1F42E10E0D6018D916D018C
:104950000E94CCD8882309F46DC0133009F063C0DD
:104960000E9495D84B015C0120E030E040EA51E420
:104970000E94B1EC87FF4EC0A50194016091BE1664
:104980007091BF168091C0169091C1160E9427F4B5
:104990002B013C019B01AC01609161167091621684
:1049A00080916316909164160E9416ED60936116D3
:1049B000709362168093631690936416A30192011C
:1049C00060917D1670917E1680917F169091801671
:1049D0000E9416ED60937D1670937E1680937F166D
:1049E0009093801660919E1670919F168091A016EC
:1049F0009091A1160E94B5ECA30192010E9416EDC0
:104A00000E9494F460939E1670939F168093A01654
:104A10009093A1168092BE169092BF16A092C016D7
:104A2000B092C11607C00E9495D8F70160837183C8
:104A3000828393831F5FF4E0EF0EF11C143009F0C2
:104A400084CF0E940B820C9404120E943AD70E94D9
:104A5000C85D0C94041285E40E94CCD8882381F0B0
:104A60000E9486D8882361F0E2EBF2E184918F0105
:104A70000F5F1F4F882321F00E9417D9F801F6CF4E
:104A800081E40E94CCD8882381F00E9486D88823B4
:104A900061F0E2E6F4E084918F010F5F1F4F8823FD
:104AA00021F00E9417D9F801F6CF009190051091DE
:104AB0009105D8018D918D01882309F415CE0E94AE
:104AC00017D9F7CF0E94ED840C94041281E08093F3
:104AD000F4058093771A0C94041288EC90E00E94FD
:104AE000356F81110C94041284E40E94CCD8882381
:104AF00009F443C00E9495D86B017C0111E020E0CD
:104B000030E0A9010E94B1EC811101C010E01093C6
:104B1000CF1620E030E0A901C701B6010E94B1EC38
:104B2000882359F10091920510E00E9495D8000F5A
:104B3000111F000F111FF801E553F94E60837183B7
:104B40008283938320E030E0A9016091CB167091BD
:104B5000CC168091CD169091CE160E94B1EC8111A9
:104B60000CC080E090E0A0EEBFE38093CB16909362
:104B7000CC16A093CD16B093CE160E9455AE0C94D1
:104B80000412F70181917F010E94CCD8882351F053
:104B90000E9495D80E9494F4D8016D937D938D93D3
:104BA0009C9313970C5F1F4FC016D10651F70E94BC
:104BB000FF720C940412B5E6EB2EB2E0FB2E01E777
:104BC00016E1F70181917F010E94CCD8882341F042
:104BD0000E9495D8D8016D937D938D939C931397E4
:104BE0000C5F1F4FB6E101381B0759F70C940412F4
:104BF00083E50E94CCD88823D9F00E9495D8AB01D8
:104C0000BC014093691650936A1660936B167093BB
:104C10006C164093651650936616609367167093F2
:104C2000681680EC94E00E9477538AE00E9417D9BE
:104C300080E50E94CCD8882399F00E9495D8AB01DA
:104C4000BC014093691650936A1660936B1670937B
:104C50006C1683EA94E00E9477538AE00E9417D989
:104C600082E50E94CCD8882399F00E9495D8AB01A8
:104C7000BC0140936D1650936E1660936F1670933F
:104C8000701684E894E00E9477538AE00E9417D956
:104C900084E50E94CCD8882311F40C9404120E945D
:104CA00095D8AB01BC01409365165093661660938E
:104CB00067167093681686E694E00E9477538AE040
:104CC0000E9417D90C9404120E94578A0C94041263
:104CD000F70181917F010E94CCD8882339F00E948E
:104CE00095D8AB01BC01C8010E94F96E0F5F1F4F40
:104CF0000330110569F70E941ED80E94C85D0C940C
:104D000004120E94EF8F0C94041283E50E94FBD8DA
:104D1000882311F40C9404120E9465D870930C023D
:104D200060930B020C9404128DED90E00E94356F9D
:104D300081110C94041283E50E94FBD8882311F49E
:104D40000C9404120091920510E00E9465D8000FA7
:104D5000111FF801EF5DFD4F718360830C94041205
:104D600080E50E94CCD8882311F40C9404120E9490
:104D700065D8F62EC62ED72E83E50E94FBD8882351
:104D800021F00E9465D88B0102C00FEF1FEFC80110
:104D90000196039710F00C940412D7FE02C00C94F5
:104DA0000412E8EEF4E080E195E02491F21611F4AB
:104DB0000C94041231968E179F07B9F77EC380E5D5
:104DC0000E94CCD8882311F40C9404120E9465D858
:104DD0006B017C018B01672B19F0ECE7F2E181C0DC
:104DE00083E50E94CCD8811103C0E2EBF2E108C058
:104DF0000E9465D886E492E10E9423520C9404122A
:104E000084917F012FEFE21AF20A882321F00E9499
:104E100017D9F701F5CF60E070E089E295E00E94D4
:104E200094538091481228E532E06901C81AD108EC
:104E300087FDD394CC0CDD1CCC0CDD1C0D2C000CA0
:104E4000EE08FF088091471228E830E04901881AEF
:104E5000910887FD9394880C991C880C991C092C47
:104E6000000CAA08BB08809146128F3FB9F090E071
:104E7000FC01EE0FFF1F8E0F9F1FFC01E752FE4E3D
:104E80000181128153E0000F111F5A95E1F764E090
:104E9000169507956A95E1F70E5F1F4F98012F5FF2
:104EA0003F4FC901330FAA0BBB0B9C01AD01281961
:104EB00039094A095B09A4EBB0E00E942BF3A70172
:104EC0009601281939094A095B090E940FF3B901B3
:104ED00086E295E00E9494538AE00E9417D90C94D0
:104EE000041284918F010F5F1F4F882321F00E94CD
:104EF00017D9F801F6CFB6018FE195E00E949453DF
:104F0000E0E1F5E084918F010F5F1F4F882311F4DA
:104F10000C9404120E9417D9F801F4CF83E50E9483
:104F2000FBD8882319F00E9465D802C064E071E0C4
:104F300079A368A380E50E94FBD8882339F00E94FA
:104F400065D8693833E1730730F402C068EE73E066
:104F50007A83698304C088E893E19A838983BE01D8
:104F6000605E7F4FCE0101960E94E0940C94041283
:104F70000E94518F0C94041283E50E94CCD8182F04
:104F8000882371F00E9495D80E948FF470931302C9
:104F90006093120221E0672B09F020E02093C10703
:104FA00080E50E94CCD8882361F0209112023091D4
:104FB0001302232B11F00E9486D88093C1070C9412
:104FC000041211110C940412E2EBF2E184918F01AE
:104FD0000F5F1F4F882321F00E9417D9F801F6CFE9
:104FE0008091C107882319F068E374E002C069E585
:104FF00073E086E495E00E94AD53609112027091D7
:10500000130285E395E00E949453E1E3F5E0849177
:105010008F010F5F1F4F882311F40C9404120E941C
:1050200017D9F801F4CF81E00E949B6D0C94041213
:1050300080E00E949B6D0C9404120E947D890C9468
:10504000041240E95AE15DA74CA782EE882E86E162
:10505000982E92EDA92E96E1B92E28E7C22E2AE1CC
:10506000D22E3FE3232E32E0332E0BE91DE1E12C5B
:10507000F12CACA5BDA58D91BDA7ACA7882309F4E3
:1050800081C0F5014080518062807380D1012D91F3
:105090003D914D915C91F601608171818281938196
:1050A0000E944BF320E030E040E05FE30E9416ED09
:1050B0009B01AC01C301B2010E9471F5181654F4B2
:1050C000F80185919591A591B49188AB98AFACAB5F
:1050D000BCAF04C018AA18AE1CAA1CAED4012D91F6
:1050E0003D914D915C91C301B2010E944AF39B0135
:1050F000AC0168A978AD8CA99CAD0E944AF32B0144
:105100003C0120E030E040EA51EC0E9471F587FD5F
:105110000AC020E030E040EA51E4C301B2010E943D
:10512000B1EC18161CF4ECE7F2E109C0B301A201DE
:10513000C7010E94F96E26C00E9417D9F801849118
:105140008F010F5F1F4F8111F7CFE9E5F5E08491E3
:105150008F010F5F1F4F882321F00E9417D9F8019C
:10516000F6CF88E290E09A83898388EC90E099A357
:1051700088A3BE016F5F7F4FCE0180960E94E094AE
:105180000C940412BFEFEB1AFB0AE4E08E0E911CA4
:10519000F4E0AF0EB11C24E0C20ED11C34E0230EAB
:1051A000311C0C5F1F4F43E0E416F10409F061CF9E
:1051B0000E941ED80E94C85D83E992E099A388A34B
:1051C00004E610E01A830983BE01605E7F4FCE01C2
:1051D00001960E94E0948AEB92E099A388A31A8337
:1051E0000983BE01605E7F4FCE0101960E94E0946C
:1051F0000C9404120E94869F0C9404120E948199C0
:105200000C94041283E50E94CCD8882319F00E94E4
:1052100086D801C081E091E089270E944F850C94D7
:1052200004120E9417D9F80184918F010F5F1F4F5C
:105230008111F7CFE0EAF5E084918F010F5F1F4FF6
:10524000882309F41FCA0E9417D9F801F5CFE9E8AD
:10525000F5E084918F010F5F1F4F882309F444CA42
:105260000E9417D9F801F5CF40912E1750912F17B2
:10527000609130177091311787E795E00E9477535E
:1052800033CA0E9417D9F80184918F010F5F1F4F15
:105290008111F7CFEAEAF5E084918F010F5F1F4F8C
:1052A000882311F40C9404120E9417D9F801F4CF4A
:1052B00081E08093600283E50E94CCD8811104C014
:1052C0000E94F7B10C9404120E9486D881110C94AC
:1052D0000412F6CFF0909905FF2021F1E2EBF2E104
:1052E00084918F010F5F1F4F882321F00E9417D9EF
:1052F000F801F6CF84E50E9417D96F2D70E080E0A9
:1053000090E04AE00E941ED980E20E9417D90DE584
:1053100013E0D8018D918D01882309F4E5C90E941D
:1053200017D9F7CF10929305E2EBF2E184918F0148
:105330000F5F1F4F882321F00E9417D9F801F6CF85
:1053400060E070E089EB95E00E9494538AE00E944F
:1053500017D90C9404124091900550919105452B5A
:1053600039F4AF0141505109509391054093900594
:1053700040E050E00C94911280E00E94716B0E941A
:10538000336C83E50E94CCD8882309F44AC00E947C
:1053900086D821E0482FBE016F5F7F4FCE018096F7
:1053A0000E941E936B017C019B01AC010E94F9F5E8
:1053B000811131C02CEA35EC47E257E368A179A1AD
:1053C0008AA19BA10E944BF3AB01BC018EE493E048
:1053D0000E9477532CEA35EC47E257E369817A81E2
:1053E0008B819C810E944BF3AB01BC0189E493E06B
:1053F0000E9477532CEA35EC47E257E3C701B60128
:105400000E944BF3AB01BC0184E493E00E9477530C
:105410008AE00E9417D90E94196C0E94C85D0C9402
:10542000041281E0B6CF61E0812F0E94D0DA6E2DA8
:10543000812F0E943D95F12CB701812F0E940CDB3A
:10544000B9E0CB16D10411F00C940412F0923B1782
:10545000E0923A170C9404120E943AD788E50E9411
:10546000CCD8882319F05F9A1092F50589E50E943F
:10547000CCD8882319F08A9A1092F6058AE50E9402
:10548000CCD8882351F09FB7F894809108018160AF
:10549000809308019FBF1092F70585E40E94CCD845
:1054A000882311F40C940412129A0C9404120E9492
:1054B0003AD70E9438AE0C9404120E943AD760E0AA
:1054C0008F2D0E94D0DA0F3FEFEF1E0759F48F2D7A
:1054D0000E94149531E020E0892B09F030E0032F81
:1054E000122F05C00130110569F401E010E08F2D85
:1054F0000E9414958017910711F40C9404120E94D5
:10550000A8ABF5CF00E010E0F2CFC15ADF4F0FB6E5
:10551000F894DEBF0FBECDBFDF91CF911F910F91E9
:10552000FF90EF90DF90CF90BF90AF909F908F90C3
:105530007F906F905F904F903F902F9008952F92A3
:105540003F924F925F926F927F928F929F92AF9213
:10555000BF92CF92DF92EF92FF920F931F93CF9360
:10556000DF93CDB7DEB7C254D1090FB6F894DEBFD2
:105570000FBECDBF0E9438978091D71B823009F0B3
:10558000ABC080917712882309F4A6C06499A4C0A7
:105590008091D81B8F5F8093D81B65E070E080E01E
:1055A00090E00E94D4DB8091D81B83330CF494C02C
:1055B0008091D51B882349F081E09AE590937E1570
:1055C00080937D1586E590E008C081E09AE5909390
:1055D0007E1580937D1587E590E0909380158093EC
:1055E0007F1587E08093711582E88093741584E8B5
:1055F00090E0A0E0B0E08093751590937615A093AD
:105600007715B09378150E94566685E08093D91B74
:105610008091DA169091DB16A091DC16B091DD1620
:105620008093EA059093EB05A093EC05B093ED050C
:1056300020E030E040E251E46091DE167091DF1628
:105640008091E0169091E1160E944AF36093E6057E
:105650007093E7058093E8059093E905109277121F
:105660000E9410C98091E4059091E505892B41F4D1
:1056700080912206909123069093E5058093E4059E
:105680008091AD059091AE05892B41F48091200663
:10569000909121069093AE058093AD05109221065E
:1056A000109220060E944FC681E08093DC15109274
:1056B000D81B1092D71B84E08093391710923517AE
:1056C0001092F91B1092F81B8EE597E0909315113C
:1056D000809314110E94C5D70E9485B991ECA92E20
:1056E00095E1B92E2AE1722E86E191E10E9479C1FD
:1056F0008090AF059090B0051816190634F42AE191
:105700008216910414F40C94D2491814190414F05C
:105710000C94FD49909122158091C115981322C0D7
:10572000909123158091C21598131CC023E0821616
:105730009104C4F09091C315909321158091C415E4
:10574000809324159330D9F4982F9D7F9038B9F425
:105750009091C5159F3409F05BC09091C6159B349C
:1057600009F056C08AE1E1ECF5E1DF011D928A956E
:10577000E9F71092B0051092AF050C94FD498338FB
:1057800009F046C08091C5159091C61598278927C4
:105790009827A0E0B0E08093251590932615A0935C
:1057A0002715B09328154091C71550E060E070E0D0
:1057B0004093291550932A1560932B1570932C153F
:1057C00088EC682E85E1782E80E090E0DC0184177B
:1057D0009507A607B70708F049C09C01359527959E
:1057E000F901EE0FFF1F9F01235D3A4E5901F301AE
:1057F000208130E0322F222791802929F501318341
:1058000020830296A11DB11DF2E06F0E711CDFCF47
:10581000813861F58091C51590E0A0E0B0E08093FB
:10582000251590932615A0932715B09328158091E0
:10583000C615482F50E060E070E040932915509362
:105840002A1560932B1570932C15A7ECB5E1EDE2AA
:10585000F5E190E020E030E02817390739F04D916C
:1058600050E0419351932F5F3F4FF6CF8AE1E1EC37
:10587000F5E1DF011D928A95E9F71092B0051092CB
:10588000AF058091D91B181614F40C94C4494091AB
:105890002515509126156091271570912815A9E6B8
:1058A000B2E0E0E0F0E08D909D90AD90BD9081146D
:1058B0009104A104B104B1F184169506A606B706B9
:1058C00079F5DB01CA0188509041A109B10905971A
:1058D000A105B10550F1DB01CA01877F82339041F8
:1058E000A105B10529F1443330E153076105710584
:1058F000F9F0DB01CA0186549041A109B10907976B
:10590000A105B105C0F0DB01CA0184559041A10990
:10591000B1090597A105B10580F4E2E1F0E00DC001
:105920003196C1CFEFEFFFEF08C0E3E0F0E005C034
:10593000E8E0F0E002C0EFE0F0E0DB01CA018A50ED
:105940009042A109B109833D9105A105B10510F46B
:105950000C949746EF3F8FEFF80711F40C94C4496D
:10596000EA31F10510F00C94C4498827EE58FF4F36
:105970008F4F0C944BF680912D1590912E15813000
:10598000910509F052C010923C0281E080933E17CD
:105990008FEF809342170E9438978091D51B882300
:1059A00011F181E09AE590937E1580937D1582E058
:1059B00090E09093801580937F1587E08093711518
:1059C00082E88093741584E890E0A0E0B0E08093D2
:1059D000751590937615A0937715B09378150E945E
:1059E00056660C94C44981E09AE590937E158093A5
:1059F0007D158EE290E09093801580937F1587E06F
:105A00008093711582E88093741584E890E0A0E09B
:105A1000B0E08093751590937615A0937715B093A9
:105A200078150E9456660C94C4498230910509F09D
:105A3000F7C081E080933C02109235170E94278ABC
:105A40008BE090E090937E1580937D1505E00093A8
:105A5000711512E81093741580E092E1A0E0B0E0B7
:105A60008093751590937615A0937715B09378155C
:105A70000E94566610927E1510927D150093711546
:105A8000109374158EE090E1A0E0B0E0809375155E
:105A900090937615A0937715B09378150E9456666B
:105AA00010927E1510927D15009371151093741548
:105AB0008FE090E1A0E0B0E08093751590937615AB
:105AC000A0937715B09378150E94566610927E15B4
:105AD00010927D15009371151093741586E190E175
:105AE000A0E0B0E08093751590937615A09377159C
:105AF000B09378150E94566662E070E080E090E016
:105B00000E94D4DB10927E1510927D1500937115C2
:105B10001093741580E190E1A0E0B0E080937515DA
:105B200090937615A0937715B09378150E945666DA
:105B300010927E1510927D150093711510937415B7
:105B400082E190E1A0E0B0E0809375159093761526
:105B5000A0937715B09378150E945666109268123C
:105B60001092671210926D1210926E1210926F12B4
:105B7000109270121092711210927212109273128F
:105B8000109274121092691210926A1210926B1293
:105B900010926C128091D51B882309F181E09AE55F
:105BA00090937E1580937D1581E090E09093801511
:105BB00080937F1587E0809371151093741584E8A6
:105BC00090E0A0E0B0E08093751590937615A093D7
:105BD0007715B09378150E9456660C94C44981E0FD
:105BE0009AE590937E1580937D158DE290E09093D9
:105BF000801580937F1587E080937115109374153D
:105C000084E890E0A0E0B0E080937515909376155D
:105C1000A0937715B09378150E9456660C94C449EA
:105C20008330910509F098C081E080933C02109286
:105C300035179091D51B80913E02992309F446C0F7
:105C4000882311F181E09AE590937E1580937D156C
:105C500080E190E09093801580937F1587E080939A
:105C6000711582E88093741584E890E0A0E0B0E0BC
:105C70008093751590937615A0937715B09378154A
:105C80000E9456660C94C44981E09AE590937E1573
:105C900080937D158FE090E09093801580937F1521
:105CA00087E08093711582E88093741584E890E012
:105CB000A0E0B0E08093751590937615A0937715CA
:105CC000B09378150E9456660C94C449882311F14C
:105CD00081E09AE590937E1580937D158AE390E0AC
:105CE0009093801580937F1587E08093711582E8EB
:105CF0008093741584E890E0A0E0B0E0809375157F
:105D000090937615A0937715B09378150E945666F8
:105D10000C94C44981E09AE590937E1580937D159B
:105D200089E390E09093801580937F1587E08093BE
:105D3000711582E88093741584E890E0A0E0B0E0EB
:105D40008093751590937615A0937715B093781579
:105D50000E9456660C94C449049711F00C94C449EF
:105D600010923C020C94C44980912D1590912E15EF
:105D700081309105E1F580913E028823E1F082E0D7
:105D800090E090937E1580937D1585E0809371154A
:105D900082E8809374158EE190E1A0E0B0E08093FA
:105DA000751590937615A0937715B09378150E948A
:105DB00056660C94C44983E090E090937E158093DE
:105DC0007D1585E08093711582E8809374158EE1CE
:105DD00090E1A0E0B0E08093751590937615A093C4
:105DE0007715B09378150E9456660C94C44982309A
:105DF000910509F0FCC081E080933C029091391735
:105E00008091D51B933009F046C0882311F181E0C1
:105E10009AE590937E1580937D158AE090E09093AB
:105E2000801580937F1587E08093711582E88093B9
:105E3000741584E890E0A0E0B0E08093751590932D
:105E40007615A0937715B09378150E9456660C943A
:105E5000C44981E09AE590937E1580937D1584E393
:105E600090E09093801580937F1587E08093711563
:105E700082E88093741584E890E0A0E0B0E080931D
:105E8000751590937615A0937715B09378150E94A9
:105E900056660C94C449943009F063C0882311F10C
:105EA00081E09AE590937E1580937D158CE090E0DB
:105EB0009093801580937F1587E08093711582E819
:105EC0008093741584E890E0A0E0B0E080937515AD
:105ED00090937615A0937715B09378150E94566627
:105EE0000C94C44981E09AE590937E1580937D15CA
:105EF00086E390E09093801580937F1587E08093F0
:105F0000711582E88093741584E890E0A0E0B0E019
:105F10008093751590937615A0937715B0937815A7
:105F20000E9456660C94C449483090E159076105B7
:105F3000710509F0CEC19091DC158091D51B91308F
:105F400009F455C191115BC120912D1530912E1589
:105F5000203F310509F053C190913917933009F46E
:105F600054CF882311F181E09AE590937E158093B8
:105F70007D158BE090E09093801580937F1587E0EE
:105F80008093711582E88093741584E890E0A0E016
:105F9000B0E08093751590937615A0937715B09324
:105FA00078150E9456660C94C44981E09AE5909356
:105FB0007E1580937D1585E390E090938015809306
:105FC0007F1587E08093711582E88093741584E8CB
:105FD00090E0A0E0B0E08093751590937615A093C3
:105FE0007715B09378150E9456660C94C449833097
:105FF000910509F049C020913E02222311F19093AE
:106000007E1580937D1585E08093711582E88093DD
:1060100074158EE190E1A0E0B0E080937515909347
:106020007615A0937715B09378150E9456668FEF7A
:1060300090E090933B1780933A1710923E020C9495
:10604000C44982E090E090937E1580937D1585E0B1
:106050008093711582E8809374158EE190E1A0E041
:10606000B0E08093751590937615A0937715B09353
:1060700078150E94566610923B1710923A1781E0ED
:1060800080933E020C94C449049711F00C94C449C7
:1060900080910D02882309F452C082E090E0909331
:1060A0007E1580937D1505E00093711512E810931D
:1060B00074158FE190E1A0E0B0E0809375159093A6
:1060C0007615A0937715B09378150E945666809147
:1060D000AD059091AE050097D1F090932106809385
:1060E000200690937E1580937D1500937115109373
:1060F00074158AE390E1A0E0B0E080937515909369
:106100007615A0937715B09378150E945666109275
:106110000D02109204028091D51B882319F088E0AB
:1061200090E002C08AE090E090937E1580937D1508
:1061300085E08093711582E88093741538C083E000
:1061400090E090937E1580937D1505E00093711586
:1061500012E8109374158FE190E1A0E0B0E0809315
:10616000751590937615A0937715B09378150E94C6
:10617000566680912006909121069093AE058093FB
:10618000AD0581E080930D02809304028091D51BC0
:10619000882319F087E090E002C089E090E09093B6
:1061A0007E1580937D15009371151093741588E109
:1061B00090E1A0E0B0E08093751590937615A093E0
:1061C0007715B09378150E94566660910D0280E6AF
:1061D00090E00E94D0F20C94C44980912D159091CA
:1061E0002E1590930C0280930B020C94C4492091BD
:1061F0002D1530912E15203F310509F44FCE8823FF
:1062000049F081E09AE590937E1580937D1586E5AF
:1062100090E008C081E09AE590937E1580937D150B
:1062200087E590E09093801580937F1587E08093B9
:10623000711582E88093741584E890E0A0E0B0E0E6
:106240008093751590937615A0937715B093781574
:106250000E94566610927E1510927D1505E00093FF
:10626000711512E81093741580E190E1A0E0B0E0A0
:106270008093751590937615A0937715B093781544
:106280000E94566610927E1510927D15009371152E
:106290001093741582E190E1A0E0B0E08093751551
:1062A00090937615A0937715B09378150E94566653
:1062B0001092F91B1092F81B10923F171092AE0526
:1062C0001092AD051092E5051092E4050E948590AC
:1062D00050C24A30A0E15A076105710509F098C023
:1062E00080912D1590912E15813F910511F00C9400
:1062F000C4498091D51B882349F081E09AE59093A9
:106300007E1580937D1586E590E008C081E09AE5D2
:1063100090937E1580937D1587E590E0909380158E
:1063200080937F1587E08093711582E880937415C0
:1063300084E890E0A0E0B0E0809375159093761526
:10634000A0937715B09378150E94566681E08093EC
:10635000D91B8091DA169091DB16A091DC16B091D2
:10636000DD168093EA059093EB05A093EC05B093BE
:10637000ED0520E030E040E251E46091DE167091DE
:10638000DF168091E0169091E1160E944AF3609327
:10639000E6057093E7058093E8059093E905109270
:1063A00077120E9410C98091E4059091E505892B30
:1063B00041F480912206909123069093E505809305
:1063C000E4058091AD059091AE05892B41F4809153
:1063D0002006909121069093AE058093AD05109212
:1063E0002106109220060E944FC681E08093DC15A2
:1063F00084E0809339171092F91B1092F81B84E502
:1064000097E090931511809314110E94C5D7B1C1E4
:106410004C3050416105710509F0ABC180912D15DB
:1064200090912E15019709F0A4C180E090E00E94A0
:106430005AC8892B09F485C08091220690912306C1
:10644000893B9105B4F11092AC051092AB0515E0B3
:10645000A12E02E8B02E8EE8C82E80E1D82EE12CC5
:10646000F12C0091AB051091AC050530110514F02D
:106470000C94C44910937E1500937D15A09271155C
:10648000B0927415C0927515D0927615E09277157A
:10649000F09278150E94566660E971E080E090E025
:1064A0000E94D4DB0F5F1F4F1093AC050093AB0528
:1064B000D8CF8091D51B882311F181E09AE5909384
:1064C0007E1580937D158CE290E0909380158093EB
:1064D0007F1587E08093711582E88093741584E8B6
:1064E00090E0A0E0B0E08093751590937615A093AE
:1064F0007715B09378150E9456660C94C44981E0D4
:106500009AE590937E1580937D1581E590E09093B8
:10651000801580937F1587E08093711582E88093C2
:10652000741584E890E0A0E0B0E080937515909336
:106530007615A0937715B09378150E9456660C9443
:10654000C4498091D51B882349F081E09AE5909356
:106550007E1580937D1586E590E008C081E09AE580
:1065600090937E1580937D1587E590E0909380153C
:1065700080937F1587E08093711582E8809374156E
:1065800084E890E0A0E0B0E08093751590937615D4
:10659000A0937715B09378150E9456667E01EFE1BF
:1065A000EE0EF11CA0E1BA2ED701EB2D1D92EA955B
:1065B000E9F76091EA057091EB058091EC05909107
:1065C000ED05870122E043E00E94EEE79E012F5F88
:1065D0003F4F6901D9011D92BA94E9F76091E60530
:1065E0007091E7058091E8059091E905890122E025
:1065F00043E00E94EEE706EC15E0BEE1BB2EF80199
:106600002B2D11922A95E9F78091AE058F938091F9
:10661000AD058F938BE497E09F938F931F930F9318
:106620000E9483ECC8010E941D67D801EB2D1D92CA
:10663000EA95E9F78091E5058F938091E4058F93C2
:1066400082E497E09F938F931F930F930E9483ECB4
:10665000C8010E941D67D8011D92BA94E9F7FF9204
:10666000EF928BE397E09F938F931F930F930E947A
:1066700083ECC8010E941D67DF92CF9283E397E00D
:106680009F938F931F930F930E9483ECC8010E94E6
:106690001D671092AE051092AD051092E50510929F
:1066A000E4050FB6F894DEBF0FBECDBF809178121F
:1066B000882319F081E0809377120E94B8C88091F6
:1066C000D51B882319F081E090E002C08DE090E0B6
:1066D00090937E1580937D1585E08093711582E8F7
:1066E0008093741584E190E1A0E0B0E0809375158B
:1066F00090937615A0937715B09378150E945666FF
:106700001092DC151092F91B1092F81B83E0809315
:10671000391781E080933F178091D51B882349F07A
:1067200081E09AE590937E1580937D158AE090E054
:1067300008C081E09AE590937E1580937D1584E3EF
:1067400090E09093801580937F1587E0809371157A
:1067500082E88093741584E890E0A0E0B0E0809334
:10676000751590937615A0937715B09378150E94C0
:1067700056668091251590912615A0912715B09108
:1067800028158C309041A105B10511F00C94C44935
:1067900080912D1590912E15029711F00C94C449FB
:1067A00081E08093AA058091E4059091E50590939E
:1067B0002306809322061092AC051092AB058091BF
:1067C000D51B882309F181E09AE590937E1580938B
:1067D0007D1587E090E09093801580937F158093DE
:1067E000711582E88093741584E890E0A0E0B0E031
:1067F0008093751590937615A0937715B0937815BF
:106800000E9456660C94C44981E09AE590937E15E7
:1068100080937D1582E590E09093801580937F159D
:1068200087E08093711582E88093741584E890E086
:10683000A0E0B0E08093751590937615A09377153E
:10684000B09378150E9456660C94C44920912D157A
:1068500030912E15B90180E090E037FF09C00E9409
:10686000B5EC20E030E040E857E40E944AF302C073
:106870000E94B5EC20E030E048EC52E40E9427F49E
:1068800060932E1770932F178093301790933117C2
:10689000C0902E17D0902F17E0903017F09031173E
:1068A00020E030E040EA51ECC701B6010E9471F5EA
:1068B00087FF02C00C94C44920E030E040EA51E474
:1068C000C701B6010E94B1EC181614F40C94C44927
:1068D0008091F705882311F40C94C4490091B41BEE
:1068E0001091B51B20910A0630910B0640910C06C1
:1068F00050910D06C701B6010E944AF320E030E036
:1069000040EA52E40E9416ED0E948FF4600F711F5E
:106910007093B51B6093B41B0C94C44980912D15E2
:1069200090912E15009739F481E080933C021092EB
:1069300035170C94C4499C0121503109223031058E
:1069400010F40C94C4498330910509F0B8C09091BB
:106950003E028091D51B992309F464C02FEF30E0EB
:1069600030933B1720933A1710923E028823C1F1CF
:1069700081E09AE590937E1580937D158FE090E0FD
:106980009093801580937F1587E08093711582E83E
:106990008093741584E890E0A0E0B0E080937515D2
:1069A00090937615A0937715B09378150E9456664C
:1069B0000C94C449423320E152076105710509F086
:1069C0000CC280912D1590912E15009709F0C2C12F
:1069D0009091D51B80913E029111B9C181114DC09A
:1069E00081E09AE590937E1580937D1589E390E090
:1069F0009093801580937F1587E08093711582E8CE
:106A00008093741584E890E0A0E0B0E08093751561
:106A100090937615A0937715B09378150E945666DB
:106A20000C94C44910923B1710923A1791E090933E
:106A30003E02882311F181E09AE590937E158093C0
:106A40007D1580E190E09093801580937F1587E01D
:106A50008093711582E88093741584E890E0A0E03B
:106A6000B0E08093751590937615A0937715B09349
:106A700078150E9456660C94C44981E09AE590937B
:106A80007E1580937D158AE390E090938015809326
:106A90007F1587E08093711582E88093741584E8F0
:106AA00090E0A0E0B0E08093751590937615A093E8
:106AB0007715B09378150E9456660C94C4498530BA
:106AC000910509F04BC080E090E0A9E3B3E4809326
:106AD000000290930102A0930202B093030289EB9B
:106AE00090E00E94E7C6FDE2EF2EF12CF092210625
:106AF000E09220060E944FC689EB90E090937E15AD
:106B000080937D1505E00093711512E810937415BC
:106B100084E390E1A0E0B0E0809375159093761542
:106B2000A0937715B09378150E945666F0927E1563
:106B3000E0927D1500937115109374158AE390E12E
:106B4000A0E0B0E08093751590937615A09377152B
:106B5000B09378150E9456660C94C449863091050E
:106B600009F04BC080E090E0A0E7B3E4809300021E
:106B700090930102A0930202B093030280EF90E091
:106B80000E94E7C6EEE6EE2EF12CF0922106E0928E
:106B900020060E944FC680EF90E090937E15809370
:106BA0007D1505E00093711512E81093741584E3C8
:106BB00090E1A0E0B0E08093751590937615A093D6
:106BC0007715B09378150E945666F0927E15E09284
:106BD0007D1500937115109374158AE390E1A0E080
:106BE000B0E08093751590937615A0937715B093C8
:106BF00078150E9456660C94C449813F910511F0A6
:106C00000C94C4498FEF90E090933B1780933A1710
:106C100010923E020E94EDC610927E1510927D15D4
:106C200005E00093711512E81093741584E390E168
:106C3000A0E0B0E08093751590937615A09377153A
:106C4000B09378150E94566661E070E080E090E0B5
:106C50000E94D4DB10927E1510927D150093711561
:106C6000109374158AE390E1A0E0B0E0809375156D
:106C700090937615A0937715B09378150E94566679
:106C800061E070E080E090E00E94D4DB8091D51B51
:106C9000882309F188E090E090937E1580937D151C
:106CA000009371151093741584E190E1A0E0B0E0B9
:106CB0008093751590937615A0937715B0937815FA
:106CC0000E94566681E09AE590937E1580937D152B
:106CD0008FE090E020C084E190E090937E15809357
:106CE0007D15009371151093741584E190E1A0E077
:106CF000B0E08093751590937615A0937715B093B7
:106D000078150E94566681E09AE590937E158093EF
:106D10007D1589E390E09093801580937F1587E03F
:106D2000809371151093741584E890E0A0E0B0E0B2
:106D30008093751590937615A0937715B093781579
:106D40000E94566682E0809339170C94C4498111E1
:106D500072CE0ECE81309105F1F41092230610927E
:106D6000220610927E1510927D1585E08093711594
:106D700082E88093741584E390E1A0E0B0E0809312
:106D8000751590937615A0937715B09378150E949A
:106D900056660C94C449029711F00C94C4491092A1
:106DA00021061092200610927E1510927D1585E026
:106DB0008093711582E8809374158AE390E1A0E0D6
:106DC000B0E08093751590937615A0937715B093E6
:106DD00078150E9456660C94C449443330E1530739
:106DE0006105710561F480912D1590912E15909398
:106DF0002306809322060E94E7C60C94C4494A33B6
:106E000050416105710511F00C94C44980912D1514
:106E100090912E158E37910514F08DE790E09093A8
:106E20002106809320060E944FC60C94C44980918D
:106E30002D1590912E15009709F476CD813091058E
:106E400009F09FC080910E06882319F082E090E03F
:106E500002C083E090E090937E1580937D1585E0DD
:106E60008093711582E88093741585E490E1A0E029
:106E7000B0E08093751590937615A0937715B09335
:106E800078150E9456668AE090E090937E15809374
:106E90007D1585E08093711512E81093741580E0DC
:106EA00092E1A0E0B0E08093751590937615A093E1
:106EB0007715B09378150E94566686E08093D91BAB
:106EC00081E08093361780933C021092A7051092C0
:106ED000F91B1092F81B8FE297E0909315118093A5
:106EE00014110E94C5D782E297E090931511809308
:106EF00014110E94C5D78091D51B882309F181E028
:106F00009AE590937E1580937D1580E290E09093B2
:106F1000801580937F1587E0809371151093741509
:106F200084E890E0A0E0B0E080937515909376152A
:106F3000A0937715B09378150E9456660C94C449B7
:106F400081E09AE590937E1580937D158AE490E028
:106F50009093801580937F1587E08093711510932F
:106F6000741584E890E0A0E0B0E0809375159093EC
:106F70007615A0937715B09378150E9456660C94F9
:106F8000C4498230910509F0ECC081E080933C0255
:106F90001092351788E0EFE9F5E0DF011D928A9540
:106FA000E9F780E090E0A0E2B1E480939F05909340
:106FB000A005A093A105B093A2058093A30590938B
:106FC000A405A093A505B093A60584E690E0909350
:106FD0007E1580937D1505E00093711512E81093DE
:106FE000741584E590E1A0E0B0E08093751590936E
:106FF0007615A0937715B09378150E94566620E019
:1070000030E040E251E46091A3057091A4058091C5
:10701000A5059091A6050E9416ED0E948FF470932D
:107020007E1560937D15009371151093741588E596
:1070300090E1A0E0B0E08093751590937615A09351
:107040007715B09378150E9456666091FC05709193
:10705000FD058091FE059091FF050E948FF47093CD
:107060007E1560937D15009371151093741586E35A
:1070700090E1A0E0B0E08093751590937615A09311
:107080007715B09378150E945666809122069091EC
:1070900023060E94E7C680912206909123069093D2
:1070A0007E1580937D15009371151093741584E3FC
:1070B00090E1A0E0B0E08093751590937615A093D1
:1070C0007715B09378150E94566662E070E080E014
:1070D00090E00E94D4DB8091D51B882309F181E0E8
:1070E0009AE590937E1580937D1587E190E09093CB
:1070F000801580937F1587E0809371151093741528
:1071000084E890E0A0E0B0E0809375159093761548
:10711000A0937715B09378150E9456660C94C449D5
:1071200081E09AE590937E1580937D1581E490E04F
:107130009093801580937F1587E08093711510934D
:10714000741584E890E0A0E0B0E08093751590930A
:107150007615A0937715B09378150E9456660C9417
:10716000C4498330910509F0C2C010928E0520E019
:1071700030E040E251E46091D2167091D3168091D4
:10718000D4169091D5160E9416ED0E948FF470933C
:107190007E1560937D1505E00093711512E810933C
:1071A000741588E490E1A0E0B0E0809375159093A9
:1071B0007615A0937715B09378150E94566620E057
:1071C00030E040E251E46091D6167091D71680917C
:1071D000D8169091D9160E9416ED0E948FF47093E4
:1071E0007E1560937D1500937115109374158AE4D4
:1071F00090E1A0E0B0E08093751590937615A09390
:107200007715B09378150E94566620E030E040E292
:1072100051E46091DA167091DB168091DC16909142
:10722000DD160E9416ED0E948FF470937E15609318
:107230007D1500937115109374158CE490E1A0E016
:10724000B0E08093751590937615A0937715B09361
:1072500078150E94566662E070E080E090E00E943F
:10726000D4DB8091D51B882309F181E09AE59093C6
:107270007E1580937D158DE190E09093801580932D
:107280007F1587E0809371151093741584E890E062
:10729000A0E0B0E08093751590937615A0937715D4
:1072A000B09378150E9456660C94C44981E09AE523
:1072B00090937E1580937D1587E490E090938015E0
:1072C00080937F1587E0809371151093741584E87F
:1072D00090E0A0E0B0E08093751590937615A093B0
:1072E0007715B09378150E9456660C94C449843083
:1072F000910511F40C94C44985309105A1F4809155
:10730000D51B4EE750E160E070E0882331F08EE657
:1073100093E00E940CC80C94C44980E893E00E945A
:107320000CC80C94C449069711F00C94C4498EE122
:1073300097E090931511809314110E94C5D78BE0AC
:1073400090E090937E1580937D1585E08093711574
:1073500082E88093741580E092E1A0E0B0E0809331
:10736000751590937615A0937715B09378150E94B4
:1073700056660C94C44980912D1590912E15019755
:1073800009F077C080EA9FE09093F91B8093F81B87
:1073900010923C02C0902E17D0902F17E09030171B
:1073A000F0903117A701960160910A0670910B06C3
:1073B00080910C0690910D060E94B1EC882361F13A
:1073C000C0920A06D0920B06E0920C06F0920D06CF
:1073D00020E030E048EC52E4C701B6010E9416ED0F
:1073E0000E948FF470937E1560937D1585E08093E5
:1073F000711582E88093741586E290E1A0E0B0E018
:107400008093751590937615A0937715B0937815A2
:107410000E9456660E94869F8091D51B882349F062
:1074200081E09AE590937E1580937D1585E190E04B
:1074300008C081E09AE590937E1580937D158FE3D7
:1074400090E09093801580937F1587E0809371156D
:1074500082E88093741584E890E0A0E0B0E0809327
:10746000751590937615A0937715B09378150E94B3
:10747000566680912D1590912E15029711F00C945F
:10748000C4498091D51B882311F181E09AE590933E
:107490007E1580937D1586E190E090938015809312
:1074A0007F1587E08093711582E88093741584E8D6
:1074B00090E0A0E0B0E08093751590937615A093CE
:1074C0007715B09378150E9456660C94C44981E0F4
:1074D0009AE590937E1580937D1580E490E09093DB
:1074E000801580937F1587E08093711582E88093E3
:1074F000741584E890E0A0E0B0E080937515909357
:107500007615A0937715B09378150E9456660C9463
:10751000C44980912D1590912E1581309105F1F47B
:107520000E943AD786E08093D91B10923C0281E0FA
:10753000809336178091F505882321F08091F60518
:10754000811103C08AE197E002C083E197E0909344
:107550001511809314110E94C5D7F0C18230910596
:1075600071F52DEC3CEC4CEC5DE360912E177091C5
:107570002F1780913017909131170E944BF36B01B8
:107580007C0120E030E040EA51EC0E9471F587FD7B
:10759000D5C120E030E040EA51E4C701B6010E94C5
:1075A000B1EC18160CF4CAC18091F7058823D9F103
:1075B0008091B41B9091B51B805B9F4F30C083308E
:1075C0009105D1F52DEC3CEC4CEC5DE360912E1770
:1075D00070912F1780913017909131170E944AF3C4
:1075E0006B017C0120E030E040EA51EC0E9471F533
:1075F00087FDA4C120E030E040EA51E4C701B601B4
:107600000E94B1EC18160CF499C18091F7058823FB
:1076100051F08091B41B9091B51B805591099093C6
:10762000B51B8093B41BC0922E17D0922F17E092F7
:107630003017F092311782C18430910549F584E00A
:107640008093D91B8FE097E09093151180931411CC
:107650000E94C5D78BE097E0909315118093141189
:107660000E94C5D78091D51B882349F081E09AE517
:1076700090937E1580937D158CE190E0C9C181E0E7
:107680009AE590937E1580937D1584E590E0C0C1C6
:107690008530910509F04CC083E08093D91B81E0CF
:1076A00090E090937E1580937D1585E08093711511
:1076B00012E8109374158DE890E1A0E0B0E080939B
:1076C000751590937615A0937715B09378150E9451
:1076D00056668091D51B882349F081E09AE5909306
:1076E0007E1580937D158BE290E008C081E09AE5DD
:1076F00090937E1580937D1585E590E0909380159D
:1077000080937F1587E0809371151093741584E83A
:1077100090E0A0E0B0E08093751590937615A0936B
:107720007715B09378150E94566687E097E00FCFE3
:1077300086309105B1F484E08093D91B8CEF96E0FC
:1077400090931511809314110E94C5D789EE96E08D
:1077500090931511809314110E94C5D78EED96E079
:107760004AC087309105B1F484E08093D91B83ED42
:1077700096E090931511809314110E94C5D782EC66
:1077800096E090931511809314110E94C5D787EB52
:1077900096E031C088309105B1F484E08093D91B24
:1077A0008CEA96E090931511809314110E94C5D72E
:1077B0008AE996E090931511809314110E94C5D721
:1077C0008FE896E018C089309105F1F484E0809349
:1077D000D91B84E896E090931511809314110E94B0
:1077E000C5D781E796E090931511809314110E94FC
:1077F000C5D786E696E090931511809314110E94E8
:10780000C5D71092D91B9AC08A309105B1F484E093
:107810008093D91B8BE596E09093151180931411FA
:107820000E94C5D789E496E09093151180931411B6
:107830000E94C5D78EE396E0DECF0B9709F07EC09D
:1078400080910E068823F9F083E090E090937E15F6
:1078500080937D1585E08093711582E8809374157F
:1078600085E490E1A0E0B0E08093751590937615E3
:10787000A0937715B09378150E94566610920E0665
:1078800086E396E01FC082E090E090937E1580939F
:107890007D1585E08093711582E88093741585E4E9
:1078A00090E1A0E0B0E08093751590937615A093D9
:1078B0007715B09378150E94566681E080930E0686
:1078C0008EE296E090931511809314110E94C5D713
:1078D00060912E1770912F1780913017909131176A
:1078E00060930A0670930B0680930C0690930D0626
:1078F00020E030E048EC52E40E9416ED0E948FF444
:1079000070937E1560937D1585E08093711582E8F4
:107910008093741586E290E1A0E0B0E08093751545
:1079200090937615A0937715B09378150E945666BC
:1079300060910E068CE590E00E94D0F28AE090E023
:1079400090937E1580937D1585E08093711582E874
:107950008093741580E092E1A0E0B0E0809375150B
:1079600090937615A0937715B09378150E9456667C
:107970000C94C44984E08093D91B80912D1590917B
:107980002E154834B0E15B076105710509F45FC04D
:107990004A34E0E15E076105710509F461C04C34C9
:1079A000F0E15F076105710509F463C04634504199
:1079B0006105710509F065C08330910509F041C08A
:1079C0008AE296E090931511809314110E94C5D716
:1079D00081E08093361780933C021092A7051092A5
:1079E000F91B1092F81B8091D51B882349F081E088
:1079F0009AE590937E1580937D1580E290E008C013
:107A000081E09AE590937E1580937D158AE490E05D
:107A10009093801580937F1587E08093711582E89D
:107A20008093741584E890E0A0E0B0E08093751531
:107A300090937615A0937715B09378150E945666AB
:107A40007DCF80938E051092D91B0C94C449C12C14
:107A5000D12C74EBE72E73E4F72E00E010E011C098
:107A6000C12CD12C64EBE62E63E4F62E01E010E08D
:107A700008C0C12CD12C5DECE52E53E4F52E02E0BC
:107A800010E0BC0180E090E00E94B5EC20E030E026
:107A900040E251E40E9427F42B013C0120E030E059
:107AA000A9010E94B1EC5801AA0CBB1CAA0CBB1C7A
:107AB00087FF08C0F501EE52F94E10821182128242
:107AC000138214C0A7019601C301B2010E9471F58F
:107AD000F501EE52F94E18162CF040825182628266
:107AE000738204C0C082D182E282F382C8010E9404
:107AF00002B920E030E040E251E46091D21670918A
:107B0000D3168091D4169091D5160E9416ED0E943E
:107B10008FF470937E1560937D1505E000937115C9
:107B200012E81093741588E490E1A0E0B0E080932F
:107B3000751590937615A0937715B09378150E94DC
:107B4000566620E030E040E251E46091D616709134
:107B5000D7168091D8169091D9160E9416ED0E94E2
:107B60008FF470937E1560937D15009371151093BB
:107B700074158AE490E1A0E0B0E0809375159093CD
:107B80007615A0937715B09378150E94566620E07D
:107B900030E040E251E46091DA167091DB1680919A
:107BA000DC169091DD160E9416ED0E948FF4709302
:107BB0007E1560937D1500937115109374158CE4F8
:107BC00090E1A0E0B0E08093751590937615A093B6
:107BD0007715B09378150E94566661E070E080E0FA
:107BE00090E00E94D4DB8AE090E090937E15809331
:107BF0007D15009371151093741580E092E1A0E05B
:107C0000B0E08093751590937615A0937715B09397
:107C100078150E9456661092D91B0C94C44983E0D3
:107C200090E00E945AC8892B11F00C94C4498091AD
:107C3000251590912615A0912715B0912815863508
:107C400030E19307A105B10509F0E5C280912D153A
:107C500090912E1581309105C9F480919305809300
:107C60009E051092930520919F053091A0054091AB
:107C7000A1055091A2056091DE167091DF168091EA
:107C8000E0169091E1160E944AF31CC082309105E3
:107C900009F008C18091930580939E051092930589
:107CA00020919F053091A0054091A1055091A2051A
:107CB0006091DE167091DF168091E0169091E116CA
:107CC0000E944BF36093DE167093DF168093E016EC
:107CD0009093E1168091A905882309F458C083E0A8
:107CE00090E00E9402B920E030E040E251E460916F
:107CF0009F057091A0058091A1059091A2050E9419
:107D000016ED0E948FF470937E1560937D1505E04B
:107D10000093711512E81093741584E590E1A0E0CA
:107D2000B0E08093751590937615A0937715B09376
:107D300078150E94566620E030E040E251E4609100
:107D4000A3057091A4058091A5059091A6050E94B8
:107D500016ED0E948FF470937E1560937D1500934D
:107D600071151093741588E590E1A0E0B0E0809360
:107D7000751590937615A0937715B09378150E949A
:107D8000566680919E05809393050C94C449C090DB
:107D90000002D0900102E0900202F090030220E085
:107DA00030E040EA50E4C701B6010E944AF39B016B
:107DB000AC016091FC057091FD058091FE059091EC
:107DC000FF050E94B1EC87FF8ACF81E08093A9056F
:107DD000C701B6010E948FF470937E1560937D15E4
:107DE00085E08093711582E88093741580E290E1BC
:107DF000A0E0B0E08093751590937615A093771569
:107E0000B09378150E94566665E070E080E090E0DF
:107E10000E94D4DB8091D51B882311F181E09AE583
:107E200090937E1580937D1588E190E09093801566
:107E300080937F1587E08093711582E88093741595
:107E400084E890E0A0E0B0E08093751590937615FB
:107E5000A0937715B09378150E9456660C94C44988
:107E600081E09AE590937E1580937D1582E490E001
:107E70009093801580937F1587E08093711582E839
:107E80008093741584E890E0A0E0B0E080937515CD
:107E900090937615A0937715B09378150E94566647
:107EA0000C94C44983309105D1F48091930580935B
:107EB0009E0511E0109393052091A3053091A40530
:107EC0004091A5055091A6056091DE167091DF16D0
:107ED0008091E0169091E1160E944AF31DC0843013
:107EE000910509F046C08091930580939E0511E0AD
:107EF000109393052091A3053091A4054091A50509
:107F00005091A6056091DE167091DF168091E01603
:107F10009091E1160E944BF36093DE167093DF168A
:107F20008093E0169093E1168091A9058111D7CE38
:107F3000C0900002D0900102E0900202F090030293
:107F400020E030E040EA50E4C701B6010E944AF365
:107F50009B01AC016091FC057091FD058091FE05CF
:107F60009091FF050E94B1EC87FFB9CE1093A9054F
:107F70002FCF8530910509F0ECC081E08093A805F2
:107F80000091220610912306C0900002D0900102B9
:107F9000E0900202F0900302B801012E000C880B61
:107FA000990B0E94B7ECA70196010E9471F587FF1B
:107FB00005C0C701B6010E948FF48B011093230600
:107FC0000093220620E030E048EC52E46091FC058A
:107FD0007091FD058091FE059091FF050E9416EDC0
:107FE0006B017C01B801110F880B990B0E94B7EC53
:107FF0009B01AC01C701B6010E9427F40E9494F4D2
:108000006436710510F064E670E070937E1560933D
:108010007D1505E00093711512E81093741584E244
:1080200090E1A0E0B0E08093751590937615A09351
:108030007715B09378150E9456666091FC05709193
:10804000FD058091FE059091FF050E948FF47093CD
:108050007E1560937D15009371151093741586E35A
:1080600090E1A0E0B0E08093751590937615A09311
:108070007715B09378150E945666809122069091EC
:1080800023060E94E7C680912206909123069093D2
:108090007E1580937D15009371151093741584E3FC
:1080A00090E1A0E0B0E08093751590937615A093D1
:1080B0007715B09378150E94566665E070E080E011
:1080C00090E00E94D4DB8091D51B882309F181E0E8
:1080D0009AE590937E1580937D158AE190E09093C8
:1080E000801580937F1587E0809371151093741528
:1080F00084E890E0A0E0B0E0809375159093761549
:10810000A0937715B09378150E9456660C94C449D5
:1081100081E09AE590937E1580937D1584E490E04C
:108120009093801580937F1587E08093711510934D
:10813000741584E890E0A0E0B0E08093751590930A
:108140007615A0937715B09378150E9456660C9417
:10815000C4498630910509F04AC01092A905809162
:10816000D51B882311F181E09AE590937E158093C9
:108170007D1587E190E09093801580937F1587E0CF
:108180008093711582E88093741584E890E0A0E0F4
:10819000B0E08093751590937615A0937715B09302
:1081A00078150E9456660C94C44981E09AE5909334
:1081B0007E1580937D1581E490E0909380158093E7
:1081C0007F1587E08093711582E88093741584E8A9
:1081D00090E0A0E0B0E08093751590937615A093A1
:1081E0007715B09378150E9456660C94C449813F68
:1081F000910559F41092A9051092A80561E070E06C
:1082000080E090E00E94D4DBAACF803F910509F086
:1082100066CD0C94C4498435E0E19E07A105B10503
:10822000C1F460912D1570912E1580E090E00E94B0
:10823000B5EC20E030E040E251E40E9427F4609386
:108240009F057093A0058093A1059093A2050C94BF
:10825000C44988359041A105B10511F00C94C44979
:1082600060912D1570912E1580E090E00E94B5EC84
:1082700020E030E040E251E40E9427F46093A3053F
:108280007093A4058093A5059093A6050C94C4490A
:1082900060912D156093D51B8AE590E00E94D0F285
:1082A000909178128091D51B9923C1F18823D1F048
:1082B00010927E1510927D1585E08093711582E8ED
:1082C0008093741584E190E1A0E0B0E0809375158F
:1082D00090937615A0937715B09378150E94566603
:1082E0000C94C4498CE090E090937E1580937D15AA
:1082F00085E08093711582E88093741584E190E1A4
:10830000A0E0B0E08093751590937615A093771553
:10831000B09378150E9456660C94C4498823E1F006
:1083200086E090E090937E1580937D1585E08093A4
:10833000711582E88093741584E190E1A0E0B0E0CB
:108340008093751590937615A0937715B093781553
:108350000E9456660C94C44982E190E090937E1589
:1083600080937D1585E08093711582E88093741564
:1083700084E190E1A0E0B0E08093751590937615CC
:10838000A0937715B09378150E945666FDC780912B
:108390002D1590912E158130910509F0E9C180E0ED
:1083A00090E00E945AC8892B09F0EEC78091D61B35
:1083B000813009F0F1C082EB95E00E941D6786E2F2
:1083C00096E090931511809314110E94C5D7C12C8B
:1083D00030E2D32EE12CF12C05E012E810927E154C
:1083E00010927D150093711510937415C092751538
:1083F000D0927615E0927715F09278150E94566625
:108400002FEFC21AD20AE20AF20A3AE0C31630E2A9
:10841000D306E104F10411F78091B105A2E18A02CB
:10842000C0011124FC01EB56F84E7F0101900020A1
:10843000E9F7C7018E1B9F0B439697FD01968C01B0
:108440001595079510161106DCF49E012F5F3F4F1E
:10845000690184E1D9011D928A95E9F7A80162E9D1
:1084600073E0C9010E94C2F6B701C601800F911FD7
:108470000E94ADF640E050E260E070E0C60105C049
:1084800040E050E260E070E0C7010E940CC862E08A
:1084900070E080E090E00E94D4DB8091D51B8823BF
:1084A00049F181E090E090937E1580937D1585E001
:1084B0008093711512E81093741584E190E1A0E0A7
:1084C000B0E08093751590937615A0937715B093CF
:1084D00078150E94566662E070E080E090E00E94AD
:1084E000D4DB81E09AE590937E1580937D158AE038
:1084F00090E028C08DE090E090937E1580937D15EC
:1085000085E08093711512E81093741584E190E171
:10851000A0E0B0E08093751590937615A093771541
:10852000B09378150E94566662E070E080E090E0BB
:108530000E94D4DB81E09AE590937E1580937D15AF
:1085400084E390E09093801580937F1587E080937B
:1085500071151093741584E890E0A0E0B0E080936A
:10856000751590937615A0937715B09378150E94A2
:10857000566681E080933C028093351780933817CC
:1085800093E09093391780933F171092DC15109267
:10859000B1051092D61BF8C6823009F0E5C06E0115
:1085A000B3E3CB0ED11C80E1B82EF6012B2D119236
:1085B0002A95E9F76091EA057091EB058091EC0549
:1085C0009091ED05860122E043E00E94EEE77E01F6
:1085D0003FE1E30EF11CD7011D92BA94E9F76091D7
:1085E000E6057091E7058091E8059091E90587011E
:1085F00022E043E00E94EEE78091AE058F938091E8
:10860000AD058F938DE196E09F938F930E511109E5
:108610001F930F930E9483ECC8010E941D679EE187
:10862000B92EF8012B2D11922A95E9F78091E505D5
:108630008F938091E4058F9384E196E09F938F93CD
:108640001F930F930E9483ECC8010E941D67D801FD
:108650001D92BA94E9F7DF92CF928DE096E09F9356
:108660008F931F930F930E9483ECC8010E941D6794
:10867000FF92EF9285E096E09F938F931F930F9365
:108680000E9483ECC8010E941D671092AE051092F3
:10869000AD051092E5051092E4050FB6F894DEBF23
:1086A0000FBECDBF80917812882319F081E08093AE
:1086B00077120E94B8C88091D51B882319F081E0F9
:1086C00090E002C08DE090E090937E1580937D1540
:1086D00085E08093711582E88093741584E190E1C0
:1086E000A0E0B0E08093751590937615A093771570
:1086F000B09378150E9456661092DC1583E0809343
:10870000391781E080933F178091D51B882349F06A
:1087100081E09AE590937E1580937D158AE090E044
:1087200008C081E09AE590937E1580937D1584E3DF
:1087300090E09093801580937F1587E0809371156A
:1087400082E88093741584E890E0A0E0B0E0809324
:10875000751590937615A0937715B09378150E94B0
:1087600056661092D61B10C6833009F00DC6F7CCA2
:10877000892B09F009C68091D61B813081F5809143
:10878000D51B882349F081E09AE590937E1580936C
:108790007D1582E090E008C081E09AE590937E1517
:1087A00080937D158EE290E09093801580937F15E5
:1087B00087E08093711582E88093741584E890E0D7
:1087C000A0E0B0E08093751590937615A09377158F
:1087D000B09378150E9456661092381747C08230C1
:1087E000B1F48091D51B882349F081E09AE59093FC
:1087F0007E1580937D158CE090E020C081E09AE5A5
:1088000090937E1580937D1586E390E017C08330AA
:1088100069F58091D51B882349F081E09AE5909312
:108820007E1580937D1587E190E008C081E09AE590
:1088300090937E1580937D1581E490E09093801550
:1088400080937F1587E08093711582E8809374157B
:1088500084E890E0A0E0B0E08093751590937615E1
:10886000A0937715B09378150E9456661092D61B88
:108870008BC5E0902D15F0902E15F1E0EF16F10468
:1088800009F032C180913C1790913D1718161906D6
:108890000CF07AC58091DC0C8F938091DB0C8F9368
:1088A0008CEF95E09F938F938E010F5F1F4F1F9367
:1088B0000F930E9483ECC8010E941D678091DA0C1F
:1088C0008F938091D90C8F9383EF95E09F938F9333
:1088D0001F930F930E9483ECC8010E941D6789EECD
:1088E00095E090931511809314110E94C5D7F092D2
:1088F0009D05E0929C058FEF90E090933B1780934D
:108900003A1710923E021092DC1581E080933817DE
:1089100093E09093391780938F0580933C02809366
:10892000351780933F171092F91B1092F81B109285
:10893000C81A1092C71A0FB6F894DEBF0FBECDBF8B
:108940008091D51B882309F1F0927E15E0927D1568
:1089500085E08093711512E81093741584E190E11D
:10896000A0E0B0E08093751590937615A0937715ED
:10897000B09378150E94566681E09AE590937E1533
:1089800080937D158AE090E022C08DE090E0909386
:108990007E1580937D1585E08093711512E8109304
:1089A000741584E190E1A0E0B0E080937515909398
:1089B0007615A0937715B09378150E94566681E0DE
:1089C0009AE590937E1580937D1584E390E09093D3
:1089D000801580937F1587E080937115109374152F
:1089E00084E890E0A0E0B0E0809375159093761550
:1089F000A0937715B09378150E9456669091D51B79
:108A000080910D029923C1F18823D9F087E090E08D
:108A100090937E1580937D1585E08093711582E893
:108A20008093741588E190E1A0E0B0E08093751523
:108A300090937615A0937715B09378150E9456669B
:108A4000A3C488E090E090937E1580937D1585E027
:108A50008093711582E88093741588E190E1A0E01D
:108A6000B0E08093751590937615A0937715B09329
:108A700078150E94566688C48823D9F089E090E072
:108A800090937E1580937D1585E08093711582E823
:108A90008093741588E190E1A0E0B0E080937515B3
:108AA00090937615A0937715B09378150E9456662B
:108AB0006BC48AE090E090937E1580937D1585E0ED
:108AC0008093711582E88093741588E190E1A0E0AD
:108AD000B0E08093751590937615A0937715B093B9
:108AE00078150E94566650C432E0E316F10409F08E
:108AF0004BC481E080933C021092351780EA9FE0DE
:108B00009093F91B8093F81B8091D51B882349F023
:108B100081E09AE590937E1580937D1581E090E049
:108B200008C081E09AE590937E1580937D158DE2D3
:108B300090E09093801580937F1587E08093711566
:108B400082E88093741584E890E0A0E0B0E0809320
:108B5000751590937615A0937715B09378150E94AC
:108B600056660E94CAC780913417809333171092BB
:108B700032170E94278A0E943D660E94EDC610921D
:108B800068121092671210926D1210926E1210926B
:108B90006F12109270121092711210927212109243
:108BA0007312109274121092691210926A1210923B
:108BB0006B1210926C126AE588EF9EE00E94326A96
:108BC0001092C00C1092080F0E948F6A019669F4EF
:108BD0000CE913E0F80181918F01882319F00E94BC
:108BE00017D9F8CF8AE00E9417D981E694E10E9454
:108BF0008FB210923D1710923C1710923D021092C6
:108C0000381764EF71E080E090E00E94D4DBBCC3D1
:108C100080912D1590912E158F3F910531F028F000
:108C20008FEF90E0A0E0B0E002C0A0E0B0E0809361
:108C30000E0290930F02A0931002B0931102809144
:108C40000E0290910F02A0911002B09111020097B4
:108C5000A105B10519F510927E1510927D1505E05C
:108C60000093711512E8109374158AE890E1A0E062
:108C7000B0E08093751590937615A0937715B09317
:108C800078150E94566689E090E090937E15809357
:108C90007D15009371151093741522C00196A11DC6
:108CA000B11D05E0B695A795979587950A95D1F7DB
:108CB000BC01CD0161507109810991092AE830E1B7
:108CC00040E050E00E94FA6688E090E090937E15C4
:108CD00080937D1585E08093711582E880937415EB
:108CE0008CE890E1A0E0B0E0809375159093761544
:108CF000A0937715B09378150E94566660910E0286
:108D00008EE590E00E94D0F280910E0290910F02C9
:108D1000A0911002B09111026627782F892F9A2F07
:108D200021EA30E040E050E00E94FA662DC3209135
:108D30007812222309F457C1433DF0E25F07610531
:108D4000710509F050C180912D1590912E1520913B
:108D50004317309144172817390708F415C3815079
:108D600080934217A4ED8A2EA0E29A2EA12CB12C5A
:108D700005E012E810927E1510927D150093711592
:108D8000109374158092751590927615A0927715B0
:108D9000B09278150E9456662FEF821A920AA20AA4
:108DA000B20A3EED831630E29306A104B10411F736
:108DB00080914217A2E18A02C0011124FC01EB5606
:108DC000F84E7F0101900020E9F7C7018E1B9F0B31
:108DD000439697FD01968C0115950795101611067F
:108DE000FCF49E012F5F3F4F690184E1D9011D9280
:108DF0008A95E9F7A80162E973E0C9010E94C2F609
:108E0000B701C601800F911F0E94ADF644ED50E2FC
:108E100060E070E0C6010E940CC805E012E806C0E0
:108E200044ED50E260E070E0C701F5CF10927E158E
:108E300010927D150093711510937415809275151D
:108E400090927615A0927715B09278150E9456668A
:108E5000BFEF8B1A9B0AAB0ABB0AE6EE8E16E0E266
:108E60009E06A104B10411F78E010F5F1F4F84E12C
:108E7000D8011D928A95E9F7809144178F938091CC
:108E800043178F9380912E158F9380912D158F937B
:108E900081EC93E09F938F931F930F930E94D1F6E1
:108EA0004EED50E260E070E0C8010E940CC862E044
:108EB00070E080E090E00E94D4DB0FB6F894DEBF53
:108EC0000FBECDBF31E2C32E32E1D32EE12CF12C07
:108ED00043E1442E40E6542E612C712C8824839467
:108EE000912CAA24AA94BA2C75E0272EE2E83E2EF3
:108EF0000AE010E080914317909144178815990576
:108F000094F1B0927E15A0927D1520927115309249
:108F1000741540927515509276156092771570927F
:108F200078150E94566610937E1500937D15209249
:108F3000711530927415C0927515D0927615E09225
:108F40007715F09278150E945666FFEF8F1A9F0AE8
:108F500020E1420E511C611C711C3FEFC31AD30A61
:108F6000E30AF30AC7CF80912D1590912E1524E0C6
:108F7000880F991F2A95E1F78D5F9F49A0E0B0E027
:108F800020EF37E830937E1520937D1505E00093A0
:108F9000711512E8109374158093751590937615DA
:108FA000A0937715B09378150E94566680912D1581
:108FB00090912E15805E9D4EA0E0B0E026E030E05E
:108FC00030937E1520937D150093711510937415C1
:108FD0008093751590937615A0937715B0937815B7
:108FE0000E945666D1C1423D50426105710509F0AB
:108FF000CBC180912D1590912E158130910509F0EE
:10900000BFC1222309F4C0C18091421787FDBCC1B2
:10901000A2E18A02C00111248350974E9F938F933F
:1090200082EE95E09F938F938E010F5F1F4F1F93EA
:109030000F930E9483EC0F900F900F900F900F9062
:109040000F907E01B5E0EB0EF11CF70180818823C3
:1090500049F0082E000C990B0E945DF6D7018D9304
:109060007D01F3CF809142178093B10584E1E2EB5B
:10907000F5E0DF011D928A95E9F7B801CF010E9462
:10908000ADF681E090E00E945AC8892B09F07CC1BE
:10909000C8010E941D678EED95E090931511809395
:1090A00014110E94C5D7C12C90E2D92EE12CF12CCD
:1090B00005E012E810927E1510927D15009371154F
:1090C00010937415C0927515D0927615E0927715AD
:1090D000F09278150E945666BFEFCB1ADB0AEB0AB6
:1090E000FB0AEAE0CE16E0E2DE06E104F10411F745
:1090F00080914217F2E18F02C00111249C012B568E
:10910000384E7901F90101900020E9F7C9018E1B61
:109110009F0B439697FD01968C01159507951016A8
:109120001106DCF46E013FE1C30ED11C84E1D601CF
:109130001D928A95E9F7A80162E973E0C6010E94D1
:10914000C2F6B701C601800F911F0E94ADF640E044
:1091500050E260E070E0C60105C040E050E260E02F
:1091600070E0C7010E940CC862E070E080E090E00F
:109170000E94D4DB8FEF90E090933B1780933A17D7
:1091800010923E028091D51B882349F181E090E046
:1091900090937E1580937D1585E08093711512E87C
:1091A0001093741584E190E1A0E0B0E08093751510
:1091B00090937615A0937715B09378150E94566614
:1091C00062E070E080E090E00E94D4DB81E09AE50C
:1091D00090937E1580937D158AE090E028C08DE005
:1091E00090E090937E1580937D1585E080937115B6
:1091F00012E81093741584E190E1A0E0B0E0809350
:10920000751590937615A0937715B09378150E94F5
:10921000566662E070E080E090E00E94D4DB81E07E
:109220009AE590937E1580937D1584E390E090936A
:10923000801580937F1587E08093711510937415C6
:1092400084E890E0A0E0B0E08093751590937615E7
:10925000A0937715B09378150E94566681E08093AD
:109260003C0280933517809304021092DC15109213
:10927000D71B8093381793E09093391780933F174B
:1092800081E090E09093C81A8093C71A1092F91B5E
:109290001092F81B9091D51B80910D029923C1F17A
:1092A0008823D9F087E090E090937E1580937D1518
:1092B00085E08093711582E88093741588E190E1D0
:1092C000A0E0B0E08093751590937615A093771584
:1092D000B09378150E94566657C088E090E090934E
:1092E0007E1580937D1585E08093711582E88093CB
:1092F000741588E190E1A0E0B0E08093751590933B
:109300007615A0937715B09378150E9456663CC0E9
:109310008823D9F089E090E090937E1580937D15A5
:1093200085E08093711582E88093741588E190E15F
:10933000A0E0B0E08093751590937615A093771513
:10934000B09378150E9456661FC08AE090E0909313
:109350007E1580937D1585E08093711582E880935A
:10936000741588E190E1A0E0B0E0809375159093CA
:109370007615A0937715B09378150E94566604C0B1
:10938000892B11F40C94943480E5E1E2F5E1DF01DE
:109390001D928A95E9F78AE58093221585EA8093E4
:1093A00023152BC086E191E10E9457C1F401EF53D0
:1093B000FA4E80838091C1158A3581F01814190402
:1093C00014F00C94742BD501E72D1D92EA95E9F762
:1093D0001092B0051092AF050C94742B6AE070E007
:1093E00080E090E00E94D4DBFFEF8F1A9F0A9092FA
:1093F000B0058092AF050C94742BCE5BDF4F0FB697
:10940000F894DEBF0FBECDBFDF91CF911F910F91BA
:10941000FF90EF90DF90CF90BF90AF909F908F9094
:109420007F906F905F904F903F902F900895CF92D4
:10943000DF92EF92FF920F931F93CF93DF936C0114
:109440008B017A01EC01C756D34F888187FF04C096
:10945000FB011182108224C02CE02C9DC0012D9DA7
:10946000900D11242881AC01420F511D27FD5A9502
:109470002091451230E04217530794F42881AC0143
:10948000420F511D27FD5A959A01FA01EE0FFF1F59
:109490002E0F3F1FF901E752FE4E208126FD19C015
:1094A00088818F5F88832CE02C9DC0012D9D900DBD
:1094B00011242881AC01420F511D27FD5A9520919E
:1094C000451230E042175307BCF428812C3044F198
:1094D00013C02881820F911D27FD9A95FC01EE0F84
:1094E000FF1F8E0F9F1FFC01E752FE4E808160E040
:1094F0008F730E943D95D4CFF801808191810496AD
:1095000080349C4918F480E49CE904C0F80180810F
:1095100091810496F701918380838FEF888345C002
:10952000F801408151812881BC01620F711D27FD26
:109530007A959B01FB01EE0FFF1F2E0F3F1FF901D4
:10954000E752FE4E21813281240F351FF70131830E
:1095500020832881AC01420F511D27FD5A959A01A5
:10956000FA01EE0FFF1F2E0F3F1FF901E752FE4ECB
:10957000208126FF1AC02881820F911D27FD9A9510
:10958000FC01EE0FFF1F8E0F9F1FFC01E752FE4EE6
:10959000808161E08F73DF91CF911F910F91FF90D8
:1095A000EF90DF90CF900C943D95DF91CF911F917C
:1095B0000F91FF90EF90DF90CF9008958091960CDF
:1095C00080FF03C089988FEF02C0899A81E0809361
:1095D00014028091960C81FF03C08F988FEF02C018
:1095E0008F9A81E0809315028091960C9FB782FF3D
:1095F00009C0F89480910B018D7F80930B019FBF70
:109600008FEF08C0F89480910B01826080930B016A
:109610009FBF81E0809316028091960C83FF03C068
:1096200016988FEF02C0169A81E080931702089572
:109630009091D7118091D811981731F08091D8115D
:109640008F5F8F708093D81108951F920F920FB67D
:109650000F9211240BB60F92BF92CF92DF92EF922E
:10966000FF920F931F932F933F934F935F936F93AB
:109670007F938F939F93AF93BF93EF93FF93CF937A
:10968000DF9300D000D0CDB7DEB780916E008B7F26
:1096900080936E0080916F008D7F80936F0078942F
:1096A000C090BA0CD090BB0CE090BC0CF090BD0CFC
:1096B000C114D104E104F10409F442C08091F4051D
:1096C000811104C080910F068823D1F10E944C843F
:1096D000F9EBCF16FBE0DF06E104F10488F008EBBC
:1096E000C01A0BE0D00AE108F108C092BA0CD0927F
:1096F000BB0CE092BC0CF092BD0C88EB9BE009C067
:10970000C6011092BA0C1092BB0C1092BC0C1092B5
:10971000BD0C90938900809388002091880030913F
:109720008900809184009091850040962817390720
:1097300008F072C08091840090918500409622C00C
:109740000091970C1091980C1A830983012B09F44E
:1097500098C009811A81015011091093980C009347
:10976000970C1092DF1B1092DE1B62DF012B41F47D
:109770008DE990E190931511809314110E94C5D743
:1097800088EC90E0909389008093880045C089819F
:109790009A810E948E9224E630E08091F40588231D
:1097A00009F4D9C4C901293BBBE03B0708F012C644
:1097B00090938900809388008091AC0C9091AD0CBF
:1097C000A091AE0CB091AF0C820F931FA11DB11DE3
:1097D0008093AC0C9093AD0CA093AE0CB093AF0CF7
:1097E00020918800309189008091840090918500BB
:1097F00040962817390748F480918400909185009D
:1098000040969093890080938800BB2029F01092A5
:10981000DF1B1092DE1B0CDFF8948091B91B8823AC
:1098200021F080916E008B7F03C080916E00846078
:1098300080936E0080916F00826080936F00269607
:109840000FB6F894DEBF0FBECDBFDF91CF91FF9171
:10985000EF91BF91AF919F918F917F916F915F91A8
:109860004F913F912F911F910F91FF90EF90DF90BB
:10987000CF90BF900F900BBE0F900FBE0F901F9018
:109880001895E091DE1BF091DF1B309709F0BBC10A
:109890009091D7118091D811981751F1E091D8117A
:1098A0001DE4E19FF0011124EA53F84FC090C20774
:1098B000D090C307E090C407F090C507CF01875B45
:1098C0009F4FDC014D915D916D917C91D701C60157
:1098D000841B950BA60BB70B8093C2079093C3070D
:1098E000A093C407B093C5078081886080830BC0B4
:1098F0008FB7F8941092C2071092C3071092C40752
:109900001092C5078FBFF093DF1BE093DE1B3097EB
:1099100009F476C152A18091960C418158130AC076
:10992000242F30E080911802082E000C990B281784
:10993000390729F05093960C409318023FDE10929D
:10994000B60C1092B70C1092B80C1092B90CE091B2
:10995000DE1BF091DF1B87A990AD8134BCE99B072A
:1099600028F48132EEE49E0748F002C080E49CE9CE
:10997000969587959695879524E007C08131F7E203
:109980009F0730F09695879522E02093B50C08C08C
:1099900021E02093B50C8032910510F480E290E034
:1099A0008C01005211091A830983011528E012075E
:1099B000D8F0E12FFF27EE0FFF1FEE0FFF1FCF01A3
:1099C0008356934FFC01329645915491AA27059FE7
:1099D0009001049F210D3A1F06942A1F3A1F11245B
:1099E000FC01859194911FC089819A8196958795F4
:1099F0008C7F8356974FFC0145915491FC01329620
:109A00008591949169817A8167707727689F900129
:109A1000699F300D789F300D112483E0369527958E
:109A20008A95E1F7CA01821B930B8436910580F475
:109A30000EE014E0D8018D918D01882319F00E9469
:109A400017D9F8CF89819A810E948E9284E690E09E
:109A50009093B40C8093B30C8091B50C8093B20CAE
:109A6000E091DE1BF091DF1B83AD94AD9093B10CC0
:109A70008093B00C8134BCE99B0728F48132EEE47A
:109A80009E0748F002C080E49CE9969587959695DC
:109A9000879524E007C08131F7E29F0730F0969563
:109AA000879522E02093B50C08C021E02093B50CE7
:109AB0008032910510F480E290E08C01005211098F
:109AC0001A830983011528E01207D8F0E12FFF2738
:109AD000EE0FFF1FEE0FFF1FCF018356934FFC01C8
:109AE000329645915491AA27059F9001049F210D1C
:109AF0003A1F06942A1F3A1F1124FC018591949164
:109B00001FC089819A81969587958C7F8356974F40
:109B1000FC0145915491FC013296859194916981A3
:109B20007A8167707727689F9001699F300D789FD1
:109B3000300D112463E0369527956A95E1F7CA0147
:109B4000821B930B8436910580F40EE014E0D8015B
:109B50008D918D01882319F00E9417D9F8CF898142
:109B60009A810E948E9284E690E0AC0160E070E001
:109B70004093AC0C5093AD0C6093AE0C7093AF0C53
:109B80009093890080938800E091DE1BF091DF1BA9
:109B900082899389A489B589B695A7959795879564
:109BA000B095A095909581959F4FAF4FBF4F8093F3
:109BB000A80C9093A90CA093AA0CB093AB0C809323
:109BC000A40C9093A50CA093A60CB093A70C809323
:109BD000A00C9093A10CA093A20CB093A30C809323
:109BE0009C0C90939D0CA0939E0CB0939F0C109294
:109BF000DA1B1092DB1B1092DC1B1092DD1B03C0E2
:109C000080ED97E0BFCD8091F4058111E0C3809194
:109C10000F068111DCC32091B50C222309F4AFC1DA
:109C2000E091DE1BF091DF1B4281538164817581DD
:109C300080919C0C90919D0CA0919E0CB0919F0CDA
:109C4000840F951FA61FB71F80939C0C90939D0CAB
:109C5000A0939E0CB0939F0C181619061A061B06AB
:109C60000CF4889AE091DE1BF091DF1B468157814E
:109C7000608571858091A00C9091A10CA091A20C9F
:109C8000B091A30C840F951FA61FB71F8093A00C43
:109C90009093A10CA093A20CB093A30C18161906D4
:109CA0001A061B060CF48E9AE091DE1BF091DF1B66
:109CB00042855385648575858091A40C9091A50C8F
:109CC000A091A60CB091A70C840F951FA61FB71FDB
:109CD0008093A40C9093A50CA093A60CB093A70C12
:109CE000181619061A061B0644F49FB7F8948091BB
:109CF0000B01886080930B019FBFE091DE1BF09108
:109D0000DF1B46855785608971898091A80C9091E9
:109D1000A90CA091AA0CB091AB0C840F951FA61FA3
:109D2000B71F8093A80C9093A90CA093AA0CB09392
:109D3000AB0C181619061A061B060CF4149A80911F
:109D40009C0C90919D0CA0919E0CB0919F0C1816AC
:109D500019061A061B0684F5E091DE1BF091DF1B45
:109D60004289538964897589841B950BA60BB70BAF
:109D700080939C0C90939D0CA0939E0CB0939F0C91
:109D8000809114024091E01B5091E11B6091E21B15
:109D90007091E31B082E000C990BAA0BBB0B840FD0
:109DA000951FA61FB71F8093E01B9093E11BA09304
:109DB000E21BB093E31B88988091A00C9091A10CBA
:109DC000A091A20CB091A30C181619061A061B0636
:109DD00084F5E091DE1BF091DF1B42895389648991
:109DE0007589841B950BA60BB70B8093A00C9093E1
:109DF000A10CA093A20CB093A30C809115024091EA
:109E0000E41B5091E51B6091E61B7091E71B082E47
:109E1000000C990BAA0BBB0B840F951FA61FB71F35
:109E20008093E41B9093E51BA093E61BB093E71B84
:109E30008E988091A40C9091A50CA091A60CB09145
:109E4000A70C181619061A061B06BCF5E091DE1BB6
:109E5000F091DF1B4289538964897589841B950BB6
:109E6000A60BB70B8093A40C9093A50CA093A60C03
:109E7000B093A70C809116024091E81B5091E91B0A
:109E80006091EA1B7091EB1B082E000C990BAA0B3A
:109E9000BB0B840F951FA61FB71F8093E81B9093E1
:109EA000E91BA093EA1BB093EB1B9FB7F89480913A
:109EB0000B01877F80930B019FBF8091A80C90912D
:109EC000A90CA091AA0CB091AB0C181619061A0691
:109ED0001B0684F5E091DE1BF091DF1B428953895C
:109EE00064897589841B950BA60BB70B8093A80C0E
:109EF0009093A90CA093AA0CB093AB0C809117027D
:109F00004091EC1B5091ED1B6091EE1B7091EF1B8B
:109F1000082E000C990BAA0BBB0B840F951FA61FD4
:109F2000B71F8093EC1B9093ED1BA093EE1BB09397
:109F3000EF1B14988091DA1B9091DB1BA091DC1B26
:109F4000B091DD1B0196A11DB11D8093DA1B90938A
:109F5000DB1BA093DC1BB093DD1B2150E091DE1BCB
:109F6000F091DF1B428953896489758984179507AD
:109F7000A607B70708F451CEBB24B39401C0B12C97
:109F8000E091DE1BF091DF1B8091DA1B9091DB1BCF
:109F9000A091DC1BB091DD1B46895789608D718DC6
:109FA000481759076A077B0708F4DBC04091AC0CDF
:109FB0005091AD0C6091AE0C7091AF0C068D178D69
:109FC00020A131A1AA27419FB12D529FC001629FBC
:109FD000900D619F800D911D429FB00D811D9A1FB4
:109FE000519FB00D811D9A1F609FB00D811D9A1F5A
:109FF000509FB10D8A1F9A1FB6958A1F9A1F349FD2
:10A00000800D911D359F900D112423AD34AD820F2D
:10A01000931F9093B10C8093B00C47A950AD61ADE4
:10A0200072ADA0E0B0E0481759076A077B0720F43B
:10A030005093B10C4093B00CE091B00CF091B10C86
:10A04000FA83E983E1340CE9F00720F4E132FE44BD
:10A0500078F004C020E43CE93A83298389819A811D
:10A0600096958795969587959A83898384E00BC00A
:10A07000A981BA81A131E7E2BE0740F0B695A79564
:10A08000BA83A98382E08093B50C0CC081E08093F1
:10A09000B50C09811A810032110520F420E230E06C
:10A0A0003A83298309811A81005211091A8309838D
:10A0B000011528E01207E8F0E12FFF27EE0FFF1F40
:10A0C000EE0FFF1FCF018356934FFC01329625916F
:10A0D0003491AA27039FA001029F410D5A1F0694A5
:10A0E0004A1F5A1F1124FC0125913491241B350B62
:10A0F00021C029813A81369527952C7F2356374FE9
:10A10000F90145915491F901329625913491698173
:10A110007A8167707727629FC001639F900D729F5D
:10A12000900D1124F3E096958795FA95E1F79A0141
:10A13000281B390B2436310508F02FCB7EE0E72EA3
:10A1400074E0F72ED7018D917D01882309F41FCB90
:10A150000E9417D9F7CF80910F06811123CBC90137
:10A1600027CB8091DA1B9091DB1BA091DC1BB09177
:10A17000DD1B428D538D648D758D481759076A0715
:10A180007B0708F0F1C00091B60C1091B70C20913C
:10A19000B80C3091B90C09831A832B833C83468D0C
:10A1A000578D60A171A1AA27059FB12D169F70013F
:10A1B000269FF00C259FE00CF11C069FB00DE11CC2
:10A1C000FA1E159FB00DE11CFA1E249FB00DE11C74
:10A1D000FA1E149FB10DEA1EFA1EB695EA1EFA1E6B
:10A1E000709FE00CF11C719FF00C11248091B00C59
:10A1F0009091B10CFF96E816F90680F48E199F092C
:10A2000040815181628173816C01E12CF12CC41673
:10A21000D506E606F70620F4CA0102C080819181C6
:10A2200081341CE9910728F481322EE4920748F02A
:10A2300002C080E49CE9969587959695879524E0E1
:10A2400007C0813137E2930730F09695879522E079
:10A250002093B50C08C021E02093B50C8032910505
:10A2600010F480E290E08C01005211091E830D83EE
:10A27000011528E01207E8F0E12FFF27EE0FFF1F7E
:10A28000EE0FFF1FCF018356934FFC0132962591AD
:10A290003491AA27039FA001029F410D5A1F0694E3
:10A2A0004A1F5A1F1124FC0125913491241B350BA0
:10A2B00021C02D813E81369527952C7F2356374F1F
:10A2C000F90145915491F9013296259134916D81AE
:10A2D0007E8167707727629FC001639F900D729F98
:10A2E000900D112423E0969587952A95E1F79A0120
:10A2F000281B390B2436310590F48EE0E82E84E0DB
:10A30000F82ED7018D917D01882319F00E9417D96D
:10A31000F8CF8D819E810E948E9224E630E080915C
:10A32000F405811104C080910F06882339F0C9011A
:10A33000293BBBE03B0708F068C001C0C90190930E
:10A3400089008093880089819A81AB81BC81820FCA
:10A35000931FA11DB11D8093B60C9093B70CA093D1
:10A36000B80CB093B90C3CCA2091B30C3091B40C2A
:10A370008091F405811104C080910F068823F1F0CB
:10A38000293BEBE03E07D0F0C90168EB7BE00E947F
:10A3900024F6883E63E0960708F052C08854944F34
:10A3A000A901481B590B60E070E04093BA0C509330
:10A3B000BB0C6093BC0C7093BD0C9C013093890066
:10A3C000209388008091B20C8093B50C09CA0E943A
:10A3D0004C8421CC68EB7BE00E9424F6883E13E09D
:10A3E000910780F48854944FA901481B590B60E0F1
:10A3F00070E04093BA0C5093BB0C6093BC0C70930C
:10A40000BD0CD6C988EB9BE0EFCF68EB7BE00E94E8
:10A4100024F6883E43E0940780F48854944FA901C1
:10A42000481B590B60E070E04093BA0C5093BB0C92
:10A430006093BC0C7093BD0C82CF88EB9BE0EFCF98
:10A4400088EB9BE0ADCF8F929F92AF92BF92CF925D
:10A45000DF92EF92FF920F931F93CF93DF938C01C4
:10A46000EB0160E070E00E949A9287FD8CC0C032E0
:10A4700082E0D8070CF042C0F801828128E532E082
:10A48000281B310987FD3395220F331F220F331FFD
:10A490004901330FAA08BB08818128E830E069012F
:10A4A000C81AD10887FDD394CC0CDD1CCC0CDD1C64
:10A4B0000D2C000CEE08FF08D7FD0AC0C53BD105E6
:10A4C00014F0C4EBD0E0BE01DD0F880B990B03C084
:10A4D00060E070E0CB01A50194012C193D094E0903
:10A4E0005F090E94DEF224EB30E040E050E00E9481
:10A4F0000FF3C20ED31EE41EF51EE601F801208103
:10A50000243278F5318188E890E0831B910937FD8A
:10A510009395880F991F880F991FC817D90784F042
:10A52000F801328188E592E0831B910937FD93950C
:10A53000880F991F880F991FC817D9070CF4CE01EF
:10A5400002974FB7F89430E0F901EE0FFF1F2E0F7E
:10A550003F1FF901E752FE4E880F991F92838183B6
:10A560004FBF62E370E080E090E0DF91CF911F91F8
:10A570000F91FF90EF90DF90CF90BF90AF909F90A2
:10A580008F900C94D4DBDF91CF911F910F91FF90AE
:10A59000EF90DF90CF90BF90AF909F908F900895F5
:10A5A0001F920F920FB60F9211240BB60F922F939A
:10A5B0003F934F935F936F937F938F939F93AF934B
:10A5C000BF93EF93FF9348E251E064E271E082E0D1
:10A5D00090E00E94174AFF91EF91BF91AF919F9138
:10A5E0008F917F916F915F914F913F912F910F903C
:10A5F0000BBE0F900FBE0F901F9018951F920F92D9
:10A600000FB60F9211240BB60F922F933F934F93D7
:10A610005F936F937F938F939F93AF93BF93EF93CA
:10A62000FF9348EA50E064EA70E081E090E00E9425
:10A63000174AFF91EF91BF91AF919F918F917F91B9
:10A640006F915F914F913F912F910F900BBE0F90A3
:10A650000FBE0F901F9018951F920F920FB60F927A
:10A6600011240BB60F922F933F934F935F936F93E9
:10A670007F938F939F93AF93BF93EF93FF9348E99B
:10A6800050E064E970E080E090E00E94174AFF919A
:10A69000EF91BF91AF919F918F917F916F915F915A
:10A6A0004F913F912F910F900BBE0F900FBE0F90C7
:10A6B0001F901895CF92DF92EF92FF92CF93DF9386
:10A6C0006A017B01FC018491EF012196882321F02E
:10A6D0000E9417D9FE01F7CF4AE0C701B601DF910A
:10A6E000CF91FF90EF90DF90CF900C941ED9CF9236
:10A6F000DF92EF92FF92CF93DF936A017B01FC011F
:10A700008491EF012196882321F00E9417D9FE0140
:10A71000F7CF42E0C701B601DF91CF91FF90EF90F4
:10A72000DF90CF900C94A3D90F931F93CF93DF9317
:10A730008B01FC018491EF012196882321F00E9476
:10A7400017D9FE01F7CFB801110F880B990BDF91D4
:10A75000CF911F910F910C9489D90F931F93CF9391
:10A76000DF938B01FC018491EF012196882321F076
:10A770000E9417D9FE01F7CFE8018991882319F0CB
:10A780000E9417D9FACFDF91CF911F910F910895B1
:10A790004F925F926F927F92AF92BF92CF92DF9271
:10A7A000EF92FF920F931F93CF93DF938C01EB01F6
:10A7B000FC0147A050A461A472A4AFA0B8A4C9A48E
:10A7C000DAA49501A601C301B2010E94B1EC87FF92
:10A7D00040C0A3019201C301B2010E9416ED2B01FA
:10A7E0003C01F80183A994A9A5A9B6A9BC01CD0192
:10A7F00090589B01AC010E944BF3F80127A530A9AA
:10A8000041A952A90E9416ED9B01AC01C301B201FE
:10A810000E944AF30E94B7F57B018C019B01AC01B9
:10A82000B501C6010E94B1EC87FF02C07501860127
:10A830009701A801B501C6010E94B1EC882349F037
:10A84000C701D8018FA398A7A9A7BAA7888181605B
:10A850008883DF91CF911F910F91FF90EF90DF9050
:10A86000CF90BF90AF907F906F905F904F90089582
:10A870008091C10781111AC0609112027091130278
:10A88000072E000C880B990B0E94B7EC9B01AC01C2
:10A890006091FC057091FD058091FE059091FF058A
:10A8A0000E94B1EC881F8827881F089580E00895D2
:10A8B0000F931F93CF93DF938C01EEEEF0E1849121
:10A8C000EF012196882321F00E9417D9FE01F7CFCE
:10A8D000F8018491EF012196882321F00E9417D975
:10A8E000FE01F7CFE5EDF0E18491EF012196882399
:10A8F00021F00E9417D9FE01F7CFDF91CF911F9170
:10A900000F910895CF92DF92EF92FF920F931F93D2
:10A91000CF93DF9385E6E82E82E0F82E03E91AE173
:10A92000C2EDD6E194E9C92E95E0D92EF7018191C7
:10A930007F010E94CCD88823E1F00E9495D89B012A
:10A94000AC01F6018081811104C0809198058823B3
:10A9500029F0688179818A819B8103C060E070E081
:10A96000CB010E944BF3F801608371838283938350
:10A9700009C088819981AA81BB81F8018083918374
:10A98000A283B3830C5F1F4F2496FFEFCF1ADF0A19
:10A9900089E6E81682E0F80649F686E40E94FBD8CC
:10A9A0008823C9F00E9495D820E030E0A9010E94D8
:10A9B00071F5181684F40E9495D820E030E040E745
:10A9C00052E40E9427F4609334027093350280931E
:10A9D000360290933702DF91CF911F910F91FF9034
:10A9E000EF90DF90CF9008954F925F926F927F9299
:10A9F0008F929F92AF92BF92CF92DF92EF92FF928F
:10AA00000F931F93CF93DF93CDB7DEB72C970FB67D
:10AA1000F894DEBF0FBECDBF7C012A013B01B22EF0
:10AA2000A32E82E0E816F10449F420E030E0A90109
:10AA3000C301B2010E94B1EC87FD90C0D12CEE0C95
:10AA4000FF1CEE0CFF1CF701EE52F94E4F01108275
:10AA50001182128213820E941ED8F4014082518218
:10AA600062827382C090930520E030E0A901B801B2
:10AA70008B2D9A2D0E94B1EC81110CC0F701E95584
:10AA8000F24E85919591A591B491982E892EBA2E6A
:10AA9000AB2E02C0902E812E8091DA169091DB169B
:10AAA000A091DC16B091DD164091D6165091D716C4
:10AAB0006091D8167091D9160091D2161091D316C4
:10AAC0002091D4163091D51609831A832B833C83A9
:10AAD0004D835E836F83788789879A87AB87BC872E
:10AAE00080910E0681110AC0AE01475F5F4FBE0123
:10AAF0006B5F7F4FCE0101960E943681E92CF82CC6
:10AB00000B2D1A2D2EED36E1AE01475F5F4FBE01D2
:10AB10006B5F7F4FCE0101960E941D740E943AD751
:10AB2000DD2019F080E00E94B86B109240062C9650
:10AB30000FB6F894DEBF0FBECDBFDF91CF911F914E
:10AB40000F91FF90EF90DF90CF90BF90AF909F90CC
:10AB50008F907F906F905F904F90089581E00E945A
:10AB6000B86BDD24D3946BCFCF92DF92EF92FF923C
:10AB70006091731A7091741A072E000C880B990B50
:10AB80000E94B7EC6B017C012DEB37E346E855EBF7
:10AB90000E9471F587FD0AC02DEB37E346E855E3C7
:10ABA000C701B6010E94B1EC18164CF4A70196013A
:10ABB00060E070E080E89FE30E9427F403C060E05B
:10ABC00070E0CB0160934F1B7093501B8093511B1F
:10ABD0009093521B6091751A7091761A072E000C93
:10ABE000880B990B0E94B7EC6B017C012DEB37E3CE
:10ABF00046E855EB0E9471F587FD0AC02DEB37E35F
:10AC000046E855E3C701B6010E94B1EC18164CF4B2
:10AC1000A701960160E070E080E89FE30E9427F4BE
:10AC200003C060E070E0CB016093531B7093541B32
:10AC30008093551B9093561BFF90EF90DF90CF9021
:10AC400008958F929F92AF92BF92CF92DF92EF9230
:10AC5000FF920F931F93CF93DF93ECEBF0E184917E
:10AC6000EF012196882321F00E9417D9FE01F7CF2A
:10AC7000C12CD12C7601C0E080E20E9417D9CF5FB1
:10AC8000C730D1F7C701B6010E9489D98FEFC81A22
:10AC9000D80AE80AF80A94E0C916D104E104F104DC
:10ACA00051F78AE00E9417D90EEE16E1C12CD12C83
:10ACB000760180E20E9417D9C701B6010E9489D9A6
:10ACC000C0E0D0E080E20E9417D9F801EC0FFD1F30
:10ACD00080809180A280B380A5019401C501B40158
:10ACE0000E94F9F5811112C020E030E0A901C501F0
:10ACF000B4010E9471F587FD03C08BE20E9417D951
:10AD000044E0C501B4010E94A3D909C0B12C80E27E
:10AD10000E9417D9B3948DE397E0B912F9CF6096EA
:10AD2000C034D10579F68AE00E9417D98FEFC81A8E
:10AD3000D80AE80AF80A0C5F1F4F94E0C916D1043C
:10AD4000E104F10409F0B5CF8AE00E9417D989EA3D
:10AD500090E19093151180931411DF91CF911F9181
:10AD60000F91FF90EF90DF90CF90BF90AF909F90AA
:10AD70008F900C94C5D780E00E94716B1092761A68
:10AD80001092751A1092741A1092731A1092721A05
:10AD90001092711A1092701A10926F1AEEEEF6E17C
:10ADA0002EE237E180E090E0A0ECBFE78083918362
:10ADB000A283B38384839583A683B7838087918797
:10ADC000A287B38784879587A687B78770962E1743
:10ADD0003F0761F708952F923F924F925F926F92D3
:10ADE0007F928F929F92AF92BF92CF92DF92EF921B
:10ADF000FF920F931F93CF93DF93CDB7DEB7E59705
:10AE00000FB6F894DEBF0FBECDBF80910E0688232B
:10AE100029F080913817813009F424C680913717C2
:10AE2000813021F482E08093371703C0823009F427
:10AE300019C6B090901A81E0B8260091911A08279F
:10AE40001091921A1827B11004C0011102C009F420
:10AE500056C0E2EBF2E184917F012FEFE21AF20A91
:10AE6000811103C0E4E0F1E104C00E9417D9F701A9
:10AE7000F2CF84917F013FEFE31AF30A882321F098
:10AE80000E9417D9F701F5CFBB2069F0E2E0F1E1AC
:10AE900084917F019FEFE91AF90A882321F00E942B
:10AEA00017D9F701F5CF002369F0E0E0F1E18491D3
:10AEB0007F01AFEFEA1AFA0A882321F00E9417D91E
:10AEC000F701F5CF112319F0EEEFF0E103C0E6EF43
:10AED000F0E10AC084918F010F5F1F4F8823B9F3FF
:10AEE0000E9417D9F801F6CF84918F010F5F1F4F91
:10AEF000882309F4B7C50E9417D9F801F5CF30901F
:10AF0000541687E50E94CCD8882309F429C1809182
:10AF1000731A9091741A892BD1F4ECE7F2E18491C1
:10AF20008F010F5F1F4F811103C0EDE8F1E104C0F5
:10AF30000E9417D9F801F3CF84918F010F5F1F4F43
:10AF4000882309F48FC50E9417D9F801F5CFC09066
:10AF5000DA16D090DB16E090DC16F090DD168090CB
:10AF6000EA169090EB16A090EC16B090ED168AE5DC
:10AF70000E94FBD8811107C0A5019401C701B60149
:10AF80000E944AF302C00E9495D86B017C0120E028
:10AF900030E040E251EC0E9471F587FD0AC020E0EC
:10AFA00030E040E251E4C701B6010E94B1EC18164E
:10AFB000D4F4ECE7F2E184918F010F5F1F4F811110
:10AFC00003C0E0E8F1E104C00E9417D9F801F3CF13
:10AFD00084918F010F5F1F4F882309F443C50E949E
:10AFE00017D9F801F5CF88E50E94FBD8882329F00E
:10AFF0000E9495D82B013C0106C0412C512C60ECDD
:10B00000662E6FE7762E89E50E94FBD8882329F00B
:10B010000E9495D84B015C0106C0812C912C50EC0C
:10B02000A52E5FE7B52E89E40E94FBD8882319F08E
:10B030000E9475D801C08FEF082F8AE40E94FBD8C8
:10B04000882319F00E9475D801C08FEF182FA30133
:10B050009201C301B2010E94F9F5811162C0A501FC
:10B060009401C501B4010E94F9F581115AC06091A3
:10B070006F1A7091701A072E000C880B990B0E94A2
:10B08000B7EC2091E2163091E3164091E41650910E
:10B09000E5160E944BF39B01AC01C301B2010E9473
:10B0A0004AF320E030E0A9010E944BF320E030E0B9
:10B0B000A9010E9427F40E948FF4062F6091711A53
:10B0C0007091721A072E000C880B990B0E94B7EC36
:10B0D0002091E6163091E7164091E8165091E91656
:10B0E0000E944BF39B01AC01C501B4010E944AF3DD
:10B0F00020E030E0A9010E944BF320E030E0A901FC
:10B100000E9427F40E948FF4E02F04300CF0E3E05B
:10B110000E2FE7FD00E0162F64300CF013E017FD52
:10B1200010E0043008F09EC4153008F09BC480E0A5
:10B130000E94716BB4E00B02F0011124E10FF11DCC
:10B1400017FDFA95EE0FFF1FEE0FFF1FE251F94EAC
:10B15000C082D182E282F382832D0E94716B82C40D
:10B160008AE40E94CCD8882311F005DE7BC486E5F2
:10B170000E94FBD8882329F00E9465D879A768A788
:10B1800002C019A618A6E8A5F9A5359768F0E8E564
:10B19000F1E184918F010F5F1F4F882309F462C48E
:10B1A0000E9417D9F801F5CF84E40E94CCD8282E4C
:10B1B000882319F00E9486D8282E8AE50E94FBD8A1
:10B1C000882339F00E9495D86EA77FA788AB99ABEA
:10B1D00004C01EA61FA618AA19AA83E50E94FBD8C0
:10B1E000882319F00E9495D804C060E070E08AEFCF
:10B1F00095E420E030E040E752E40E9427F46093B9
:10B200002F0270933002809331029093320220E03B
:10B2100030E048E452E46091E2167091E3168091C8
:10B22000E4169091E5160E944BF34B015C018CE40F
:10B230000E94FBD8882321F00E9495D84B015C0125
:10B24000C501B4010E948FF469877A878B879C8738
:10B2500009851A8520E030E046E953E46091E21662
:10B260007091E3168091E4169091E5160E944BF3DD
:10B270004B015C0182E50E94FBD8882321F00E94EB
:10B2800095D84B015C01C501B4010E948FF46D8714
:10B290007E878F87988B2D853E853E8F2D8F20E072
:10B2A00030E048E452E46091E6167091E716809130
:10B2B000E8169091E9160E944BF34B015C0186E47D
:10B2C0000E94FBD8882321F00E9495D84B015C0195
:10B2D000C501B4010E948FF4698B7A8B8B8B9C8B98
:10B2E00089899A899BA38AA320E030E046E953E448
:10B2F0006091E6167091E7168091E8169091E91634
:10B300000E944BF34B015C0182E40E94FBD888232E
:10B3100021F00E9495D84B015C01C501B4010E9447
:10B320008FF46D8B7E8B8F8B988FAD89BE89BBA779
:10B33000AAA7E985FA85BF01FF0F880B990B0E9428
:10B34000B7EC6CA37DA38EA39FA38090E216909090
:10B35000E316A090E416B090E51620E030E0A901D5
:10B36000C501B4010E944BF39B01AC016CA17DA10E
:10B370008EA19FA10E94B1EC87FD0AC0F1E0F9A364
:10B380008D859E8509970817190724F419A202C014
:10B3900021E029A3AD85BE85BD01BB0F880B990BAC
:10B3A0000E94B7EC2B013C0120E030E044EB53E479
:10B3B000C501B4010E944BF39B01AC01C301B20172
:10B3C0000E9471F501E018164CF089859A8509965E
:10B3D000ED8DFE8D8E179F070CF400E029893A89C8
:10B3E000B901330F880B990B0E94B7EC6D8F7E8FDC
:10B3F0008F8F98A38090E6169090E716A090E8169D
:10B40000B090E91620E030E0A901C501B4010E9426
:10B410004BF39B01AC016D8D7E8D8F8D98A10E94A9
:10B42000B1EC11E087FD09C08D899E890997AAA119
:10B43000BBA1A817B9070CF410E0ED89FE89BF0184
:10B44000FF0F880B990B0E94B7EC2B013C0120E009
:10B4500030E044EB53E4C501B4010E944BF39B017F
:10B46000AC01C301B2010E9471F5BB24B39418165C
:10B470004CF089899A8909962AA53BA582179307DA
:10B480000CF4B12C39A131110BC0002321F089E457
:10B4900091E10EDA0AC011110AC0B1100EC011C03C
:10B4A00081E591E105DA0111F2CF112319F081E470
:10B4B00091E1FED9BB2009F4D5C28AE391E1F8D924
:10B4C000D1C288A599A5892BD1F0E3E2F1E184915D
:10B4D0008F010F5F1F4F882321F00E9417D9F801B9
:10B4E000F6CF222061F0EAE0F1E184918F010F5F55
:10B4F0001F4F882321F00E9417D9F801F6CF0E9430
:10B500003AD710925416211006C084E690E00E94AB
:10B5100088AF0E941ED881E00E949B6D882319F09D
:10B52000309254169FC28D859E85A985BA858A1B47
:10B530009B0B03E010E0B8010E9438F65B01072E78
:10B54000000C880B990B0E94B7EC6AA77BA78CA70D
:10B550009DA78D899E89E989FA898E1B9F0BB80169
:10B560000E9438F68B01072E000C880B990B0E9465
:10B57000B7EC2B013C010E94336C6091731A7091FF
:10B58000741A072E000C880B990B0E94B7EC9B01D4
:10B59000AC016AA57BA58CA59DA50E94B1EC81118B
:10B5A0004EC06091751A7091761A072E000C880BA8
:10B5B000990B0E94B7EC9B01AC01C301B2010E9440
:10B5C000B1EC81113CC060916F1A7091701A072E16
:10B5D000000C880B990B0E94B7EC2091E216309179
:10B5E000E3164091E4165091E5160E944BF39B013F
:10B5F000AC016CA17DA18EA19FA10E94B1EC811133
:10B600001EC06091711A7091721A072E000C880B7F
:10B61000990B0E94B7EC2091E6163091E716409105
:10B62000E8165091E9160E944BF39B01AC016D8D19
:10B630007E8D8F8D98A10E94B1EC8823A9F12110F5
:10B640003092541698DBB092741AA092731A109329
:10B65000761A0093751A2091E2163091E316409104
:10B66000E4165091E5166CA17DA18EA19FA10E94C8
:10B670004AF30E948FF47093701A60936F1A2091AE
:10B68000E6163091E7164091E8165091E9166D8D57
:10B690007E8D8F8D98A10E944AF30E948FF4709343
:10B6A000721A6093711A312C85E40E94CCD8898B70
:10B6B000882319F00E9486D8898B812C912C1D86B5
:10B6C000F1E0FD8BA7019601C701B6010E94F9F5D3
:10B6D000811121C0AD89AA2309F4A2C121E02AA3C6
:10B6E00034E039A3198681E09D8998279D8BC40198
:10B6F000092C000CAA0BBB0B8AAB9BABACABBDAB54
:10B7000099A1A9859A13B3C08FEF881A980A94E07B
:10B7100089169104B9F680E00E949B6D882319F088
:10B720003092541687C0A7019601C701B6010E9446
:10B73000F9F581117FC0222039F083DA8091D91B7D
:10B74000833009F055C025C011E083E0F82E01E0F8
:10B75000EF2CE11ADF2CD01A21E041E0602F812F7D
:10B760000E9412E521E04FEF602F8E2D0E9412E51E
:10B770002FEF41E06D2D812F0E9412E52FEF4FEF4B
:10B780006D2D8E2D0E9412E5015020F71150F8F614
:10B79000D4CF1092D91B8091D51B882349F081E02A
:10B7A0009AE590937E1580937D1586E190E008C020
:10B7B00081E09AE590937E1580937D1580E490E07A
:10B7C0009093801580937F1587E08093711582E8B0
:10B7D0008093741584E890E0A0E0B0E08093751544
:10B7E00090937615A0937715B09378150E945666BE
:10B7F0000E94869FB9D921101AC082ED96E10E945D
:10B80000D4AF9B01AC016091DA167091DB16809188
:10B81000DC169091DD160E944AF36093DA1670935D
:10B82000DB168093DC169093DD1681E001C0832D3A
:10B83000809354168091C71A9091C81A892B31F0C1
:10B840000E949E6A7093C81A6093C71A0E94196C6E
:10B850009FD181E090E09093581B8093571B80917B
:10B860005416882309F4FEC00E941ED8FBC06A2F1C
:10B87000AA0F770B880B990B0E94B7EC2AA53BA562
:10B880004CA55DA50E9416ED2CA13DA14EA15FA186
:10B890000E944BF3698F7A8F8B8F9C8F6AA97BA94B
:10B8A0008CA99DA90E94B7ECA30192010E9416EDFC
:10B8B0002D8D3E8D4F8D58A10E944BF36B017C0165
:10B8C00020E030E0A901698D7A8D8B8D9C8D0E94DE
:10B8D000B1EC87FF04C060E070E0CB0104C060E021
:10B8E00070E080E09FE3298D3A8D4B8D5C8D0E9446
:10B8F0004BF30E94C0F469837A838B839C8320E09E
:10B9000030E0A901C701B6010E94B1EC87FF04C075
:10B9100060E070E0CB0104C060E070E080E09FE395
:10B92000A70196010E944BF30E94C0F46D837E83B1
:10B930008F83988728A54989BE016B5F7F4FCE0111
:10B9400001960E941E936B017C019B01AC010E9439
:10B95000F9F5882319F030925416D6CEB985E4E073
:10B96000BE02500111248501080D191D000F111F81
:10B97000000F111F0251194E2EA53FA548A959A924
:10B98000C701B6010E944BF3D8016D937D938D934F
:10B990009C9313971D851F5FBD85B03128F480915E
:10B9A000D91B833009F443C0F501E80DF91DEE0FF2
:10B9B000FF1FEE0FFF1FE251F94E20E030E44CE193
:10B9C00056E460817181828193810E9416ED0E940C
:10B9D0008FF470937E1560937D15E5E0E09371150B
:10B9E000F2E8F0937415812F90E08158974F880FFB
:10B9F000991F092E000CAA0BBB0B80937515909311
:10BA00007615A0937715B09378150E9456660E941C
:10BA1000A8AB2AA13985230F2987312C1D8770CE29
:10BA2000BFEFBAA3EFEFE9A3F3E0F9875CCE812F74
:10BA300090E090937E1580937D1525E020937115FD
:10BA400032E8309374158DE890E1A0E0B0E0809387
:10BA5000751590937615A0937715B09378150E947D
:10BA60005666A2CFE5960FB6F894DEBF0FBECDBFE7
:10BA7000DF91CF911F910F91FF90EF90DF90CF90CA
:10BA8000BF90AF909F908F907F906F905F904F90FE
:10BA90003F902F900895CF92DF92EF92FF92CF9335
:10BAA0006B017C01C091541660935016709351162F
:10BAB00080935216909353162DEB37E346E855EBDF
:10BAC0000E9471F587FD0AC02DEB37E346E855E388
:10BAD000C701B6010E94B1EC18164CF4A7019601FB
:10BAE00060E070E080E89FE30E9427F403C060E01C
:10BAF00070E0CB0160934C1670934D1680934E16F8
:10BB000090934F16CC2349F082E090E0CF91FF90C4
:10BB1000EF90DF90CF900C9488AFCF91FF90EF9093
:10BB2000DF90CF900895DF92EF92FF920F931F93D3
:10BB3000CF93DF937C018B01D42EC2E2D4E08991B4
:10BB4000882319F00E9417D9FACF8FEFD81611F079
:10BB500084E501C082E40E9417D98AE30E9417D9C4
:10BB6000F701608171818281938142E00E94A3D9B3
:10BB7000F801408151816281738189ED91E1DF910A
:10BB8000CF911F910F91FF90EF90DF900C9477531E
:10BB90004F925F926F927F928F929F92AF92BF92DD
:10BBA000CF92DF92EF92FF92CF93DF93EFE1F2E13A
:10BBB0008491EF012196882321F00E9417D9FE017C
:10BBC000F7CF6091D2167091D3168091D4169091D0
:10BBD000D51642E00E94A3D9EBE1F2E18491EF0196
:10BBE0002196882321F00E9417D9FE01F7CF60919A
:10BBF000D6167091D7168091D8169091D91642E03A
:10BC00000E94A3D9E7E1F2E18491EF012196882314
:10BC100021F00E9417D9FE01F7CF6091DA167091DA
:10BC2000DB168091DC169091DD1642E00E94A3D9CC
:10BC3000E3E1F2E18491EF012196882321F00E9453
:10BC400017D9FE01F7CF6091DE167091DF16809153
:10BC5000E0169091E11642E00E94A3D98FB7F894C4
:10BC60004090E01B5090E11B6090E21B7090E31B42
:10BC70008090E41B9090E51BA090E61BB090E71B22
:10BC8000C090E81BD090E91BE090EA1BF090EB1B02
:10BC90008FBFE9E0F2E18491EF012196882321F042
:10BCA0000E9417D9FE01F7CFC301B2010E9489D9C2
:10BCB000E5E0F2E18491EF012196882321F00E94D2
:10BCC00017D9FE01F7CFC501B4010E9489D9E1E07F
:10BCD000F2E18491EF012196882321F00E9417D987
:10BCE000FE01F7CFC701B6010E9489D98AE0DF9132
:10BCF000CF91FF90EF90DF90CF90BF90AF909F904B
:10BD00008F907F906F905F904F900C9417D90F9306
:10BD10001F93CF93DF93CDB7DEB728970FB6F89474
:10BD2000DEBF0FBECDBF6091220670912306072EA5
:10BD3000000C880B990B0E94B7EC6D837E838F8378
:10BD400098878091FC059091FD05A091FE05B0912A
:10BD5000FF0589839A83AB83BC834EEFBE016B5F83
:10BD60007F4FCE010196DFDE6091200670912106A3
:10BD7000072E000C880B990B0E94B7EC6D837E8315
:10BD80008F8398878091F8059091F905A091FA0525
:10BD9000B091FB0589839A83AB83BC834FEFBE01CF
:10BDA0006B5F7F4FCE010196BEDEE1EEF1E1849143
:10BDB0008F010F5F1F4F882321F00E9417D9F801D0
:10BDC000F6CFE0919205F0E0E854F44E608170E027
:10BDD00080E090E00E9489D9ECEDF1E184918F013F
:10BDE0000F5F1F4F882321F00E9417D9F801F6CF6B
:10BDF0006091B71B70E080E090E00E9489D928969E
:10BE00000FB6F894DEBF0FBECDBFDF91CF911F916B
:10BE10000F9108952F923F924F925F926F927F926F
:10BE20008F929F92AF92BF92CF92DF92EF92FF924A
:10BE30000F931F93CF93DF93CDB7DEB72F970FB636
:10BE4000F894DEBF0FBECDBF8091911683FD02C274
:10BE500083E50E94FBD88887811106C082E50E9495
:10BE6000FBD8882309F4F6C10E9495D80E948FF46C
:10BE70006E37710514F06DE770E0709321066093E2
:10BE800020060E944FC60E9495D820E030E040EA8C
:10BE900050EC0E9471F5181614F40E94B8C881E0A5
:10BEA00080933D028091930580939205412C512C03
:10BEB00032011C821D821E821F821B8219862CE386
:10BEC0002A873CE13B8746E44C8710E000E050E8DD
:10BED00059838FEB8A83812C912C54016091200629
:10BEE00070912106072E000C880B990B0E94B7EC6D
:10BEF0007B018F879D879B01AC01612F702F89810A
:10BF00009A810E94B1EC882361F12091F80530916B
:10BF1000F9054091FA055091FB059885B7018F8589
:10BF200091110EC09D850E94B1EC881F8827881F43
:10BF30008B831E2D0F2DAF85A983BD85BA8311C0BC
:10BF40009D850E94B1EC87FF05C080913D02811163
:10BF5000CAC080C11E2D0F2D2F8529833D853A83B0
:10BF60001B820E940CDC6B017C01DC01CB012C816B
:10BF70003D814E815F81821B930BA40BB50BB7FDF6
:10BF80003BC0D701C60188519C4FAF4FBF4F8C8338
:10BF90009D83AE83BF83BBDEEDEFF1E18491DF01D2
:10BFA0001196BE87AD87882329F00E9417D9ED85A9
:10BFB000FE85F4CF81149104A104B104B9F0D50138
:10BFC000C401805F984DAF4FBF4FBC01CD016C19CC
:10BFD0007D098E099F0928EE33E040E050E00E9481
:10BFE000EDF2CA01B9010E9489D903C08FE30E9412
:10BFF00017D98AE00E9417D90E94A8AB0E940DD9D8
:10C000002090F8053090F905B091FA05BF8720918E
:10C01000FB052D8791014B2F5D85612F702F898145
:10C020009A810E944AF39F7781149104A104B1047C
:10C0300049F420E030E040E85FE30E94B1EC87FF84
:10C040000BC008C020E030E040E450E40E9471F5ED
:10C05000181614F4460157013B81332361F1411452
:10C0600051046104710441F0D701C6018419950996
:10C07000A609B709B7FD1FC091014F855D85698588
:10C080007A858B859C850E944AF320E030E040EC65
:10C090005FE30E94B1EC87FD58CF2601370140E6EF
:10C0A000440E4AEE541E611C711C29863A865F8537
:10C0B0005B878D858C8780913D02882309F445CF6D
:10C0C00081149104A104B10409F408CF90E1C91AC4
:10C0D00097E2D90AE108F108C818D908EA08FB086C
:10C0E000F7FE33CFFBCE8091C61A882309F4AFC088
:10C0F00080918F05882341F083EF91E19093151192
:10C10000809314110E94C5D780913917833009F0AC
:10C1100084C01092391781E080933C0280EA9FE04E
:10C120009093F91B8093F81B8091D51B882391F184
:10C1300082E090E090937E1580937D1585E080935A
:10C140007115A2E8A093741584E190E1A0E0B0E03D
:10C150008093751590937615A0937715B093781505
:10C16000A5D561E070E080E090E00E94D4DB81E042
:10C170009AE590937E1580937D158BE090E09093E7
:10C18000801580937F1587E080937115B2E8B09396
:10C19000741531C08EE090E090937E1580937D15EC
:10C1A00085E08093711522E82093741584E190E175
:10C1B000A0E0B0E08093751590937615A093771565
:10C1C000B093781573D561E070E080E090E00E9454
:10C1D000D4DB81E09AE590937E1580937D1585E30D
:10C1E00090E09093801580937F1587E08093711580
:10C1F00032E83093741584E890E0A0E0B0E08093DA
:10C20000751590937615A0937715B09378154ED544
:10C2100081E080933F178093D71B2F960FB6F89439
:10C22000DEBF0FBECDBFDF91CF911F910F91FF9069
:10C23000EF90DF90CF90BF90AF909F908F907F90C6
:10C240006F905F904F903F902F900C94B5A681E037
:10C250008093C51A2F960FB6F894DEBF0FBECDBFE0
:10C26000DF91CF911F910F91FF90EF90DF90CF90D2
:10C27000BF90AF909F908F907F906F905F904F9006
:10C280003F902F9008952F923F924F925F926F921E
:10C290007F928F929F92AF92BF92CF92DF92EF9256
:10C2A000FF920F931F93CF93DF93CDB7DEB76097C5
:10C2B0000FB6F894DEBF0FBECDBF8DE690E00E94B2
:10C2C000356F81115CC28091911683FD58C283E560
:10C2D0000E94FBD88987811106C082E50E94FBD8A5
:10C2E000882309F44CC20E9495D80E948FF4CB0198
:10C2F0000E94E7C60E9495D820E030E04AEA52E466
:10C300000E94B1EC181614F0B8D402C00E94B8C84C
:10C310000E94CF7281E080933D0219821A821B82B3
:10C320001C821D821E821F821886312C1A862CE3E5
:10C330002B873CE13C8746E44D87412C512C80E81B
:10C34000782E9FEB692E812C912C5401609122064E
:10C3500070912306072E000C880B990B0E94B7ECF6
:10C360008B01888B9E879B01AC01B201872D962D96
:10C370000E94B1EC882339F12091FC053091FD0534
:10C380004091FE055091FF058985B80181110CC0CF
:10C3900088899E850E94B1EC382E331C3324331CCF
:10C3A000280178886E840FC088899E850E94B1EC30
:10C3B00087FF05C080913D028111B8C0E0C128010E
:10C3C00078886E84312C0E940CDC6B017C01DC01CE
:10C3D000CB012D813E814F815885821B930BA40B8D
:10C3E000B50BB7FD3BC0D701C60188519C4FAF4F7D
:10C3F000BF4F8D839E83AF83B88789DCEFEEF1E179
:10C400008491DF011196BF87AE87882329F00E94AF
:10C4100017D9EE85FF85F4CF81149104A104B104EE
:10C42000B9F0D501C401805F984DAF4FBF4FBC013B
:10C43000CD016C197D098E099F0928EE33E040E09B
:10C4400050E00E94EDF2CA01B9010E9489D903C0EF
:10C450008FE30E9417D98AE00E9417D90E94A8ABE7
:10C460000E940DD90091FC051091FD05B091FE05CB
:10C47000B88B2091FF052E8798014B2F5E85B20166
:10C48000872D962D0E944AF39F7781149104A10471
:10C49000B10449F420E030E040E85FE30E94B1ECF1
:10C4A00087FF0BC008C020E030E040E450E40E9469
:10C4B00071F5181614F446015701332009F4EEC043
:10C4C00089819A81AB81BC81892B8A2B8B2B61F06E
:10C4D000D701C60129813A814B815C81821B930B74
:10C4E000A40BB50BB7FD0AC1980148895E856A8522
:10C4F0007B858C859D850E944AF320E030E040ECEE
:10C500005FE30E94B1EC87FD55CFD701C601805A89
:10C510009541AF4FBF4F89839A83AB83BC830A8712
:10C520001B8798899C87AE85AD87E8C08091C51A26
:10C53000882309F4AFC080918F05882341F085EEF0
:10C5400091E190931511809314110E94C5D78091A9
:10C550003917833009F084C01092391781E0809335
:10C560003C0280EA9FE09093F91B8093F81B809136
:10C57000D51B882391F182E090E090937E15809303
:10C580007D1585E08093711532E83093741584E150
:10C5900090E1A0E0B0E08093751590937615A0939C
:10C5A0007715B093781582D361E070E080E090E079
:10C5B0000E94D4DB81E09AE590937E1580937D15EF
:10C5C0008BE090E09093801580937F1587E08093B7
:10C5D000711542E84093741531C08EE090E090935D
:10C5E0007E1580937D1585E08093711552E85093F8
:10C5F000741584E190E1A0E0B0E08093751590930C
:10C600007615A0937715B093781550D361E070E05C
:10C6100080E090E00E94D4DB81E09AE590937E1563
:10C6200080937D1585E390E09093801580937F152E
:10C6300087E08093711582E88093741584E890E018
:10C64000A0E0B0E08093751590937615A0937715D0
:10C65000B09378152BD381E080933F178093D71B3D
:10C6600060960FB6F894DEBF0FBECDBFDF91CF91BD
:10C670001F910F91FF90EF90DF90CF90BF90AF9000
:10C680009F908F907F906F905F904F903F902F90F2
:10C690000C94B5A681E08093C61A71C06091220601
:10C6A00070912306072E000C880B990B0E94B7ECA3
:10C6B0009B01AC01B80188899E850E94B1EC282EAF
:10C6C000221C2224221C2092BF0C80913D02882330
:10C6D00061F1222051F181149104A104B10409F403
:10C6E0004BC0D701C60180519742A109B1098819F1
:10C6F0009909AA09BB09B7FF18C03EC0609122067C
:10C7000070912306072E000C880B990B0E94B7EC42
:10C710009B01AC0122242394B80188899E850E9444
:10C7200071F5181684F2212CCECF8091BE0C91E0C9
:10C73000980F9093BE0C833308F03CCEB1E0B093D9
:10C74000BF0C80913D02882309F434CE81149104FA
:10C75000A104B10461F020E1C21A27E2D20AE10883
:10C76000F108C818D908EA08FB08F7FE23CE809123
:10C77000BF0C8111EBCD1ECE1092BE0CE2CF6096A5
:10C780000FB6F894DEBF0FBECDBFDF91CF911F91E2
:10C790000F91FF90EF90DF90CF90BF90AF909F9060
:10C7A0008F907F906F905F904F903F902F90089563
:10C7B0008F929F92AF92BF92CF92DF92EF92FF92B1
:10C7C0000F931F93CF93DF93CDB7DEB7AC970FB620
:10C7D000F894DEBF0FBECDBF80917812882309F494
:10C7E000DEC082E494E10E944ED082E494E10E9493
:10C7F0008FB210927612109275128091781288235F
:10C8000009F4CDC0E0909005F09091050E94CAC750
:10C810001D8218861C821B828DEE92E09A8389838A
:10C8200084EA92E19093C4128093C312F70180814D
:10C830008F3209F064C06FE270E0C7010E9499F680
:10C840008C010F5F1F4FCE0101965C010115110590
:10C8500009F45BC06FE270E0C8010E9499F66C01B8
:10C86000009709F453C00817190708F04FC04C018E
:10C87000801A910AA401B801CE0180960E94C2F6E6
:10C88000E0E2F0E0EC0FFD1FE80DF91D10828E01D3
:10C89000005E1F4FF80181918F01882319F00E94DB
:10C8A00017D9F8CF8AE00E9417D96091C31270910E
:10C8B000C4126115710511F06C5F7F4F21E0AE016C
:10C8C000405E5F4FCE0105960E9424B881110FC0D3
:10C8D000BE01605E7F4F85EC91E10E94AD538EE218
:10C8E0000E9417D98AE00E9417D9C50156C0B0929C
:10C8F000C412A092C31286010F5F1F4FA7CF85EC11
:10C9000092E19093C4128093C31287018091C31265
:10C910009091C412009709F00496B8010E94A4D225
:10C92000882309F1EFE9F1E184917F019FEFE91A92
:10C93000F90A882321F00E9417D9F701F5CFF801F1
:10C9400081918F01882319F00E9417D9F8CF8AE0CE
:10C950000E9417D9109212151092131510921415E7
:10C960001092151518C0EDEAF1E184917F019FEF57
:10C97000E91AF90A882321F00E9417D9F701F5CFA7
:10C98000F80181918F01882319F00E9417D9F8CFFF
:10C990008EE20E9417D9CE0101960E949AA8AC9609
:10C9A0000FB6F894DEBF0FBECDBFDF91CF911F91C0
:10C9B0000F91FF90EF90DF90CF90BF90AF909F903E
:10C9C0008F9008958F929F92AF92BF92CF92DF92F5
:10C9D000EF92FF921F93CF93DF93C82F8BE194E1E7
:10C9E00090931311809312111092371482E090E00B
:10C9F000A0E0B0E08093201490932114A09322141F
:10CA0000B09323141092111110920D1110920E1167
:10CA100010920F11109210118FEF9FEFDC01809395
:10CA2000091190930A11A0930B11B0930C11CC2310
:10CA300079F1C53008F0F8C040E060E070E0CB016B
:10CA40000E943CCE882309F4EFC020E1C29FC001C0
:10CA500011248750914FFC01E254FE4F20812F7723
:10CA600009F0E2C03C964081518162817381443675
:10CA700051056105710508F4D7C03497C080D18095
:10CA8000E280F380C114D104E104F10421F4CCC0AC
:10CA9000C12CD12C760140E0C701B6010E943CCEEA
:10CAA000182F882309F4C0C08091140F9091150F9E
:10CAB0008115924009F0B8C0A091190FAA2309F47A
:10CAC000B3C06091170F7091180F6115710509F4CB
:10CAD000ABC02091160F222309F4A6C0A0933214F4
:10CAE0002093241480E030E041E050E0C82FFA01A8
:10CAF000082E02C0EE0FFF1F0A94E2F72E173F0721
:10CB000039F08F5FC83091F789E080932D148CC085
:10CB100080932D1420911F0F3091200F2115310586
:10CB200019F040E050E008C020912D0F30912E0FF9
:10CB300040912F0F5091300F2093251430932614DD
:10CB4000409327145093281446015701860E971ED0
:10CB5000A11CB11C8092331490923414A09235140D
:10CB6000B0923614E0911A0FF0911B0FF093391424
:10CB7000E0933814B0E00E942BF3860E971EA81E97
:10CB8000B91E80923A1490923B14A0923C14B09239
:10CB90003D1485E0EE0FFF1F8A95E1F7E150FE4F4F
:10CBA000EF2FFF27E6958E0E9F1EA11CB11C8092D1
:10CBB0002E1490922F14A0923014B0923114209120
:10CBC0001C0F30911D0F2115310521F0A90160E0E6
:10CBD00070E008C04091290F50912A0F60912B0FEF
:10CBE00070912C0FD701C60188199909AA09BB09B0
:10CBF000840F951FA61FB71F04C0B695A7959795DC
:10CC00008795CA95D2F78093291490932A14A093FC
:10CC10002B14B0932C14853F2FE09207A105B1058A
:10CC200028F48CE08093371410E01AC0853F9F4FA2
:10CC3000A105B10510F480E111C08091350F9091EC
:10CC4000360FA091370FB091380F80933A1490931C
:10CC50003B14A0933C14B0933D1480E280933714AE
:10CC6000812FDF91CF911F91FF90EF90DF90CF90B8
:10CC7000BF90AF909F908F90089580916712909190
:10CC800068120197029710F080E0089510926812E0
:10CC9000109267120E940CDC6093711270937212F2
:10CCA000809373129093741281E008950F931F93F1
:10CCB000CF93DF93209172152A3509F096C0909199
:10CCC0007315953A09F091C080917115833008F47D
:10CCD0008CC02093C1159093C2158093C315909179
:10CCE00074159093C4159038B1F490917515909384
:10CCF000C515EDE7F5E1A6ECB5E120E030E090E008
:10CD00000297281739070CF044C0408132964D93A2
:10CD10002F5F3F4FF6CF833061F4913809F062C046
:10CD2000809175158093C515809179158093C615EE
:10CD300030C09238F1F490917515209176152093BA
:10CD4000C5159093C615E7ECF5E120E030E090E0E2
:10CD5000039728173907ECF4D901AE7FA358BA4ED0
:10CD60004C9111965C91508341832E5F3F4F3296D8
:10CD7000F0CF843071F4933861F4809175159091FF
:10CD800076159093C5158093C6158091791580937B
:10CD9000C71501EC15E1C0E0D0E08091711590E07D
:10CDA00002968C179D074CF0D8016D918D0186E19C
:10CDB00091E10E94B0C12196F0CF80E5E1E7F5E175
:10CDC000DF011D928A95E9F78AE1E1ECF5E1DF01E7
:10CDD0001D928A95E9F78AE58093721585EA80931A
:10CDE000731503C09238A9F6A6CFDF91CF911F919A
:10CDF0000F91089561157105E1E08E07910550F0DE
:10CE000090937E1580937D157093801560937F15A8
:10CE100087E005C070937E1560937D1585E0809353
:10CE2000711582E8809374152093751530937615EB
:10CE3000409377155093781539CFEF92FF921F9357
:10CE4000CF93DF937C0160E00E94A9D7182F88233D
:10CE5000B1F0E2EBF2E18491EF012196882321F019
:10CE60000E9417D9FE01F7CFB70185EA92E10E942F
:10CE7000AD5382E20E9417D98AE00E9417D9812F10
:10CE8000DF91CF911F91FF90EF9008952F923F92E5
:10CE90004F925F926F927F928F929F92AF92BF92CA
:10CEA000CF92DF92EF92FF920F931F93CF93DF9376
:10CEB000CDB7DEB7AA970FB6F894DEBF0FBECDBFD1
:10CEC0002DB63EB68091A3128F938091A2128F93BC
:10CED0008CE992E19F938F938E010F5D1F4F1F93FB
:10CEE0000F930E9483EC0F900F900F900F900F9074
:10CEF0000F90F12CF80101900020E9F73197E01B29
:10CF0000F10BFE1684F46801CF0CD11CF7FCDA9407
:10CF1000F6018081082E000C990B0E945DF6F60147
:10CF20008083F394E7CF88EA92E10E94ECB3A12CCE
:10CF30009E012F5F3F4F790185E9482E82E1582EEF
:10CF400091E9692E92E1792E8091AB12823080F0C6
:10CF50008091B0129091B112A091B212B091B3121F
:10CF60008F719927AA27BB27892B8A2B8B2B61F1DD
:10CF7000A11003C08FEF9FEF05C08091A212909186
:10CF8000A31201969093A3128093A2120FB6F89465
:10CF90003EBE0FBE2DBEAA960FB6F894DEBF0FBEE2
:10CFA000CDBFDF91CF911F910F91FF90EF90DF9058
:10CFB000CF90BF90AF909F908F907F906F905F9039
:10CFC0004F903F902F90089540E050E0B70188EADD
:10CFD00092E10E94ECCF18165CF6F7010190002058
:10CFE000E9F73197BE2EBE18BA943FEFB31669F039
:10CFF0006701CB0CD11CB7FCDA94F601808190E07C
:10D000000E945DF6F6018083EFCF8A858E3709F4A2
:10D010009BCF45E050E0B801C7010E94B4F6892BD0
:10D0200009F092CF8DB69EB6F80101900020E9F785
:10D03000CF01801B910B04962DB73EB7281B390BEF
:10D040000FB6F8943EBF0FBE2DBF8DB79EB70196A9
:10D050006C011F930F935F924F92DF928F930E9408
:10D0600083EC560194E0A90EB11C0F900F900F9025
:10D070000F900F900F90F5018081882349F0082EC2
:10D08000000C990B0E945DF6F50181935F01F3CFCF
:10D09000C601D3DE70921511609214110E94C5D79B
:10D0A0000FB6F8949EBE0FBE8DBEAA24A3944CCF9B
:10D0B000CF92DF92EF92FF921F93CF93DF93109264
:10D0C00078128091AB12882321F088EA92E10E94C5
:10D0D0008FB210921F1410921C1485E380931B14BE
:10D0E0000E940CDCEB01A89561E080911B140E946A
:10D0F000D0DA8BE194E10E94F1B32398229A219A2D
:10D10000209A289A85E080931D1482E58CBD1DBC71
:10D110001AE08FEF0E94F6B31150D9F720E030E00B
:10D12000A90160E08BE194E10E94FBB3182F80938A
:10D130001E14813049F00E940CDC6C1B7D0B613D9C
:10D14000774060F381E054C02AEA31E040E050E0EB
:10D1500068E08BE194E10E94FBB382FF03C010936F
:10D160001F140EC014E00E94AEA680931E1411502E
:10D17000D1F78A3A11F082E03BC082E080931F141D
:10D1800080911F14823021F0C12CD12C760105C072
:10D19000C12CD12CE12C80E4F82E20E030E0A90154
:10D1A00067E38BE194E10E94FBB3A701960169E27A
:10D1B0008BE194E10E94FBB380931E14882349F015
:10D1C0000E940CDC6C1B7D0B613D774030F38AE0E4
:10D1D0000FC080911F14823011F520E030E0A901CA
:10D1E0006AE38BE194E10E94FBB3882351F088E06D
:10D1F00080931C148BE194E10E94F1B3E2EBF2E125
:10D2000019C00E94AEA6807C803C19F483E0809314
:10D210001F140E94AEA60E94AEA60E94AEA68BE18D
:10D2200094E10E94F1B310921D1481E0CBDB8111D7
:10D2300031C015C08491EF012196882321F00E940E
:10D2400017D9FE01F7CFE3E8F2E18491EF012196CF
:10D25000882309F456C00E9417D9FE01F6CF80E05A
:10D26000B1DB811117C0ECE7F2E18491EF01219667
:10D27000882321F00E9417D9FE01F7CFE8E6F2E1FA
:10D280008491EF012196882309F43BC00E9417D9AD
:10D29000FE01F6CF60E274E188EA92E10E943CB2BE
:10D2A000811116C0ECE7F2E18491EF012196882309
:10D2B00021F00E9417D9FE01F7CFE7E5F2E1849152
:10D2C000EF0121968823E9F00E9417D9FE01F7CFDC
:10D2D00081E080937812E2EBF2E18491EF012196F4
:10D2E000882321F00E9417D9FE01F7CFEBE4F2E189
:10D2F0008491EF012196882321F00E9417D9FE0125
:10D30000F7CF8BE1E8EAF2E1A9ECB2E101900D92EE
:10D310008A95E1F78091A6129091A7129093C81276
:10D320008093C71284EA92E19093C4128093C3124F
:10D33000DF91CF911F91FF90EF90DF90CF900895F4
:10D340008F929F92AF92BF92CF92DF92EF92FF9215
:10D350000F931F93CF93DF9300D01F92CDB7DEB70B
:10D36000FC018381813011F080E06BC0818181FFFD
:10D37000FBCF81899289A389B489892B8A2B8B2B36
:10D3800009F45EC07F0140E050E0BA01CF010E9485
:10D3900080D0882349F3F70185889688A788B08CC8
:10D3A000C18CD28C82E090E0A0E0B0E0F6018083F6
:10D3B0009183A283B3839E012F5F3F4FB501A401E8
:10D3C000C6010E9405CF882379F200E010E09801A1
:10D3D000B501A401C6010E9474CE882329F2898078
:10D3E0009A80AB80BC80F6018789803141F4F8EFE8
:10D3F0008F16FFEF9F06A104B10448F4DCCF88EF3D
:10D4000088168FEF9806A8068FE0B806A0F2F701FD
:10D41000158A168A178A108E118A128A138A148A1C
:10D42000818180688183C7010E944ED0882309F4DE
:10D430009BCF40E050E0BA01C7010E9480D001C0FC
:10D4400081E00F900F900F900F90DF91CF911F917F
:10D450000F91FF90EF90DF90CF90BF90AF909F9093
:10D460008F9008950F931F93CF93DF93209178129D
:10D47000222309F44FC02091641421114BC0262FA0
:10D48000C92FD82F482F592F68EA72E181E694E11D
:10D490000E9424B8811121C0E5E2F2E184918F015C
:10D4A0000F5F1F4F882321F00E9417D9F801F6CF94
:10D4B0000D2F1C2FF80181918F01882319F00E94F4
:10D4C00017D9F8CFE2E2F2E18491EF0121968823A7
:10D4D00009F10E9417D9FE01F7CFE9E3F2E1849147
:10D4E0008F010F5F1F4F882321F00E9417D9F80189
:10D4F000F6CF0D2F1C2FF80181918F01882319F091
:10D500000E9417D9F8CF8AE0DF91CF911F910F9138
:10D510000C9417D9DF91CF911F910F91089540E09E
:10D5200050E0BA0181E694E10E9480D049E452E0E3
:10D5300060EC7CE081E694E10C9416D10F931F938C
:10D540008091671290916812019719F40E940CDC87
:10D5500008C0609171127091721280917312909153
:10D56000741200916D1210916E1220916F12309111
:10D570007012601B710B820B930B28EE33E040E0BE
:10D5800050E00E94EDF28091691290916A12A09190
:10D590006B12B0916C12BC01CD01620F731F841F1E
:10D5A000951F1F910F910895CF92EF92FF920F93C5
:10D5B0001F93CF93DF93CDB7DEB72C970FB6F894B8
:10D5C000DEBF0FBECDBFC09093058091DA1690915B
:10D5D000DB16A091DC16B091DD164091D616509165
:10D5E000D7166091D8167091D9160091D216109165
:10D5F000D3162091D4163091D51609831A832B8324
:10D600003C834D835E836F83788789879A87AB8756
:10D61000BC8780910E0681110AC0AE01475F5F4F43
:10D62000BE016B5F7F4FCE0101960E943681E09074
:10D630003402F090350200913602109137022EED3F
:10D6400036E1AE01475F5F4FBE016B5F7F4FCE019A
:10D6500001960E941D742C960FB6F894DEBF0FBE83
:10D66000CDBFDF91CF911F910F91FF90EF90CF90A1
:10D670000895FF920F931F93CF93DF93F82E092FF6
:10D68000162FECE7F2E18491EF012196882321F037
:10D690000E9417D9FE01F7CFEF2DF02F8491EF01F3
:10D6A0002196882321F00E9417D9FE01F7CF6091BF
:10D6B0004B1B70914C1B80914D1B90914E1B0E94F7
:10D6C00089D98AE00E9417D911110E94F7B11092EE
:10D6D000421610924116DF91CF911F910F91FF904A
:10D6E00008951F93CF93DF93CDB7DEB72C970FB676
:10D6F000F894DEBF0FBECDBF882331F02091731A9E
:10D700003091741A232BF9F0909154168917D9F09F
:10D71000182F8CE0E1E0F3E0DE01119601900D920C
:10D720008A95E1F7CE0101960E94D4AF109354166A
:10D73000111105C082E090E00E9488AF04C082ED24
:10D7400096E10E94B7802C960FB6F894DEBF0FBE0C
:10D75000CDBFDF91CF911F910895BC0186E492E186
:10D760000E94235267E771E080E090E00C94B6C21B
:10D770001F93CF93DF93882329F04B9908C08AE049
:10D7800090E002C08AE590E0E8DF10E04DC08CE355
:10D7900090E0E3DF8AE090E0E0DF8AE590E0DDDF23
:10D7A0006CED75E080E090E00E94B6C24B9BE7CF45
:10D7B000ECE7F2E18491EF012196882321F00E94A9
:10D7C00017D9FE01F7CFE8EBF4E18491EF01219640
:10D7D000882321F00E9417D9FE01F7CF0E94EDC6E1
:10D7E000109160021123F9F0ECE7F2E18491EF016E
:10D7F0002196882321F00E9417D9FE01F7CFE1E49A
:10D80000F4E18491EF012196882321F00E9417D939
:10D81000FE01F7CF6EE571E080E090E00E94B6C2B5
:10D820001092600201C011E0812FDF91CF911F9112
:10D8300008958091481690914916A0914A16B0918A
:10D840004B168093340290933502A0933602B09326
:10D850003702809146169091471690930C02809360
:10D860000B020C940DD98091340290913502A09155
:10D870003602B09137028093481690934916A093D0
:10D880004A16B0934B1680910B0290910C02909324
:10D8900047168093461684E690E090930C0280939E
:10D8A0000B020C940DD94F925F926F927F928F92E0
:10D8B0009F92AF92BF92CF92DF92EF92FF920F931F
:10D8C0001F93CF93DF935C014B018A01E9014090E4
:10D8D0003402509035026090360270903702FA019F
:10D8E00020813181428153816091DA167091DB167B
:10D8F0008091DC169091DD160E94B1EC87FF2DC05F
:10D90000C880D980EA80FB8020E030E0A901B60120
:10D91000C7010E94B1EC811108C0EFEAFDE18591D9
:10D920009591A591B4916C017D01C601D7018093B9
:10D93000340290933502A0933602B0933702F80177
:10D9400080819181A281B3818093DA169093DB1656
:10D95000A093DC16B093DD1627DEC880D980EA805C
:10D96000FB8020E030E0A901C701B6010E94B1ECC4
:10D97000811108C0C0902F02D0903002E090310297
:10D98000F0903202C0923402D0923502E092360218
:10D99000F0923702F50180819181A281B381809359
:10D9A000D2169093D316A093D416B093D516F40143
:10D9B00080819181A281B3818093D6169093D716EE
:10D9C000A093D816B093D916EFDDF80120813181EC
:10D9D000428153816091DA167091DB168091DC16DA
:10D9E0009091DD160E9471F518169CF5D880E9809B
:10D9F000FA80CB8120E030E0A9016D2D7E2D8F2DA6
:10DA00009C2F0E94B1EC81110AC0EFEAFDE18591E3
:10DA10009591A591B491D82EE92EFA2ECB2F8D2D6C
:10DA20009E2DAF2DBC2F8093340290933502A0938E
:10DA30003602B0933702F80180819181A281B381CF
:10DA40008093DA169093DB16A093DC16B093DD1664
:10DA5000ABDD0E943AD74092340250923502609278
:10DA6000360270923702DF91CF911F910F91FF9094
:10DA7000EF90DF90CF90BF90AF909F908F907F906E
:10DA80006F905F904F9008959B01AC0166ED76E139
:10DA900082ED96E108CFCF92DF92EF92FF921F9333
:10DAA000CF93DF93CDB7DEB728970FB6F894DEBFDC
:10DAB0000FBECDBF6D837E838F83988769017A0106
:10DAC00081E056DE882311F081E027C020E030E0BD
:10DAD00040E752E4C701B6010E9427F469837A83C4
:10DAE0008B839C83BE016F5F7F4FCE010596CCDF99
:10DAF00080914006182F147082FF04C080E038DE49
:10DB00008111E2CF1092400682E090E00E9488AF3F
:10DB10000E941ED881E0111180E028960FB6F8947B
:10DB2000DEBF0FBECDBFDF91CF911F91FF90EF9071
:10DB3000DF90CF900895CF92DF92EF92FF921F93E4
:10DB4000CF93DF93CDB7DEB72C970FB6F894DEBF37
:10DB50000FBECDBF90910F06981709F469C0182F1A
:10DB600080E090E0A0E2B1E48D839E83AF83B8872C
:10DB7000C0902E17D0902F17E0903017F0903117EB
:10DB800020E030E0A901C701B6010E94B1EC87FF97
:10DB90000CC0A701960160E070E080E291E40E9471
:10DBA0004AF36D837E838F8398872D813E814F81D9
:10DBB00058856091DA167091DB168091DC16909191
:10DBC000DD160E94B1EC87FF0AC019821A821B82FF
:10DBD0001C82BE016F5F7F4FCE01059655DF80919D
:10DBE000D2169091D316A091D416B091D5168987EC
:10DBF0009A87AB87BC878091D6169091D716A09153
:10DC0000D816B091D9168D839E83AF83B8871982B9
:10DC10001A821B821C829E012F5F3F4F4AED56E104
:10DC2000BE016B5F7F4FCE0109963DDE10930F065C
:10DC300080E02C960FB6F894DEBF0FBECDBFDF910B
:10DC4000CF911F91FF90EF90DF90CF90089580E1EA
:10DC5000E2EDF6E1A3E9BAE101900D928A95E1F7D0
:10DC6000089580E1E3E9FAE1A2EDB6E101900D92B9
:10DC70008A95E1F708958F929F92AF92BF92CF92CB
:10DC8000EF92FF920F931F93CF93DF93CDB7DEB741
:10DC90002C970FB6F894DEBF0FBECDBF4B015C01D1
:10DCA000C090930580919B1A90919C1AA0919D1A07
:10DCB000B0919E1A4091971A5091981A6091991AB2
:10DCC00070919A1A0091931A1091941A2091951AB2
:10DCD0003091961A09831A832B833C834D835E838C
:10DCE0006F83788789879A87AB87BC8780910E0678
:10DCF00081110AC0AE01475F5F4FBE016B5F7F4F6E
:10DD0000CE0101960E943681850174012FE93AE126
:10DD1000AE01475F5F4FBE016B5F7F4FCE01019643
:10DD20008CD52C960FB6F894DEBF0FBECDBFDF9119
:10DD3000CF911F910F91FF90EF90CF90BF90AF9038
:10DD40009F908F900895CF92DF92EF92FF920F9362
:10DD50001F93CF93DF93EC01CC0FDD1FCC0FDD1FA2
:10DD6000FE01E05FF94F20E030E0A90160817181A0
:10DD7000828193810E944BF3FE01EC57F54E208186
:10DD80003181428153810E944BF36B017C01FE0182
:10DD9000EE51F94E6083718382839383FE01E75DC8
:10DDA000FB4E25913591459154918E010858154EA1
:10DDB0000E944BF3F8016083718382839383FE0199
:10DDC000EB5CFB4E2591359145915491C15CDD4F43
:10DDD000C701B6010E944BF3688379838A839B83D2
:10DDE000DF91CF911F910F91FF90EF90DF90CF9037
:10DDF00008958F929F92AF92BF92EF92FF920F93EE
:10DE00001F93CF93DF938C014A015B01EC01CC0F90
:10DE1000DD1FCC0FDD1FCE018E52994E7C01C05FFD
:10DE2000D94F288139814A815B81C501B4010E94A3
:10DE30004AF3F70120813181428153810E944BF3E3
:10DE4000F701608371838283938388829982AA8297
:10DE5000BB82C801DF91CF911F910F91FF90EF908E
:10DE6000BF90AF909F908F906ECFEF92FF920F93E5
:10DE70001F93CF93DF937C0184E50E94FBD8D82FBA
:10DE8000882349F10E9475D8C82F181604F5E2EBD3
:10DE9000F2E184918F010F5F1F4F882321F00E94D0
:10DEA00017D9F801F6CF8DE40E9417D9B70180E0A9
:10DEB00090E04AE00E941ED96C2FCC0F770B86E1D0
:10DEC00094E10E9494538AE00E9417D908C080937D
:10DED0009205D0E004C080919305809392058D2F28
:10DEE000DF91CF911F910F91FF90EF9008952F92A6
:10DEF0003F924F925F926F927F928F929F92AF92DA
:10DF0000BF92CF92DF92EF92FF920F931F93CF9326
:10DF1000DF9300D0CDB7DEB70E94C5D7811129C3EA
:10DF200080913217843008F066C00E9414DA9C0198
:10DF300097FD61C0982F00914116109142168A30CA
:10DF400019F09D3009F0E7C2109243160115110532
:10DF500039F3F801EF51FA4E1082109242161092E6
:10DF6000411621EE35E18901D9018C912F5F3F4F98
:10DF70008032C9F38E3409F03DC278016AE270E064
:10DF8000C8010E9499F66C01E114F10409F478C209
:10DF90006EED73E1C8010E9469EC5C01892B09F008
:10DFA0002CC24AE050E060E070E0C70101960E9498
:10DFB00003EA6093DD157093DE158093DF1590936F
:10DFC000E01540904B1B50904C1B60904D1B709087
:10DFD0004E1BBFEF4B1A5B0A6B0A7B0A6415750573
:10DFE0008605970509F414C2AB2809F011C261E057
:10DFF0008BEA93E13EDB80917712882309F4B9C262
:10E0000080913217811102C01092451681E08B83F6
:10E0100040911215509113156091141570911515BA
:10E0200080910E1590910F15A0911015B0911115BA
:10E03000481759076A077B0708F41B8200E010E0C5
:10E0400034E6232E312C4FE0442E40E1542E612C37
:10E05000712C54E8852E912CA12CB12C8091321773
:10E06000843008F086C29B81911183C2809145164D
:10E0700081117FC280914A1490914B14A0914C144D
:10E08000B0914D148093121590931315A09314150D
:10E09000B093151541E050E0BE016F5F7F4F82E401
:10E0A00094E10E9417B5019719F4898190E002C0AC
:10E0B0008FEF9FEF8A83C0901215D0901315E090D8
:10E0C0001415F090151540910E1550910F15609193
:10E0D000101570911115A1E0AB83C416D506E606A4
:10E0E000F70608F41B82C416D506E606F706A0F468
:10E0F000019609F42BC1EA81EA3009F447C1ED30F9
:10E1000009F444C1E33219F0EA3309F056C18091B1
:10E110004416811152C134C1E2E0F4E184916F01EF
:10E120002FEFC21AD20A882321F00E9417D9F601D4
:10E13000F5CF0E943AD782E494E10E948FB2809199
:10E140007C14882371F1815080937C14ADE88A9F00
:10E15000C001112441E061E08F579B4E0E9442CBE9
:10E16000E0917C14B4E0EB9FF0011124E358FB4EE6
:10E170004081518162817381409312155093131530
:10E18000609314157093151582E494E10E9480D079
:10E1900080917812882309F440C081E0809377123F
:10E1A0003CC0109277126AE588EF9EE05BD910922E
:10E1B000C00C1092080FB3D9019679F42CE9C22E45
:10E1C00023E0D22ED6018D916D01882319F00E9493
:10E1D00017D9F8CF8AE00E9417D981E694E10E940E
:10E1E0008FB210923D1710923C17E7EEF3E1F093D7
:10E1F0001511E09314110E94C5D70E943D669ED967
:10E200006D3371058105910540F083EE93E19093A4
:10E210001511809314110E94C5D710921A15809180
:10E220007812882319F00E94466706C00E94586839
:10E23000809178128111F7CF80913817813009F0E1
:10E240009FC01092381730927E1520927D1585E080
:10E25000C82EC092711592E8D92ED092741586E11D
:10E2600090E1A0E0B0E08093751590937615A093AF
:10E270007715B09378150E94566661E070E080E0F3
:10E2800090E00E94D4DB30927E1520927D15C092E2
:10E290007115D09274158EE090E1A0E0B0E080930B
:10E2A000751590937615A0937715B09378150E9405
:10E2B000566661E070E080E090E00E94D4DB30922E
:10E2C0007E1520927D15C0927115D09274154092E2
:10E2D00075155092761560927715709278150E9498
:10E2E00056668091D51B882369F0A1E0BAE5B0930A
:10E2F0007E15A0937D15E9E0F0E0F0938015E093A2
:10E300007F150CC081E09AE590937E1580937D1572
:10E31000A3E3B0E0B0938015A0937F1587E08093CE
:10E320007115D09274158092751590927615A09201
:10E330007715B09278150E9456661092DC151092EF
:10E34000D71B10923F17109237171AC0ECE7F2E173
:10E3500084916F01BFEFCB1ADB0A882321F00E9462
:10E3600017D9F601F5CFE3EFF3E184916F012FEFB9
:10E37000C21AD20A882321F00E9417D9F601F5CFDC
:10E380008A81833219F481E08093451610924416F5
:10E390000115110509F462CE8091341790E6899F2A
:10E3A000000D111D1124F801EF5BF94F108280E080
:10E3B0000E9494D700E010E051CE0F35110508F00F
:10E3C0004DCEAA81AB3319F481E08093441680913D
:10E3D0004416811143CE80913417F801B0E68B9F2B
:10E3E000E00DF11D1124EF5BF94F2A8120830F5FAF
:10E3F0001F4F34CEE12CF12CC1CD6EE470E0C8018A
:10E4000004960E9499F6009709F4CBCD7C01C9CD02
:10E41000C114D10401F180E0F12CF801E80FF11DE5
:10E4200090819A3219F08F5FF926F7CF4AE050E0D9
:10E4300060E070E0C60101960E9403EACF2CD12C67
:10E44000E12CF12C6C157D058E059F0541F061E0F6
:10E450008CE893E1CFCD61E082E693E1CBCD809172
:10E46000DD159091DE15A091DF15B091E015809338
:10E470004B1B90934C1BA0934D1BB0934E1B06C09F
:10E48000892B21F060E088E393E1B4CD80916002B4
:10E4900081111EC067E470E0C8010E9499F60097E0
:10E4A000B9F04AE050E060E070E001960E9403EAB3
:10E4B0006430710568F4E1ECF2E184917F012FEFA3
:10E4C000E21AF20A882321F00E9417D9F701F5CF4A
:10E4D00067E274E0C8010E94A4F6892B11F410923F
:10E4E0003D026CE274E0C8010E94A4F6892B21F47D
:10E4F00088EB92E10E94BEA861E374E0C8010E942B
:10E50000A4F6892B11F40E94278A61E081EE95E13F
:10E510000E94A9D705CD0F3511050CF001CD9C3512
:10E52000A1F40E9414DA97FDFBCC2091431621112F
:10E53000F7CC98012F5F3F4F30934216209341163E
:10E54000F801EF51FA4E8083EBCC9B3319F481E054
:10E5500080934316809143168111E2CCC801019645
:10E560009093421680934116F801EF51FA4E2083A2
:10E57000D7CC0F900F900F90DF91CF911F910F91FB
:10E58000FF90EF90DF90CF90BF90AF909F908F90D3
:10E590007F906F905F904F903F902F90089586E40A
:10E5A0000E94CCD88093AF1B882351F00E9495D84D
:10E5B00060932B0270932C0280932D0290932E0275
:10E5C00083E50E94CCD8882351F00E9495D86093AF
:10E5D0002702709328028093290290932A0282E4F2
:10E5E0000E94CCD8882351F00E9495D860932302D2
:10E5F00070932402809325029093260208954F92EF
:10E600005F926F927F928F929F92AF92BF92EF92A2
:10E61000FF920F931F93CF93DF93C2EAD6E182EB71
:10E62000E82E86E1F82E02E916E1412C512C320148
:10E6300043946991799189919991F7018190919091
:10E64000A190B1907F010E94B5ECA50194010E94B8
:10E6500016ED0E9494F4F801619371938193919364
:10E660008F01461657066806790610F42B013C0107
:10E67000F6E1C23BDF07E9F66FEF7FEFCB01A301C5
:10E6800092010E94EDF22093C7163093C816409372
:10E69000C9165093CA16DF91CF911F910F91FF9029
:10E6A000EF90BF90AF909F908F907F906F905F9012
:10E6B0004F9008952F923F924F925F926F927F9268
:10E6C0008F929F92AF92BF92CF92DF92EF92FF9282
:10E6D0000F931F93CF93DF9300D01F92CDB7DEB778
:10E6E0007B016A011901A2EBB6E12D913D914D919B
:10E6F0005C91FC0160817181828193810E9416EDA1
:10E700000E947DF52B013C0107EC11E1D8016D93CE
:10E710007D938D939C9313972091B6163091B716E5
:10E720004091B8165091B916F701608171818281CC
:10E7300093810E9416ED0E947DF54B015C01D8018A
:10E7400014966D937D938D939C9317972091BA1691
:10E750003091BB164091BC165091BD16F6016081F8
:10E760007181828193810E9416ED0E947DF56B017B
:10E770007C01D80118966D937D938D939C931B9784
:10E780002091BE163091BF164091C0165091C1160F
:10E79000F10160817181828193810E9416ED0E9456
:10E7A0007DF569837A838B839C83D8011C966D9356
:10E7B0007D938D939C931F970E943AD78FB7F894BF
:10E7C000E0EEFBE140825182628273828482958214
:10E7D000A682B782C086D186E286F38629813A81F5
:10E7E0004B815C8124873587468757878FBF10927E
:10E7F000B3111092B4111092B5111092B61180E1BC
:10E80000E7EBF1E1DF011D928A95E9F70F900F9098
:10E810000F900F90DF91CF911F910F91FF90EF908C
:10E82000DF90CF90BF90AF909F908F907F906F9030
:10E830005F904F903F902F9008952F923F924F926C
:10E840005F926F927F928F929F92AF92BF92CF9280
:10E85000DF92EF92FF920F931F93CF93DF93CDB789
:10E86000DEB7C657D1090FB6F894DEBF0FBECDBFD5
:10E870003B014A015901E9A6FBAE0CAF1EAF3C2C8F
:10E880002091B2163091B3164091B4165091B5163E
:10E89000DC016D917D918D919C910E9416ED0E94FD
:10E8A0007DF5AF966CAF7DAF8EAF9FAFAF972091E8
:10E8B000B6163091B7164091B8165091B916F301BB
:10E8C00060817181828193810E9416ED0E947DF5A5
:10E8D000E3966CAF7DAF8EAF9FAFE3972091BA16F2
:10E8E0003091BB164091BC165091BD16D4016D916C
:10E8F0007D918D919C910E9416ED0E947DF5E79689
:10E900006CAF7DAF8EAF9FAFE7972091BE16309171
:10E91000BF164091C0165091C116F50160817181FA
:10E92000828193810E9416ED0E947DF569966CAFFD
:10E930007DAF8EAF9FAF69978091C7119091C8113D
:10E94000A091C911B091CA11AF968CAC9DACAEAC80
:10E95000BFACAF97881A990AAA0ABB0A8091CB115B
:10E960009091CC11A091CD11B091CE11E396CCAC89
:10E97000DDACEEACFFACE397C81AD90AEA0AFB0A91
:10E98000CFA6D8AAE9AAFAAA8091CF119091D01166
:10E99000A091D111B091D211E796CCACDDACEEAC28
:10E9A000FFACE797C81AD90AEA0AFB0ACBAADCAA85
:10E9B000EDAAFEAA8091911683FF0EC06996CCAC99
:10E9C000DDACEEACFFAC6997C092D311D092D411FC
:10E9D000E092D511F092D6118091D3119091D4117B
:10E9E000A091D511B091D61169964CAC5DAC6EACCE
:10E9F0007FAC6997481A590A6A0A7B0A09F473C0FE
:10EA00000E943854882349F16996CCACDDACEEAC59
:10EA1000FFAC6997C092D311D092D411E092D51176
:10EA2000F092D611E2EBF2E184918F010F5F1F4F5C
:10EA3000882321F00E9417D9F801F6CFE1E1F5E132
:10EA400084918F010F5F1F4F882321F00E9417D9F7
:10EA5000F801F6CF412C512C32017301620177FE8F
:10EA600007C0CC24DD247601C418D508E608F708D1
:10EA70006091BE167091BF168091C0169091C1161C
:10EA80000E948FF49B01AC01A8EEB3E00E942BF32F
:10EA90006C157D058E059F054CF56996CCACDDACFB
:10EAA000EEACFFAC6997C092D311D092D411E09232
:10EAB000D511F092D611E2EBF2E184918F010F5F54
:10EAC0001F4F882321F00E9417D9F801F6CFE2EFFB
:10EAD000F4E184918F010F5F1F4F882321F00E9482
:10EAE00017D9F801F6CF412C512C3201D501C401C0
:10EAF0008827B7FD83959927AA27BB27182FCFA46E
:10EB0000D8A8E9A8FAA8F7FC1260CBA8DCA8EDA861
:10EB1000FEA8F7FC146077FC1860E32CF12CC70109
:10EB2000880F991F880F991F9C012357394E69013F
:10EB3000C301B2010E94B7ECD6012D913D914D91D8
:10EB40005C910E9416ED2B013C01F701EE0FFF1FB7
:10EB5000EF5DFD4F60817181072E000C880B990BD2
:10EB60000E94B7EC9B01AC01C301B2010E9416EDFB
:10EB70002AE037ED43E25CE30E9416ED2B013C01F5
:10EB800020E030E0A9010E9471F518164CF420E055
:10EB900030E040E05FE3C301B2010E944BF308C0E4
:10EBA000A301920160E070E080E09FE30E944AF3DD
:10EBB0000E948FF46FAB78AF89AF9AAF8091D71175
:10EBC0008F5F8F70A1968FAFA1978091D811A1967A
:10EBD000CFACA197C81203C00E94A8ABF6CFE091BA
:10EBE000D711EE2EF12CFEA6EDA62DE4E29FF0014A
:10EBF0001124EA53F84F108212A3D501C401B7FEC5
:10EC000007C088279927DC0188199909AA09BB0937
:10EC100082839383A483B5838DE4CDA4DEA48C9DED
:10EC2000F0018D9DF00D1124EA53F84F8FA598A99E
:10EC3000A9A9BAA9B7FF07C0B095A09590958195ED
:10EC40009F4FAF4FBF4F86839783A087B1878DE4D7
:10EC5000EDA4FEA48E9DF0018F9DF00D1124EA53CA
:10EC6000F84F8BA99CA9ADA9BEA9B7FF07C0B09565
:10EC7000A095909581959F4FAF4FBF4F8287938707
:10EC8000A487B5878DE4CDA4DEA48C9DF0018D9D75
:10EC9000F00D1124EA53F84FCFA8D8ACE9ACFAAC88
:10ECA000C686D786E08AF18A028113812481358164
:10ECB0004681578160857185401751076207730748
:10ECC00014F4B901A8018DE4EDA4FEA48E9DF00119
:10ECD0008F9DF00D1124EA53F84FC284D384E4844D
:10ECE000F5848FA998ADA9ADBAADC416D506E606D0
:10ECF000F70644F484179507A607B70754F4DB0119
:10ED0000CA0107C08C159D05AE05BF0514F4D701D7
:10ED1000C6014DE4CDA4DEA44C9DF0014D9DF00D47
:10ED20001124EA53F84F828B938BA48BB58B0697F3
:10ED3000A105B10510F40C949D80DF01A95BBF4FC4
:10ED400080913A1790913B178D939C933182012BC0
:10ED5000022B032B09F05F988DE4EDA4FEA48E9D99
:10ED6000F0018F9DF00D1124EA53F84F86819781B1
:10ED7000A085B185892B8A2B8B2B09F08A988DE48D
:10ED8000CDA4DEA48C9DF0018D9DF00D1124EA53DD
:10ED9000F84F82859385A485B585892B8A2B8B2B8B
:10EDA00041F09FB7F894809108018E7F809308010D
:10EDB0009FBFCFA8D8ACE9ACFAACCD28CE28CF28DD
:10EDC00011F40C9483808091C616882319F0815029
:10EDD0008093C616311004C0129880E28093C61644
:10EDE0002090891630908A1600918B1610918C16FF
:10EDF00029A53BAD4CAD5EADB101C8010E9471F5D6
:10EE0000181614F00C949780C501B4010E94B7EC59
:10EE10002091240630912506409126065091270620
:10EE20000E9416ED69A77AA78BA79CA769837A83AE
:10EE30008B839C836FA578A989A99AA90E94B7ECB6
:10EE4000209128063091290640912A0650912B06E0
:10EE50000E9416ED4B015C016D837E838F83988742
:10EE60006BA97CA98DA99EA90E94B7EC20912C06C4
:10EE700030912D0640912E0650912F060E9416EDDE
:10EE80006B017C0169877A878B879C87209130068C
:10EE9000309131064091320650913306C301B201E0
:10EEA0000E9416ED6D877E878F87988B2DE44DA588
:10EEB0005EA5249FF001259FF00D1124EA53F84F21
:10EEC000428053806480758056E045165104610489
:10EED0007104E4F44680578060847184A6E04A1689
:10EEE00051046104710494F44284538464847584ED
:10EEF000B6E04B1651046104710444F4DC01CB010B
:10EF0000BF7787A790ABA1ABB2AB34C029A53AA518
:10EF10004BA55CA5CA01B9010E9416ED2B013C016D
:10EF2000A5019401C501B4010E9416ED9B01AC013D
:10EF3000C301B2010E944BF34B015C01A701960192
:10EF4000C701B6010E9416ED9B01AC01C501B401D9
:10EF50000E944BF30E94B7F52DE4CDA4DEA42C9DB6
:10EF6000F0012D9DF00D1124EA53F84F67A770AB07
:10EF700081AB92AB8DE4EDA4FEA48E9DF0018F9D3C
:10EF8000F00D1124EA53F84F27A530A941A952A941
:10EF900060E070E080E89FE30E9427F422966CAF67
:10EFA0007DAF8EAF9FAF22979B01AC01B101C8012D
:10EFB0000E9416ED6B017C018091D7119091D811C0
:10EFC000891B8F7027968FAF2797A701960160E066
:10EFD00074E284E799E40E9427F40E947DF54B01D6
:10EFE0005C0127968FAD27978250863008F044C089
:10EFF0008091811690918216A0918316B09184160B
:10F0000088169906AA06BB06B8F588199909AA09AF
:10F01000BB09BC01CD01660F771F881F991F27967A
:10F02000FFAC27970F2D10E020E030E0A9019801F8
:10F030000E94EDF2CA01B9010E94B5EC0E947DF573
:10F04000680D791D8A1D9B1D0E94B5EC9B01AC01CA
:10F0500060E074E284E799E40E9427F46B017C018C
:10F060009B01AC0160E074E284E799E40E9427F41C
:10F070000E947DF54B015C012FB7F8948091C20787
:10F080009091C307A091C407B091C507880E991E3F
:10F09000AA1EBB1E8092C2079092C307A092C4070B
:10F0A000B092C5072FBF8DE42DA53EA5829F80019C
:10F0B000839F100D11240A53184FD8019F964D912C
:10F0C0005D916D917C91D297A5964CAF5DAF6EAF7F
:10F0D0007FAFA5979A01AB01C701B6010E9416ED5B
:10F0E00026966CAF7DAF8EAF9FAF2697F80163A3D6
:10F0F00074A385A396A322893389448955892FA7B0
:10F1000038AB49AB5AABCA01B9010E94B5EC6BAB45
:10F110007CAB8DAB9EAB9B01AC01C701B6010E94DD
:10F1200016ED0E9411F40E9494F42B966CAF7DAF03
:10F130008EAF9FAF2B97F80167AB70AF81AF92AFE7
:10F140009E012F5F3F4F3DAF2CAFAE014F5E5F4F33
:10F1500061965FAF4EAF619761E776E12F967FAF23
:10F160006EAF2F972D965FAF4EAF2D97212C312C80
:10F1700070E879A78FE38BAFACADBDAD2D913D911C
:10F180004D915D91BDAFACAFC701B6010E9416EDC8
:10F190002D96EEADFFAD2D97619371938193919371
:10F1A0002D96FFAFEEAF2D974B015C01E894B7F8B9
:10F1B0002F96AEADBFAD2F974D905D906D907D9029
:10F1C0002F96BFAFAEAF2F97A3019201C501B40137
:10F1D0000E9471F5181694F4A5019401C301B201BF
:10F1E0000E9427F45B018C01910149A55BAD0E944F
:10F1F000B1EC87FF03C0150109A71BAF6196EEAD07
:10F20000FFAD61972CAD3DADE217F30709F0B4CF28
:10F2100020E030E040E85FE3B10189A59BAD0E94AA
:10F22000B1EC87FF4BC07E0131E2E30EF11C619629
:10F230000EAD1FAD6197910149A55BADD8016D91F0
:10F240007D918D919C910E9416EDF80161937193CF
:10F25000819391938F01EE16FF0669F78DE4CDA49B
:10F26000DEA48C9D80018D9D100D11240A53184F32
:10F2700026962CAD3DAD4EAD5FAD2697B10189A56B
:10F280009BAD0E9416EDD80193966D937D938D935F
:10F290009C9396972B966CAD7DAD8EAD9FAD2B97C5
:10F2A0000E94B5EC910149A55BAD0E9416ED0E944C
:10F2B00094F4F80167AB70AF81AF92AF2BA93CA972
:10F2C0004DA95EA922966CAD7DAD8EAD9FAD229706
:10F2D0000E9416ED69A77AA78BA79CA78DE4CDA401
:10F2E000DEA48C9DF0018D9DF00D1124EA53F84FA2
:10F2F00082809380A480B58081149104A104B1041C
:10F3000009F586819781A085B185892B8A2B8B2B66
:10F31000C9F482859385A485B585892B8A2B8B2B8F
:10F3200089F420916D1630916E1640916F165091B0
:10F33000701669A57AA58BA59CA50E9416ED0E9462
:10F3400011F42BC2CFA8D8ACE9ACFAACCD28CE28AA
:10F35000CF2849F06091691670916A1680916B16FA
:10F3600090916C1608C06091651670916616809138
:10F3700067169091681629A53AA54BA55CA50E9431
:10F3800016ED0E9411F40E9494F46B017C018091AF
:10F39000C7169091C816A091C916B091CA162FA58C
:10F3A00038A949A95AA982179307A407B50708F4F1
:10F3B000DEC081149104A104B10421F16091921680
:10F3C0007091931680919416909195166C157D0509
:10F3D0008E059F05B8F40E94DEF22B013C01A701C7
:10F3E0009601C501B4010E94DEF246165706680672
:10F3F000790640F4C301B201A50194010E94EDF227
:10F4000069017A018DE44DA55EA5849FF001859F79
:10F41000F00D1124EA53F84F86809780A084B184C0
:10F4200081149104A104B10441F160919616709188
:10F43000971680919816909199166C157D058E05FA
:10F440009F05D8F42FA538A949A95AA90E94DEF230
:10F450002B013C01A7019601C501B4010E94DEF217
:10F46000461657066806790640F4C301B201A501A5
:10F4700094010E94EDF269017A018DE46DA57EA5EB
:10F48000869FF001879FF00D1124EA53F84F828484
:10F490009384A484B58481149104A104B10441F13E
:10F4A00060919A1670919B1680919C1690919D1672
:10F4B0006C157D058E059F05D8F42FA538A949A99F
:10F4C0005AA90E94DEF22B013C01A7019601C50159
:10F4D000B4010E94DEF2461657066806790640F42B
:10F4E000C301B201A50194010E94EDF269017A0104
:10F4F0008DE4ADA5BEA58A9FF0018B9FF00D112470
:10F50000EA53F84F86849784A088B18881149104C7
:10F51000A104B10409F445C160919E1670919F1633
:10F520008091A0169091A1166C157D058E059F0502
:10F5300008F037C12FA538A949A95AA90E94DEF2BF
:10F540002B013C01A7019601C501B4010E94DEF226
:10F55000461657066806790608F023C1C301B201B2
:10F56000A50194010E94EDF269017A011AC181148A
:10F570009104A104B104B9F16091921670919316AF
:10F5800080919416909195166C157D058E059F05BA
:10F5900050F50E94B5EC2BA93CA94DA95EA90E948B
:10F5A00016ED2B013C01C501B4010E94B7EC4B01E3
:10F5B0005C01C701B6010E94B5ECA50194010E944F
:10F5C00016ED9B01AC01C301B2010E94B1EC87FFB3
:10F5D0000AC0A5019401C301B2010E9427F40E9450
:10F5E00094F46B017C018DE42DA53EA5829FF00172
:10F5F000839FF00D1124EA53F84F468057806084B2
:10F6000071844114510461047104B9F1609196163A
:10F610007091971680919816909199166C157D05AA
:10F620008E059F0550F50E94B5EC2BA93CA94DA96C
:10F630005EA90E9416ED4B015C01C301B2010E945C
:10F64000B7EC2B013C01C701B6010E94B5ECA30148
:10F6500092010E9416ED9B01AC01C501B4010E940C
:10F66000B1EC87FF0AC0A3019201C501B4010E9459
:10F6700027F40E9494F46B017C018DE44DA55EA5F6
:10F68000849FF001859FF00D1124EA53F84F4284C6
:10F690005384648475844114510461047104B9F184
:10F6A00060919A1670919B1680919C1690919D1670
:10F6B0006C157D058E059F0550F50E94B5EC2BA9B4
:10F6C0003CA94DA95EA90E9416ED4B015C01C30146
:10F6D000B2010E94B7EC2B013C01C701B6010E94A8
:10F6E000B5ECA30192010E9416ED9B01AC01C5018E
:10F6F000B4010E94B1EC87FF0AC0A3019201C501C9
:10F70000B4010E9427F40E9494F46B017C018DE403
:10F710006DA57EA5869FF001879FF00D1124EA5309
:10F72000F84F86849784A088B18881149104A1043D
:10F73000B104B9F160919E1670919F168091A01648
:10F740009091A1166C157D058E059F0550F50E94C0
:10F75000B5EC2BA93CA94DA95EA90E9416ED2B0181
:10F760003C01C501B4010E94B7EC4B015C01C7012B
:10F77000B6010E94B5ECA50194010E9416ED9B0113
:10F78000AC01C301B2010E94B1EC87FF0AC0A50120
:10F790009401C301B2010E9427F40E9494F46B010A
:10F7A0007C018DE4ADA5BEA58A9F80018B9F100DC5
:10F7B00011240A53184FF801ED5BFF4FC082D1822C
:10F7C000E282F382C701B6010E94B5EC6B017C01B5
:10F7D00029A53AA54BA55CA50E9427F4A9966CAF74
:10F7E0007DAF8EAF9FAFA997F80163AB74AB85ABCC
:10F7F00096AB20E030E040E85BE4C701B6010E9430
:10F8000016ED20E034E244EF59E40E9427F40E9410
:10F810008FF4D8015E966D937D938D939C93919711
:10F820009396CC909397CFAA9496DC909497DFA66A
:10F830009596EC909597EBAA9696FC90F9A625E5FF
:10F8400036E1AB963FAF2EAFAB972E0131E2430EC0
:10F85000511C55E5252E56E1352E61966EAC7FACD8
:10F860006197CBAEDCAEEEAE2396FFAE239710E0F1
:10F87000D3018D909D90AD90BD903D01E894B7F877
:10F88000F101C190D190E190F1901F01A701960183
:10F89000C501B4010E9471F5181694F5112349F1C0
:10F8A000A70196016FA97FA58BA999A50E9416EDC6
:10F8B0006B017C012BAD3CAD4EAD23965FAD239724
:10F8C000C501B4010E9416ED9B01AC01C701B60150
:10F8D0000E94B1EC87FF13C0A5019401C701B601D6
:10F8E0000E9427F46BAF7CAF8EAF23969FAF239718
:10F8F00006C0CBAEDCAEEEAE2396FFAE239711E092
:10F900004614570409F0B4CF2796FFAD2797F2307D
:10F9100008F499C1C090B3112796CFAE2797D09025
:10F92000B4112896DFAE2897E090B5112C96EFAE73
:10F930002C97F090B6112E96FFAE2E9727E137EB5D
:10F9400041ED58E3B601C7010E9471F518160CF09D
:10F950007AC19601A7016FA97FA58BA999A50E94DD
:10F96000B1EC87FF13C09601A7016FA97FA58BA9F2
:10F9700099A50E9427F4A0966CAF7DAF8EAF9FAF84
:10F98000A0972FA83FA40BA919A524C02FA93FA574
:10F990004BA959A527966FAD279728967FAD289735
:10F9A0002C968FAD2C972E969FAD2E970E9427F404
:10F9B000A0966CAF7DAF8EAF9FAFA09727962FAC70
:10F9C000279728963FAC28972C960FAD2C972E960C
:10F9D0001FAD2E9727EB31E16C963FAF2EAF6C97A2
:10F9E000C12CD12C40E8E42E4FE3F42E6596CCAE2A
:10F9F000DDAEEEAEFFAE65976A961FAE6A976C9667
:10FA0000AEADBFAD6C97CD90DD90ED90FD906C9656
:10FA1000BFAFAEAF6C976196EEADFFAD61978190D1
:10FA20009190A190B1906196FFAFEEAF619727964C
:10FA30002FAD279728963FAD28972C964FAD2C9742
:10FA40002E965FAD2E976FA97FA58BA999A50E94D1
:10FA5000B1EC87FF0CC0A0962CAD3DAD4EAD5FADB7
:10FA6000A097C701B6010E9416ED6B017C016A9652
:10FA7000FFAD6A97FF23C1F065962CAD3DAD4EAD4D
:10FA80005FAD6597C701B6010E9416ED6B017C0161
:10FA900065962CAD3DAD4EAD5FAD6597C501B4012A
:10FAA0000E9416ED4B015C01A5019401C701B6014E
:10FAB0000E9471F520E030E0A90118162CF5C5016F
:10FAC000B4010E9471F518164CF020E030E0A90155
:10FAD000C701B6010E94B1EC87FF05C0A5019401E2
:10FAE000C701B60124C02401350177FA709477F874
:10FAF0007094A3019201C701B6010E9471F5181616
:10FB00005CF52601370128C0C501B4010E94B1ECA3
:10FB100087FD09C020E030E0A901C701B6010E94BD
:10FB200071F518164CF4A7019601C501B4010E94A5
:10FB30004AF32B013C0110C02601370177FA70947B
:10FB400077F87094A3019201C501B4010E94B1EC51
:10FB500087FD02C024013501AB96AEADBFADAB97BA
:10FB6000CD90DD90ED90FD90AB96BFAFAEAFAB9773
:10FB7000A7019601C301B2010E9471F51816ECF4B9
:10FB8000A3019201C701B6010E9427F49B01AC01B9
:10FB900065966CAD7DAD8EAD9FAD65970E9416EDFF
:10FBA00065966CAF7DAF8EAF9FAF65976A96BFAD20
:10FBB0006A97BF5F6A96BFAF6A97E7ECF1E16C9610
:10FBC000CEACDFAC6C97EC15FD0509F018CF6A964A
:10FBD000DFAC6A97DD2061F065962CAD3DAD4EAD92
:10FBE0005FAD6597B101C8010E9416ED1B018C0144
:10FBF00024EA30E74DE75FE3B101C8010E9416ED4A
:10FC00006B017C012091C2163091C3164091C4163D
:10FC10005091C5160E94B1EC87FF28C0A70196013C
:10FC20006BAD7CAD8EAD23969FAD23970E9471F591
:10FC30001816E4F48DE4EDA4FEA48E9DF0018F9DD2
:10FC4000F00D112408C08DE4CDA4DEA48C9DF0013C
:10FC50008D9DF00D1124EA53F84F808184608083DC
:10FC60002BAC3CAC0EAD23961FAD23978DE4EDA4D9
:10FC7000FEA48E9DF0018F9DF00D1124EA53F84FE4
:10FC8000C101D80183A794A7A5A7B6A7A9966CAD73
:10FC90007DAD8EAD9FADA99790589B01AC010E94A0
:10FCA0004BF3A5962CAD3DAD4EAD5FADA5970E9433
:10FCB00016ED9B01AC016BE077ED83E29BE30E94C4
:10FCC0004AF30E94B7F56B017C019B01AC01B101C5
:10FCD000C8010E94B1EC87FD02C0160187018DE4C6
:10FCE0002DA53EA5829FF001839FF00D1124EA53BC
:10FCF000F84FC101D80187A390A7A1A7B2A7B080F0
:10FD00009601A7016FA97FA58BA999A50E94B1ECC7
:10FD1000181614F481E001C083E09DE4CDA4DEA4B4
:10FD20009C9D90019D9D300D1124A9014A53584F6F
:10FD30007A01B82ADA01BC9280E1FE017196A7EB44
:10FD4000B1E101900D928A95E1F78FA99FA5ABA92A
:10FD5000B9A58093B3119093B411A093B511B0934A
:10FD6000B6118BAD9CADAEAD2396BFAD23978093FE
:10FD7000C2169093C316A093C416B093C5162FA9AC
:10FD80003FA54BA959A5BC01CD010E9427F46DA345
:10FD90007EA38FA398A72FA93FA54BA959A5B10171
:10FDA000C8010E9427F469A37AA38BA39CA3AE0188
:10FDB0004B5D5F4FBE016F5D7F4FC7019ED3A19624
:10FDC000CFACA197C092D711AF96CCACDDACEEAC66
:10FDD000FFACAF97C092C711D092C811E092C91181
:10FDE000F092CA11E396CCACDDACEEACFFACE3977D
:10FDF000C092CB11D092CC11E092CD11F092CE11E5
:10FE0000E796CCACDDACEEACFFACE797C092CF117F
:10FE1000D092D011E092D111F092D2116996CCAC6F
:10FE2000DDACEEACFFAC6997C092D311D092D41187
:10FE3000E092D511F092D6118091D7119091D811FE
:10FE4000891B8F70843008F49DC04090D811809138
:10FE5000D71183508F70F82E812C912C00E010E088
:10FE60003DE4532E4F1409F48DC00115110521F006
:10FE7000D8018C9182FD86C08FEF8F0D8F70F82E88
:10FE8000589EC0011124FC01EA53F84FFEA7EDA7CC
:10FE90000115110521F448010DA51EA5E3CF81141C
:10FEA0009104C9F3D8019B967C909B979C96CC902B
:10FEB0009C979D96DC909D979E96EC909E9797962A
:10FEC0002D913D914D915C919A97672D7C2D8D2DB3
:10FED0009E2D0E94B1EC8823F1F2F801608061FC54
:10FEE00042C0D40197968D909D90AD90BC909A970A
:10FEF000A5019401672D7C2D8D2D9E2D0E94B1ECC6
:10FF000018168CF5A5019401C501B4010E9416EDE7
:10FF10004B015C01F80183A994A9A5A9B6A9BC016C
:10FF2000CD0190589B01AC010E944BF3D8019F96E4
:10FF30002D913D914D915C91D2970E9416ED9B01C0
:10FF4000AC01C501B4010E944AF30E94B7F51B0140
:10FF50004C019B01AC01672D7C2D8D2D9E2D0E94A7
:10FF6000B1EC87FF04C0272C3C2C8D2C9E2CC101AA
:10FF7000D401F80187A390A7A1A7B2A7862D81601D
:10FF8000808389CF1091D811F12C00E080E090E0BF
:10FF90002DE4E22E2091D7112117C1F0E19E9001AE
:10FFA0001124A9014A53584F6A01009741F0DC011E
:10FFB0002C9121FD04C06F2D702F0E94C8531F5F2C
:10FFC0001F708F2D902FFC2C0D2DE4CF009741F04A
:10FFD000FC01208121FD04C06F2D702F0E94C853A9
:10FFE000F090D81100E010E08DE4E82E8F2D0F2C5A
:10FFF000000C990B2091D71130E08217930709F478
:020000021000EC
:100000004DC0E89E9001E99E300D1124A9014A538C
:10001000584F6A0101151105D9F1D8012C9120FD25
:1000200004C0FA01208120FF33C0D80193968D903F
:100030009D90AD90BC909697E89EF001E99EF00DE2
:100040001124EA53F84FA501940167A170A581A579
:1000500092A50E9427F469A37AA38BA39CA3A50170
:100060009401F80167A170A581A592A50E9427F4CB
:100070006DA37EA38FA398A7AE014F5D5F4FBE0116
:100080006B5D7F4FC80139D2D8018C918E7F8C93E4
:1000900081E08F0D8F70F82E8601A8CF0115110514
:1000A00061F1F801C3A0D4A0E5A0F6A0A7019601D4
:1000B0006DEC7CEC8CE49DE30E9427F469A37AA3A9
:1000C0008BA39CA3A7019601D80197966D917D9172
:1000D0008D919C919A970E9427F46DA37EA38FA384
:1000E00098A7AE014F5D5F4FBE016B5D7F4FC801AA
:1000F00004D2F80180818E7F808380916F008260BE
:1001000080936F001AC0209085163090861600915B
:100110008716109188169101A80169A57BAD8CAD59
:100120009EAD0E94B1EC87FF02C00C94047729A415
:100130003BAC0CAD1EAD0C940477CA58DF4F0FB624
:10014000F894DEBF0FBECDBFDF91CF911F910F910D
:10015000FF90EF90DF90CF90BF90AF909F908F90E7
:100160007F906F905F904F903F902F9008954F92A7
:100170005F926F927F928F929F92AF92BF92CF9237
:10018000DF92EF92FF92CF93DF93209154162223B8
:1001900009F45DC0EC01C0905016D0905116E0906B
:1001A0005216F090531620E030E0A901C701B601C5
:1001B0000E94B1EC8823B1F02091EA163091EB1641
:1001C0004091EC165091ED16688579858A859B855E
:1001D0000E944AF39B01AC01C701B6010E94B1EC39
:1001E0001816ACF5CE010E94D4AF4B015C01C09053
:1001F0005016D0905116E0905216F0905316209160
:10020000EA163091EB164091EC165091ED16688588
:1002100079858A859B850E944AF3A50194010E94F5
:100220004AF3A70196010E9416ED2B013C01A5019E
:100230009401C701B6010E944AF39B01AC01C301BE
:10024000B2010E9427F4688779878A879B87DF91AC
:10025000CF91FF90EF90DF90CF90BF90AF909F90A5
:100260008F907F906F905F904F9008954F925F9224
:100270006F927F928F929F92AF92BF92CF92DF92B6
:10028000EF92FF920F931F93CF93DF93CDB7DEB71B
:100290002C970FB6F894DEBF0FBECDBF2091541639
:1002A000222309F4A1C08A015B014C014090501641
:1002B00050905116609052167090531620E030E026
:1002C000A901C301B2010E94B1EC882309F44DC019
:1002D0002091EA163091EB164091EC165091ED16F4
:1002E000F80160817181828193810E944AF36B01E0
:1002F0007C019B01AC01C301B2010E94B1EC181654
:100300000CF072C020911D0230911E0240911F021C
:1003100050912002C701B6010E94B1EC882389F1F7
:10032000C0921D02D0921E02E0921F02F0922002A3
:1003300020914C1630914D1640914E1650914F160B
:10034000C701B6010E9416ED9B01AC0160E070E0B0
:1003500080E89FE30E944AF36093190270931A02A7
:1003600080931B0290931C020CC080E090E0A0E8F8
:10037000BFE38093190290931A02A0931B02B093DB
:100380001C02CE0101962CE0FC0111922A95E9F79E
:10039000F401408151816281738149835A836B8367
:1003A0007C83F50140815181628173814D835E833D
:1003B0006F8378870E94D4AF2091190230911A027E
:1003C00040911B0250911C020E9416ED9B01AC0152
:1003D000F80160817181828193810E944BF3F80161
:1003E00060837183828393832C960FB6F894DEBF6B
:1003F0000FBECDBFDF91CF911F910F91FF90EF9076
:10040000DF90CF90BF90AF909F908F907F906F9034
:100410005F904F900895EF92FF920F931F93CF93A9
:10042000DF93CDB7DEB72C970FB6F894DEBF0FBEC3
:10043000CDBF02EB16E184E2E82E86E0F82EF8014B
:1004400021913191419151918F0160E070E080E8FC
:100450009FE30E9427F4F701619371938193919335
:100460007F01F6E1023C1F0751F78091D21690916F
:10047000D316A091D416B091D51689839A83AB83F5
:10048000BC838091D6169091D716A091D816B091C2
:10049000D9168D839E83AF83B8878091DA169091A9
:1004A000DB16A091DC16B091DD1689879A87AB87A1
:1004B000BC87AE01475F5F4FBE016B5F7F4FCE01D0
:1004C0000196D4DE2EED36E1AE01475F5F4FBE01EF
:1004D0006B5F7F4FCE0101960E945A730E94FF729C
:1004E0002C960FB6F894DEBF0FBECDBFDF91CF9133
:1004F0001F910F91FF90EF9008954F925F926F922E
:100500007F928F929F92AF92BF92CF92DF92EF92A3
:10051000FF920F931F93CF93DF93CDB7DEB76A9708
:100520000FB6F894DEBF0FBECDBF9A8F898F5B01E7
:100530008A01DC01D7966D917D918D919C91DA971E
:100540000E94B5EC6B017C01F50120813181428173
:1005500053810E9416ED0E9411F40E9494F4698761
:100560007A878B879C87D8012D913D914D915C9125
:10057000C701B6010E9416ED0E9411F40E9494F486
:100580006D877E878F87988B29853A854B855C851B
:10059000283731054105510540F488E790E0A0E097
:1005A000B0E089879A87AB87BC872D853E854F85CC
:1005B0005889283731054105510540F488E790E016
:1005C000A0E0B0E08D879E87AF87B88BE98DFA8D6C
:1005D000ED5BFF4F20813181428153812D833E832A
:1005E0004F835887CA01B9010E94B7EC69837A83A7
:1005F0008B839C8369857A858B859C850E94B5EC6D
:10060000698B7A8B8B8B9C8B20E030E0A901698110
:100610007A818B819C810E94B1EC882339F1A701FA
:100620009601C701B6010E9416ED4B015C012989B4
:100630003A894B895C89CA01B9010E9416ED9B0178
:10064000AC01C501B4010E944AF34B015C01298150
:100650003A814B815C81CA01B9010E944BF39B0135
:10066000AC01C501B4010E9427F403C060E070E052
:10067000CB010E9411F40E948FF42B013C016D818B
:100680007E818F81988590958095709561957F4F3B
:100690008F4F9F4F0E94B7EC4B015C016D857E85AB
:1006A0008F8598890E94B5EC6D837E838F839887B0
:1006B00020E030E0A901C501B4010E94B1EC88231B
:1006C00049F12D813E814F815885CA01B9010E94AF
:1006D00016ED6D8B7E8B8F8B988FA7019601C701CE
:1006E000B6010E9416ED9B01AC016D897E898F8950
:1006F000988D0E944AF36B017C01A5019401C5010C
:10070000B4010E944BF39B01AC01C701B6010E94EA
:1007100027F403C060E070E0CB010E94C0F4A98D13
:10072000BA8D52968D909D90AD90BC905597750165
:100730006401C418D508E608F7080E948FF4C61AA9
:10074000D70AE80AF90AF7FE6BC020E030E0A901F9
:1007500069817A818B819C810E94B1EC882309F4A4
:1007600047C0C501B4010E94B5EC6B017C01298131
:100770003A814B815C81CA01B9010E944BF39B0114
:10078000AC01C701B6010E9416ED6B017C012989FD
:100790003A894B895C89CA01B9010E9416ED9B0117
:1007A000AC01C701B6010E944AF36B017C012D81A7
:1007B0003E814F815885CA01B9010E9416ED9B0107
:1007C000AC01C701B6010E944BF36B017C0120E034
:1007D00030E040E850E469817A818B819C810E94FD
:1007E00016ED9B01AC01C701B6010E9427F403C0BE
:1007F00060E070E0CB010E9411F40E948FF42B01A5
:100800003C0197FF03C0412C512C3201481459047C
:100810006A047B0410F024013501C12CD12C76012F
:100820008FB7F894E98DFA8D908193FD1DC0468AAB
:10083000578A608E718EC40CD51CE61CF71CC28EC4
:10084000D38EE48EF58E29853A854B855C8523AF62
:1008500034AF45AF56AFFF962D853E854F855889FD
:1008600020833183428353838FBF6A960FB6F894F7
:10087000DEBF0FBECDBFDF91CF911F910F91FF90D3
:10088000EF90DF90CF90BF90AF909F908F907F9030
:100890006F905F904F9008950F931F93CF93DF93C6
:1008A000E091DE1BF091DF1B4281538164817581F1
:1008B000141615061606170614F52091960C20FD41
:1008C0001EC03CB12091D11635FB882780F990E0FD
:1008D000919581959109822780719927822780932C
:1008E000D1169091D0169071892349F080914006DD
:1008F00080618093400680E090E00E94F8D6E0910D
:10090000DE1BF091DF1B86819781A085B1851816CB
:1009100019061A061B061CF58091960C81FD1FC056
:10092000909103018091D11691FB002700F910E00E
:1009300011950195110908270072112708270093C6
:10094000D1168091D0168072082349F0809140061C
:1009500080628093400681E090E00E94F8D6E091AA
:10096000DE1BF091DF1B82859385A485B585181663
:1009700019061A061B0644F58091960C82FF24C0C6
:1009800080910F06882301F199B18091D11693FBD4
:10099000992790F9C92F90E0D92FD195C195D10908
:1009A000C827C470DD27C827C093D1168091D01600
:1009B0008470C82349F0809140068460809340068B
:1009C00082E090E00E94F8D68091D1168093D016F4
:1009D000DF91CF911F910F910895CF93DF93E3E9BA
:1009E000F7E18491EF012196882321F00E9417D925
:1009F000FE01F7CFEBE8F7E18491EF012196882320
:100A000021F00E9417D9FE01F7CF659903C0C6E314
:100A1000D4E002C0CBE3D4E08991882319F00E948E
:100A200017D9FACF8AE00E9417D9E3E8F7E1849159
:100A3000EF012196882321F00E9417D9FE01F7CFFC
:100A40008091030181FD03C0C6E3D4E002C0CBE383
:100A5000D4E08991882319F00E9417D9FACF8AE04F
:100A60000E9417D9EBE7F7E18491EF0121968823E3
:100A700021F00E9417D9FE01F7CF4B9903C0C6E3BE
:100A8000D4E002C0CBE3D4E08991882319F00E941E
:100A900017D9FACF8AE0DF91CF910C9417D90F9331
:100AA0001F93CF93C82F882319F0E3E6F7E10CC01A
:100AB000E2EBF2E184918F010F5F1F4F8823A9F3CE
:100AC0000E9417D9F801F6CF84918F010F5F1F4F55
:100AD000882321F00E9417D9F801F6CFCC2319F012
:100AE000E6E4F7E10CC0E2EBF2E184918F010F5FE5
:100AF0001F4F8823A9F30E9417D9F801F6CF8491DC
:100B00008F010F5F1F4F882321F00E9417D9F80132
:100B1000F6CF8AE00E9417D9C1112CC0E2EBF2E1B6
:100B200084918F010F5F1F4F882321F00E9417D9F6
:100B3000F801F6CFE3E3F7E184918F010F5F1F4FD8
:100B4000882321F00E9417D9F801F6CF8091CF16A3
:100B5000882321F08AE00E9417D93AC0E8E2F7E141
:100B600084918F010F5F1F4F882391F10E9417D945
:100B7000F801F6CF4091CB165091CC166091CD166E
:100B80007091CE168FE197E10E9477538AE00E9420
:100B900017D98091CF16811127C0CC2319F0E4E139
:100BA000F7E10CC0E2EBF2E184918F010F5F1F4F80
:100BB0008823A9F30E9417D9F801F6CF84918F01F9
:100BC0000F5F1F4F882381F00E9417D9F801F6CFDD
:100BD000E2EBF2E184918F010F5F1F4F882351F206
:100BE0000E9417D9F801F6CFC11124C0E2EBF2E15F
:100BF00084918F010F5F1F4F882321F00E9417D926
:100C0000F801F6CFE3E0F7E184918F010F5F1F4F0A
:100C1000882321F00E9417D9F801F6CFE2EBF2E128
:100C200084918F010F5F1F4F882321F00E9417D9F5
:100C3000F801F6CF4091B2165091B3166091B416F8
:100C40007091B5168BEF96E10E9477534091B616DE
:100C50005091B7166091B8167091B91688EF96E169
:100C60000E9477534091BA165091BB166091BC1602
:100C70007091BD1685EF96E10E9477534091BE16A4
:100C80005091BF166091C0167091C11682EF96E127
:100C90000E9477538AE00E9417D9C11124C0E2EB69
:100CA000F2E184918F010F5F1F4F882321F00E9492
:100CB00017D9F801F6CFE4EDF6E184918F010F5FCB
:100CC0001F4F882321F00E9417D9F801F6CFE2EBDD
:100CD000F2E184918F010F5F1F4F882321F00E9462
:100CE00017D9F801F6CF40917116509172166091A4
:100CF0007316709174168BEC96E10E9477534091B5
:100D0000751650917616609177167091781688EC6A
:100D100096E10E9477534091791650917A1660912E
:100D20007B1670917C1685EC96E10E94775340917A
:100D30007D1650917E1660917F167091801682EC20
:100D400096E10E9477538AE00E9417D9C11124C00E
:100D5000E2EBF2E184918F010F5F1F4F882321F0B6
:100D60000E9417D9F801F6CFE0EAF6E184918F01ED
:100D70000F5F1F4F882321F00E9417D9F801F6CF8B
:100D8000E2EBF2E184918F010F5F1F4F882321F086
:100D90000E9417D9F801F6CF4091A2165091A316E0
:100DA0006091A4167091A51687E996E10E945A53A6
:100DB0004091A6165091A7166091A8167091A91699
:100DC00084E996E10E945A534091AA165091AB16BD
:100DD0006091AC167091AD1681E996E10E945A536C
:100DE0004091AE165091AF166091B0167091B11649
:100DF0008EE896E10E945A538AE00E9417D9C111E9
:100E000024C0E2EBF2E184918F010F5F1F4F882332
:100E100021F00E9417D9F801F6CFE4E4F6E18491BD
:100E20008F010F5F1F4F882321F00E9417D9F8010F
:100E3000F6CFE2EBF2E184918F010F5F1F4F882321
:100E400021F00E9417D9F801F6CF40916916509110
:100E50006A1660916B1670916C168BE396E10E9496
:100E6000775340916D1650916E1660916F16709188
:100E7000701688E396E10E94775340916516509171
:100E80006616609167167091681685E396E10E9478
:100E900077538AE00E9417D9C11124C0E2EBF2E136
:100EA00084918F010F5F1F4F882321F00E9417D973
:100EB000F801F6CFE1ECF5E184918F010F5F1F4F50
:100EC000882321F00E9417D9F801F6CFE2EBF2E176
:100ED00084918F010F5F1F4F882321F00E9417D943
:100EE000F801F6CF4091891650918A1660918B16C1
:100EF00070918C1688EB95E10E947753409185168E
:100F000050918616609187167091881685EB95E151
:100F10000E947753409181165091821660918316FA
:100F20007091841682EB95E10E945A5340915516B8
:100F30005091561660915716709158168FEA95E1A8
:100F40000E9477534091591650915A1660915B1642
:100F500070915C168CEA95E10E94775340915D1682
:100F600050915E1660915F167091601689EA95E166
:100F70000E947753409161165091621660916316FA
:100F80007091641686EA95E10E9477538AE00E9488
:100F900017D9C11124C0E2EBF2E184918F010F5FF8
:100FA0001F4F882321F00E9417D9F801F6CFE8E9F6
:100FB000F5E184918F010F5F1F4F882321F00E947C
:100FC00017D9F801F6CFE2EBF2E184918F010F5FC0
:100FD0001F4F882321F00E9417D9F801F6CF4091C6
:100FE00010065091110660911206709113068FE859
:100FF00095E10E9477534091140650911506609137
:101000001606709117068CE895E10E94775340917F
:1010100018065091190660911A0670911B0689E80E
:1010200095E10E9477538AE00E9417D9C11124C02C
:10103000E2EBF2E184918F010F5F1F4F882321F0D3
:101040000E9417D9F801F6CFE5E7F5E184918F0109
:101050000F5F1F4F882321F00E9417D9F801F6CFA8
:10106000E2EBF2E184918F010F5F1F4F882321F0A3
:101070000E9417D9F801F6CF6091541670E08CE603
:1010800095E10E94945340915016509151166091F1
:1010900052167091531689E695E10E9477538AE0C3
:1010A0000E9417D9C11124C0E2EBF2E184918F01B3
:1010B0000F5F1F4F882321F00E9417D9F801F6CF48
:1010C000EAE5F5E184918F010F5F1F4F882321F03E
:1010D0000E9417D9F801F6CFE2EBF2E184918F017B
:1010E0000F5F1F4F882321F00E9417D9F801F6CF18
:1010F0004091F41B5091F51B6091F61B7091F71B0A
:1011000081E595E10E9477532CEA35EC47E25EE3F6
:101110006091F01B7091F11B8091F21B9091F31B79
:101120000E9427F4AB01BC018EE495E10E94775345
:101130002CEA35EC47E25EE36091FA1B7091FB1BF1
:101140008091FC1B9091FD1B0E9416EDAB01BC0130
:101150008BE495E10E9477538AE00E9417D9C11170
:1011600024C0E2EBF2E184918F010F5F1F4F8823CF
:1011700021F00E9417D9F801F6CFE5E3F5E184915B
:101180008F010F5F1F4F882321F00E9417D9F801AC
:10119000F6CFE2EBF2E184918F010F5F1F4F8823BE
:1011A00021F00E9417D9F801F6CF40912E175091E7
:1011B0002F1760913017709131178CE295E10E94E2
:1011C00077538AE0CF911F910F910C9417D9EF922A
:1011D000FF921F93CF93DF9389E40E94FBD888236B
:1011E00021F00E9465D8C62F01C0CFEF8AE40E948B
:1011F000FBD8882321F00E9465D8D62F01C0DFEFED
:101200008AE50E94CCD8F82E811105C081E50E94A4
:10121000CCD8182F01C010E0C7FD06C0D7FD04C010
:10122000F1101AC0111118C0ECE7F2E18491EF013E
:101230002196811103C0ECE2FBE104C00E9417D9A2
:10124000FE01F4CF8491EF012196882309F44FC069
:101250000E9417D9FE01F6CFC43010F4D430B8F094
:10126000ECE7F2E18491EF012196811103C0EDE0FA
:10127000FBE104C00E9417D9FE01F4CF8491EF0175
:1012800021968823A1F10E9417D9FE01F7CFEC2EF9
:10129000CC0FFF08CD2FDD0FDD0B0E9495D89B01F1
:1012A000AC01D701AA0FBB1FAA0FBB1F112371F0FE
:1012B000FD01EC0FFD1FEE0FFF1FEE0FFF1FE251B0
:1012C000F94E608171818281938103C060E070E09A
:1012D000CB01CA0FDB1FCC0FDD1FCC0FDD1FC251AE
:1012E000D94E0E944BF3688379838A839B83DF9175
:1012F000CF911F91FF90EF900895CF92DF92EF92E0
:10130000FF92CF93DF9386E50E94CCD8882341F0EB
:101310008091731A9091741A892B11F00E942156B2
:1013200083E50E94CCD8C82F882319F00E9486D864
:10133000C82F83E50E94CCD8882319F08C2F0E94F7
:10134000716B8AE50E94CCD8882321F00E9495D841
:101350000E944B5DF0905416C11103C0E2EBF2E124
:1013600018C0F110FBCFECE7F2E18491EF01219678
:10137000882321F00E9417D9FE01F7CFEEEEFAE1A3
:101380008491EF012196882349F30E9417D9FE0129
:10139000F7CF8491EF012196882321F00E9417D97D
:1013A000FE01F7CFF11003C069E474E002C065E408
:1013B00074E080EE9AE10E94AD538AE00E9417D952
:1013C000E2EBF2E18491EF012196882321F00E9463
:1013D00017D9FE01F7CFE3EDFAE18491EF012196F1
:1013E000882321F00E9417D9FE01F7CFC090501634
:1013F000D0905116E0905216F090531620E030E055
:10140000A901C701B6010E9471F5181674F442E0F3
:10141000C701B6010E94A3D98AE0DF91CF91FF9066
:10142000EF90DF90CF900C9417D9EEECFAE1849115
:10143000EF012196882321F00E9417D9FE01F7CFF2
:10144000DF91CF91FF90EF90DF90CF90089588E8E3
:1014500093E19093980C8093970C80916F008D7F0F
:1014600080936F009091D7118091D811981719F03F
:101470000E94184BF7CF1092DF1B1092DE1B809159
:101480006F00826080936F008FB7F8941092C2074C
:101490001092C3071092C4071092C5078FBF0E9415
:1014A0003AD784E690E00E9488AF0C941ED883E57A
:1014B0000E94CCD8882351F00E9495D86093891659
:1014C00070938A1680938B1690938C1684E50E94F5
:1014D000CCD8882351F00E9495D8609385167093DC
:1014E0008616809387169093881682E40E94CCD843
:1014F0008823C1F080918C0590918D05009739F07B
:101500004AE050E060E070E00E9430EB03C060E031
:1015100070E0CB01609381167093821680938316DE
:101520009093841688E50E94CCD8882351F00E94BD
:1015300095D86093551670935616809357169093CE
:10154000581689E50E94CCD8882351F00E9495D87E
:101550006093591670935A1680935B1690935C169D
:101560008AE50E94CCD8882351F00E9495D86093D8
:101570005D1670935E1680935F169093601685E4F7
:101580000E94CCD8882351F00E9495D860936116B0
:101590007093621680936316909364160895CF93A8
:1015A000DF93E8E8F8E18491EF012196882321F0A8
:1015B0000E9417D9FE01F7CFEAE7F8E18491EF0125
:1015C0002196882321F00E9417D9FE01F7CFE3E688
:1015D000F8E18491EF012196882321F00E9417D928
:1015E000FE01F7CFE3E5F8E18491EF01219688232E
:1015F00021F00E9417D9FE01F7CFE2E4F8E18491CF
:10160000EF012196882321F00E9417D9FE01F7CF20
:10161000E1E3F8E18491EF012196882321F00E9413
:1016200017D9FE01F7CFE2E2F8E18491EF012196AC
:10163000882321F00E9417D9FE01F7CFEDE0F8E1F1
:101640008491EF012196882321F00E9417D9FE0191
:10165000F7CFE7EFF7E18491EF012196882321F09E
:101660000E9417D9FE01F7CFE2EEF7E18491EF0176
:101670002196882321F00E9417D9FE01F7CFE5ECCF
:10168000F7E18491EF012196882321F00E9417D978
:10169000FE01F7CFEDEAF7E18491EF01219688236F
:1016A00021F00E9417D9FE01F7CFDF91CF91089565
:1016B0002F923F924F925F926F927F928F929F9262
:1016C000AF92BF92CF92DF92EF92FF920F931F9350
:1016D000CF93DF93CDB7DEB7E0970FB6F894DEBFB8
:1016E0000FBECDBF85E40E94FBD8882329F00E945D
:1016F00065D87A83698302C01A82198283E40E94C2
:10170000FBD8882329F00E9465D879A768A704C070
:1017100025E030E039A728A785E50E94CCD88F8F37
:10172000882319F00E9486D88F8F49815A8157FDEE
:1017300007C0C12CD12CB6E1EB2EB3E4FB2E06C0C2
:10174000C12CD12CACE8EA2EA2E4FA2E83E50E944B
:10175000FBD8882321F00E9495D86B017C018981F8
:101760009A81892B11F4109292050E940CDC4B0196
:101770005C01A981BA81AB2B49F1EDE4F4E0FA8375
:10178000E983A981BA818D91BA83A983882319F04D
:101790000E9417D9F6CF8AE0E0960FB6F894DEBF24
:1017A0000FBECDBFDF91CF911F910F91FF90EF90B2
:1017B000DF90CF90BF90AF909F908F907F906F9071
:1017C0005F904F903F902F900C9417D9E6E7F4E08C
:1017D000FA83E983A981BA818D91BA83A983882389
:1017E00019F00E9417D9F6CFC701B6010E948FF4F5
:1017F000072E000C880B990B0E94B7EC6B877C8737
:101800008D879E878AE00E9417D90E94EDC68FE7D8
:101810008093B81B81E080933D0288A299A2AAA27E
:10182000BBA28AA69BA6ACA6BDA61F86B0E4B88BB9
:10183000ECE1E98BF6E4FA8B1B8A1C8A1D8A1E8A6E
:101840001B8E1C8E1D8E1E8E1F8A188E198E1A8E50
:10185000412C512C3201FFE7CF2ED12CE12CF12C61
:101860002FE730E040E050E02D833E834F835887E0
:101870001CA21DA21EA21FA231E03EA71A86198635
:10188000212C312C00E010E080913D02882309F4E6
:1018900085C10E940CDC69837A838B839C83809151
:1018A000B61B882309F484C00E94A8C72090FC05B9
:1018B0003090FD050091FE051091FF052B893C89B4
:1018C0004D895E89B101C8010E9471F5181624F492
:1018D0002B8A3C8A0D8B1E8B2F85388949895A8922
:1018E000B101C8010E94B1EC87FF04C02F86388A7D
:1018F000098B1A8B4EA591014423E9F1A8016B8550
:101900007C858D859E850E94B1EC87FF51C0498101
:101910005A816B817C81481959096A097B09DB016D
:10192000CA0188589341A109B109B7FD41C08D8111
:101930009E81AF81B8858C199D09AE09BF09B59507
:10194000A795979587958093B81B4CA35DA36EA32D
:101950007FA35B855B8B8C858C8B9D859D8BAE85FA
:10196000AE8B29813A814B815C8128A339A34AA39C
:101970005BA31EA61DC0A8016B857C858D859E85F9
:101980000E9471F51816A4F489819A81AB81BC81FB
:1019900028A139A14AA15BA1821B930BA40BB50B13
:1019A000AC01BD01485853416109710977FF14C169
:1019B00020E030E040EA51E46B857C858D859E8592
:1019C0000E944BF39101A8010E94B1EC87FF10C067
:1019D000EAE5FAE184919F012F5F3F4F3A83298323
:1019E000882309F445C20E9417D9E981FA81F2CF10
:1019F00080E398EFAFEFBFEF2AA53BA54CA55DA50F
:101A0000821B930BA40BB50B29813A814B815C811E
:101A1000820F931FA41FB51FB7FD0DC00E94875EE4
:101A20008AE00E9417D989819A81AB81BC818AA7FB
:101A30009BA7ACA7BDA789819A81AB81BC81880F88
:101A4000991FAA1FBB1F28A139A14AA15BA1821B14
:101A5000930BA40BB50B88199909AA09BB0981340A
:101A60009747AB41B10580F181E09AE590937E15EF
:101A700080937D1589E590E09093801580937F1584
:101A800087E08093711582E88093741584E890E074
:101A9000A0E0B0E08093751590937615A09377152C
:101AA000B09378150E945666ECE3FAE18491AF0199
:101AB0004F5F5F4F5A834983882309F4D9C10E943D
:101AC00017D9E981FA81F2CF88A599A5A985BA85A8
:101AD0008A179B070CF05FC0EFEDF9E184919F013D
:101AE0002F5F3F4F3A832983882329F00E9417D91B
:101AF000E981FA81F3CFB301A2018AEC99E10E9456
:101B000077538AE00E9417D94F89588D698D7A8D55
:101B100085EB99E10E9477538AE00E9417D94B8D9B
:101B20005C8D6D8D7E8D80EA99E10E9477538AE00D
:101B30000E9417D93F8D332309F49AC14092F41BB8
:101B40005092F51B6092F61B7092F71B2CEA35EC55
:101B500047E25EE36F89788D898D9A8D0E9416ED3C
:101B60006093F01B7093F11B8093F21B9093F31B17
:101B70002CEA35EC47E25EE36B8D7C8D8D8D9E8D7E
:101B80000E9427F46093FA1B7093FB1B8093FC1B4D
:101B90009093FD1B6DC10E949F2A76CE80913D02DD
:101BA000811166C1E0960FB6F894DEBF0FBECDBFBF
:101BB000DF91CF911F910F91FF90EF90DF90CF9029
:101BC000BF90AF909F908F907F906F905F904F905D
:101BD0003F902F900C94EDC649855A851416150632
:101BE0000CF024C18CA09DA0AEA0BFA0880E991EB1
:101BF000AA1EBB1E2CA13DA14EA15FA1281B390B23
:101C00004A0B5B0BC701B6010E94DEF2A5019401ED
